
_icubelrwan_and_gpio_interrupt3.elf:     file format elf32-littlearm

Sections:
Idx Name          Size      VMA       LMA       File off  Algn
  0 .isr_vector   000000c0  08000000  08000000  00010000  2**0
                  CONTENTS, ALLOC, LOAD, READONLY, DATA
  1 .text         0001a14c  080000c0  080000c0  000100c0  2**2
                  CONTENTS, ALLOC, LOAD, READONLY, CODE
  2 .rodata       00001110  0801a20c  0801a20c  0002a20c  2**2
                  CONTENTS, ALLOC, LOAD, READONLY, DATA
  3 .ARM.extab    00000000  0801b31c  0801b31c  0003017c  2**0
                  CONTENTS
  4 .ARM          00000008  0801b31c  0801b31c  0002b31c  2**2
                  CONTENTS, ALLOC, LOAD, READONLY, DATA
  5 .preinit_array 00000000  0801b324  0801b324  0003017c  2**0
                  CONTENTS, ALLOC, LOAD, DATA
  6 .init_array   00000004  0801b324  0801b324  0002b324  2**2
                  CONTENTS, ALLOC, LOAD, DATA
  7 .fini_array   00000004  0801b328  0801b328  0002b328  2**2
                  CONTENTS, ALLOC, LOAD, DATA
  8 .data         0000017c  20000000  0801b32c  00030000  2**2
                  CONTENTS, ALLOC, LOAD, DATA
  9 .bss          00001444  2000017c  0801b4a8  0003017c  2**2
                  ALLOC
 10 ._user_heap_stack 00000600  200015c0  0801b4a8  000315c0  2**0
                  ALLOC
 11 .ARM.attributes 00000028  00000000  00000000  0003017c  2**0
                  CONTENTS, READONLY
 12 .debug_info   0003ca38  00000000  00000000  000301a4  2**0
                  CONTENTS, READONLY, DEBUGGING
 13 .debug_abbrev 00008197  00000000  00000000  0006cbdc  2**0
                  CONTENTS, READONLY, DEBUGGING
 14 .debug_aranges 000021d0  00000000  00000000  00074d78  2**3
                  CONTENTS, READONLY, DEBUGGING
 15 .debug_ranges 00001e88  00000000  00000000  00076f48  2**3
                  CONTENTS, READONLY, DEBUGGING
 16 .debug_macro  00023516  00000000  00000000  00078dd0  2**0
                  CONTENTS, READONLY, DEBUGGING
 17 .debug_line   0002c841  00000000  00000000  0009c2e6  2**0
                  CONTENTS, READONLY, DEBUGGING
 18 .debug_str    000a7a5a  00000000  00000000  000c8b27  2**0
                  CONTENTS, READONLY, DEBUGGING
 19 .comment      0000007b  00000000  00000000  00170581  2**0
                  CONTENTS, READONLY
 20 .debug_frame  00007c64  00000000  00000000  001705fc  2**2
                  CONTENTS, READONLY, DEBUGGING

Disassembly of section .text:

080000c0 <__do_global_dtors_aux>:
 80000c0:	b510      	push	{r4, lr}
 80000c2:	4c06      	ldr	r4, [pc, #24]	; (80000dc <__do_global_dtors_aux+0x1c>)
 80000c4:	7823      	ldrb	r3, [r4, #0]
 80000c6:	2b00      	cmp	r3, #0
 80000c8:	d107      	bne.n	80000da <__do_global_dtors_aux+0x1a>
 80000ca:	4b05      	ldr	r3, [pc, #20]	; (80000e0 <__do_global_dtors_aux+0x20>)
 80000cc:	2b00      	cmp	r3, #0
 80000ce:	d002      	beq.n	80000d6 <__do_global_dtors_aux+0x16>
 80000d0:	4804      	ldr	r0, [pc, #16]	; (80000e4 <__do_global_dtors_aux+0x24>)
 80000d2:	e000      	b.n	80000d6 <__do_global_dtors_aux+0x16>
 80000d4:	bf00      	nop
 80000d6:	2301      	movs	r3, #1
 80000d8:	7023      	strb	r3, [r4, #0]
 80000da:	bd10      	pop	{r4, pc}
 80000dc:	2000017c 	.word	0x2000017c
 80000e0:	00000000 	.word	0x00000000
 80000e4:	0801a1f4 	.word	0x0801a1f4

080000e8 <frame_dummy>:
 80000e8:	4b04      	ldr	r3, [pc, #16]	; (80000fc <frame_dummy+0x14>)
 80000ea:	b510      	push	{r4, lr}
 80000ec:	2b00      	cmp	r3, #0
 80000ee:	d003      	beq.n	80000f8 <frame_dummy+0x10>
 80000f0:	4903      	ldr	r1, [pc, #12]	; (8000100 <frame_dummy+0x18>)
 80000f2:	4804      	ldr	r0, [pc, #16]	; (8000104 <frame_dummy+0x1c>)
 80000f4:	e000      	b.n	80000f8 <frame_dummy+0x10>
 80000f6:	bf00      	nop
 80000f8:	bd10      	pop	{r4, pc}
 80000fa:	46c0      	nop			; (mov r8, r8)
 80000fc:	00000000 	.word	0x00000000
 8000100:	20000180 	.word	0x20000180
 8000104:	0801a1f4 	.word	0x0801a1f4

08000108 <__udivsi3>:
 8000108:	2200      	movs	r2, #0
 800010a:	0843      	lsrs	r3, r0, #1
 800010c:	428b      	cmp	r3, r1
 800010e:	d374      	bcc.n	80001fa <__udivsi3+0xf2>
 8000110:	0903      	lsrs	r3, r0, #4
 8000112:	428b      	cmp	r3, r1
 8000114:	d35f      	bcc.n	80001d6 <__udivsi3+0xce>
 8000116:	0a03      	lsrs	r3, r0, #8
 8000118:	428b      	cmp	r3, r1
 800011a:	d344      	bcc.n	80001a6 <__udivsi3+0x9e>
 800011c:	0b03      	lsrs	r3, r0, #12
 800011e:	428b      	cmp	r3, r1
 8000120:	d328      	bcc.n	8000174 <__udivsi3+0x6c>
 8000122:	0c03      	lsrs	r3, r0, #16
 8000124:	428b      	cmp	r3, r1
 8000126:	d30d      	bcc.n	8000144 <__udivsi3+0x3c>
 8000128:	22ff      	movs	r2, #255	; 0xff
 800012a:	0209      	lsls	r1, r1, #8
 800012c:	ba12      	rev	r2, r2
 800012e:	0c03      	lsrs	r3, r0, #16
 8000130:	428b      	cmp	r3, r1
 8000132:	d302      	bcc.n	800013a <__udivsi3+0x32>
 8000134:	1212      	asrs	r2, r2, #8
 8000136:	0209      	lsls	r1, r1, #8
 8000138:	d065      	beq.n	8000206 <__udivsi3+0xfe>
 800013a:	0b03      	lsrs	r3, r0, #12
 800013c:	428b      	cmp	r3, r1
 800013e:	d319      	bcc.n	8000174 <__udivsi3+0x6c>
 8000140:	e000      	b.n	8000144 <__udivsi3+0x3c>
 8000142:	0a09      	lsrs	r1, r1, #8
 8000144:	0bc3      	lsrs	r3, r0, #15
 8000146:	428b      	cmp	r3, r1
 8000148:	d301      	bcc.n	800014e <__udivsi3+0x46>
 800014a:	03cb      	lsls	r3, r1, #15
 800014c:	1ac0      	subs	r0, r0, r3
 800014e:	4152      	adcs	r2, r2
 8000150:	0b83      	lsrs	r3, r0, #14
 8000152:	428b      	cmp	r3, r1
 8000154:	d301      	bcc.n	800015a <__udivsi3+0x52>
 8000156:	038b      	lsls	r3, r1, #14
 8000158:	1ac0      	subs	r0, r0, r3
 800015a:	4152      	adcs	r2, r2
 800015c:	0b43      	lsrs	r3, r0, #13
 800015e:	428b      	cmp	r3, r1
 8000160:	d301      	bcc.n	8000166 <__udivsi3+0x5e>
 8000162:	034b      	lsls	r3, r1, #13
 8000164:	1ac0      	subs	r0, r0, r3
 8000166:	4152      	adcs	r2, r2
 8000168:	0b03      	lsrs	r3, r0, #12
 800016a:	428b      	cmp	r3, r1
 800016c:	d301      	bcc.n	8000172 <__udivsi3+0x6a>
 800016e:	030b      	lsls	r3, r1, #12
 8000170:	1ac0      	subs	r0, r0, r3
 8000172:	4152      	adcs	r2, r2
 8000174:	0ac3      	lsrs	r3, r0, #11
 8000176:	428b      	cmp	r3, r1
 8000178:	d301      	bcc.n	800017e <__udivsi3+0x76>
 800017a:	02cb      	lsls	r3, r1, #11
 800017c:	1ac0      	subs	r0, r0, r3
 800017e:	4152      	adcs	r2, r2
 8000180:	0a83      	lsrs	r3, r0, #10
 8000182:	428b      	cmp	r3, r1
 8000184:	d301      	bcc.n	800018a <__udivsi3+0x82>
 8000186:	028b      	lsls	r3, r1, #10
 8000188:	1ac0      	subs	r0, r0, r3
 800018a:	4152      	adcs	r2, r2
 800018c:	0a43      	lsrs	r3, r0, #9
 800018e:	428b      	cmp	r3, r1
 8000190:	d301      	bcc.n	8000196 <__udivsi3+0x8e>
 8000192:	024b      	lsls	r3, r1, #9
 8000194:	1ac0      	subs	r0, r0, r3
 8000196:	4152      	adcs	r2, r2
 8000198:	0a03      	lsrs	r3, r0, #8
 800019a:	428b      	cmp	r3, r1
 800019c:	d301      	bcc.n	80001a2 <__udivsi3+0x9a>
 800019e:	020b      	lsls	r3, r1, #8
 80001a0:	1ac0      	subs	r0, r0, r3
 80001a2:	4152      	adcs	r2, r2
 80001a4:	d2cd      	bcs.n	8000142 <__udivsi3+0x3a>
 80001a6:	09c3      	lsrs	r3, r0, #7
 80001a8:	428b      	cmp	r3, r1
 80001aa:	d301      	bcc.n	80001b0 <__udivsi3+0xa8>
 80001ac:	01cb      	lsls	r3, r1, #7
 80001ae:	1ac0      	subs	r0, r0, r3
 80001b0:	4152      	adcs	r2, r2
 80001b2:	0983      	lsrs	r3, r0, #6
 80001b4:	428b      	cmp	r3, r1
 80001b6:	d301      	bcc.n	80001bc <__udivsi3+0xb4>
 80001b8:	018b      	lsls	r3, r1, #6
 80001ba:	1ac0      	subs	r0, r0, r3
 80001bc:	4152      	adcs	r2, r2
 80001be:	0943      	lsrs	r3, r0, #5
 80001c0:	428b      	cmp	r3, r1
 80001c2:	d301      	bcc.n	80001c8 <__udivsi3+0xc0>
 80001c4:	014b      	lsls	r3, r1, #5
 80001c6:	1ac0      	subs	r0, r0, r3
 80001c8:	4152      	adcs	r2, r2
 80001ca:	0903      	lsrs	r3, r0, #4
 80001cc:	428b      	cmp	r3, r1
 80001ce:	d301      	bcc.n	80001d4 <__udivsi3+0xcc>
 80001d0:	010b      	lsls	r3, r1, #4
 80001d2:	1ac0      	subs	r0, r0, r3
 80001d4:	4152      	adcs	r2, r2
 80001d6:	08c3      	lsrs	r3, r0, #3
 80001d8:	428b      	cmp	r3, r1
 80001da:	d301      	bcc.n	80001e0 <__udivsi3+0xd8>
 80001dc:	00cb      	lsls	r3, r1, #3
 80001de:	1ac0      	subs	r0, r0, r3
 80001e0:	4152      	adcs	r2, r2
 80001e2:	0883      	lsrs	r3, r0, #2
 80001e4:	428b      	cmp	r3, r1
 80001e6:	d301      	bcc.n	80001ec <__udivsi3+0xe4>
 80001e8:	008b      	lsls	r3, r1, #2
 80001ea:	1ac0      	subs	r0, r0, r3
 80001ec:	4152      	adcs	r2, r2
 80001ee:	0843      	lsrs	r3, r0, #1
 80001f0:	428b      	cmp	r3, r1
 80001f2:	d301      	bcc.n	80001f8 <__udivsi3+0xf0>
 80001f4:	004b      	lsls	r3, r1, #1
 80001f6:	1ac0      	subs	r0, r0, r3
 80001f8:	4152      	adcs	r2, r2
 80001fa:	1a41      	subs	r1, r0, r1
 80001fc:	d200      	bcs.n	8000200 <__udivsi3+0xf8>
 80001fe:	4601      	mov	r1, r0
 8000200:	4152      	adcs	r2, r2
 8000202:	4610      	mov	r0, r2
 8000204:	4770      	bx	lr
 8000206:	e7ff      	b.n	8000208 <__udivsi3+0x100>
 8000208:	b501      	push	{r0, lr}
 800020a:	2000      	movs	r0, #0
 800020c:	f000 f8f0 	bl	80003f0 <__aeabi_idiv0>
 8000210:	bd02      	pop	{r1, pc}
 8000212:	46c0      	nop			; (mov r8, r8)

08000214 <__aeabi_uidivmod>:
 8000214:	2900      	cmp	r1, #0
 8000216:	d0f7      	beq.n	8000208 <__udivsi3+0x100>
 8000218:	e776      	b.n	8000108 <__udivsi3>
 800021a:	4770      	bx	lr

0800021c <__divsi3>:
 800021c:	4603      	mov	r3, r0
 800021e:	430b      	orrs	r3, r1
 8000220:	d47f      	bmi.n	8000322 <__divsi3+0x106>
 8000222:	2200      	movs	r2, #0
 8000224:	0843      	lsrs	r3, r0, #1
 8000226:	428b      	cmp	r3, r1
 8000228:	d374      	bcc.n	8000314 <__divsi3+0xf8>
 800022a:	0903      	lsrs	r3, r0, #4
 800022c:	428b      	cmp	r3, r1
 800022e:	d35f      	bcc.n	80002f0 <__divsi3+0xd4>
 8000230:	0a03      	lsrs	r3, r0, #8
 8000232:	428b      	cmp	r3, r1
 8000234:	d344      	bcc.n	80002c0 <__divsi3+0xa4>
 8000236:	0b03      	lsrs	r3, r0, #12
 8000238:	428b      	cmp	r3, r1
 800023a:	d328      	bcc.n	800028e <__divsi3+0x72>
 800023c:	0c03      	lsrs	r3, r0, #16
 800023e:	428b      	cmp	r3, r1
 8000240:	d30d      	bcc.n	800025e <__divsi3+0x42>
 8000242:	22ff      	movs	r2, #255	; 0xff
 8000244:	0209      	lsls	r1, r1, #8
 8000246:	ba12      	rev	r2, r2
 8000248:	0c03      	lsrs	r3, r0, #16
 800024a:	428b      	cmp	r3, r1
 800024c:	d302      	bcc.n	8000254 <__divsi3+0x38>
 800024e:	1212      	asrs	r2, r2, #8
 8000250:	0209      	lsls	r1, r1, #8
 8000252:	d065      	beq.n	8000320 <__divsi3+0x104>
 8000254:	0b03      	lsrs	r3, r0, #12
 8000256:	428b      	cmp	r3, r1
 8000258:	d319      	bcc.n	800028e <__divsi3+0x72>
 800025a:	e000      	b.n	800025e <__divsi3+0x42>
 800025c:	0a09      	lsrs	r1, r1, #8
 800025e:	0bc3      	lsrs	r3, r0, #15
 8000260:	428b      	cmp	r3, r1
 8000262:	d301      	bcc.n	8000268 <__divsi3+0x4c>
 8000264:	03cb      	lsls	r3, r1, #15
 8000266:	1ac0      	subs	r0, r0, r3
 8000268:	4152      	adcs	r2, r2
 800026a:	0b83      	lsrs	r3, r0, #14
 800026c:	428b      	cmp	r3, r1
 800026e:	d301      	bcc.n	8000274 <__divsi3+0x58>
 8000270:	038b      	lsls	r3, r1, #14
 8000272:	1ac0      	subs	r0, r0, r3
 8000274:	4152      	adcs	r2, r2
 8000276:	0b43      	lsrs	r3, r0, #13
 8000278:	428b      	cmp	r3, r1
 800027a:	d301      	bcc.n	8000280 <__divsi3+0x64>
 800027c:	034b      	lsls	r3, r1, #13
 800027e:	1ac0      	subs	r0, r0, r3
 8000280:	4152      	adcs	r2, r2
 8000282:	0b03      	lsrs	r3, r0, #12
 8000284:	428b      	cmp	r3, r1
 8000286:	d301      	bcc.n	800028c <__divsi3+0x70>
 8000288:	030b      	lsls	r3, r1, #12
 800028a:	1ac0      	subs	r0, r0, r3
 800028c:	4152      	adcs	r2, r2
 800028e:	0ac3      	lsrs	r3, r0, #11
 8000290:	428b      	cmp	r3, r1
 8000292:	d301      	bcc.n	8000298 <__divsi3+0x7c>
 8000294:	02cb      	lsls	r3, r1, #11
 8000296:	1ac0      	subs	r0, r0, r3
 8000298:	4152      	adcs	r2, r2
 800029a:	0a83      	lsrs	r3, r0, #10
 800029c:	428b      	cmp	r3, r1
 800029e:	d301      	bcc.n	80002a4 <__divsi3+0x88>
 80002a0:	028b      	lsls	r3, r1, #10
 80002a2:	1ac0      	subs	r0, r0, r3
 80002a4:	4152      	adcs	r2, r2
 80002a6:	0a43      	lsrs	r3, r0, #9
 80002a8:	428b      	cmp	r3, r1
 80002aa:	d301      	bcc.n	80002b0 <__divsi3+0x94>
 80002ac:	024b      	lsls	r3, r1, #9
 80002ae:	1ac0      	subs	r0, r0, r3
 80002b0:	4152      	adcs	r2, r2
 80002b2:	0a03      	lsrs	r3, r0, #8
 80002b4:	428b      	cmp	r3, r1
 80002b6:	d301      	bcc.n	80002bc <__divsi3+0xa0>
 80002b8:	020b      	lsls	r3, r1, #8
 80002ba:	1ac0      	subs	r0, r0, r3
 80002bc:	4152      	adcs	r2, r2
 80002be:	d2cd      	bcs.n	800025c <__divsi3+0x40>
 80002c0:	09c3      	lsrs	r3, r0, #7
 80002c2:	428b      	cmp	r3, r1
 80002c4:	d301      	bcc.n	80002ca <__divsi3+0xae>
 80002c6:	01cb      	lsls	r3, r1, #7
 80002c8:	1ac0      	subs	r0, r0, r3
 80002ca:	4152      	adcs	r2, r2
 80002cc:	0983      	lsrs	r3, r0, #6
 80002ce:	428b      	cmp	r3, r1
 80002d0:	d301      	bcc.n	80002d6 <__divsi3+0xba>
 80002d2:	018b      	lsls	r3, r1, #6
 80002d4:	1ac0      	subs	r0, r0, r3
 80002d6:	4152      	adcs	r2, r2
 80002d8:	0943      	lsrs	r3, r0, #5
 80002da:	428b      	cmp	r3, r1
 80002dc:	d301      	bcc.n	80002e2 <__divsi3+0xc6>
 80002de:	014b      	lsls	r3, r1, #5
 80002e0:	1ac0      	subs	r0, r0, r3
 80002e2:	4152      	adcs	r2, r2
 80002e4:	0903      	lsrs	r3, r0, #4
 80002e6:	428b      	cmp	r3, r1
 80002e8:	d301      	bcc.n	80002ee <__divsi3+0xd2>
 80002ea:	010b      	lsls	r3, r1, #4
 80002ec:	1ac0      	subs	r0, r0, r3
 80002ee:	4152      	adcs	r2, r2
 80002f0:	08c3      	lsrs	r3, r0, #3
 80002f2:	428b      	cmp	r3, r1
 80002f4:	d301      	bcc.n	80002fa <__divsi3+0xde>
 80002f6:	00cb      	lsls	r3, r1, #3
 80002f8:	1ac0      	subs	r0, r0, r3
 80002fa:	4152      	adcs	r2, r2
 80002fc:	0883      	lsrs	r3, r0, #2
 80002fe:	428b      	cmp	r3, r1
 8000300:	d301      	bcc.n	8000306 <__divsi3+0xea>
 8000302:	008b      	lsls	r3, r1, #2
 8000304:	1ac0      	subs	r0, r0, r3
 8000306:	4152      	adcs	r2, r2
 8000308:	0843      	lsrs	r3, r0, #1
 800030a:	428b      	cmp	r3, r1
 800030c:	d301      	bcc.n	8000312 <__divsi3+0xf6>
 800030e:	004b      	lsls	r3, r1, #1
 8000310:	1ac0      	subs	r0, r0, r3
 8000312:	4152      	adcs	r2, r2
 8000314:	1a41      	subs	r1, r0, r1
 8000316:	d200      	bcs.n	800031a <__divsi3+0xfe>
 8000318:	4601      	mov	r1, r0
 800031a:	4152      	adcs	r2, r2
 800031c:	4610      	mov	r0, r2
 800031e:	4770      	bx	lr
 8000320:	e05d      	b.n	80003de <__divsi3+0x1c2>
 8000322:	0fca      	lsrs	r2, r1, #31
 8000324:	d000      	beq.n	8000328 <__divsi3+0x10c>
 8000326:	4249      	negs	r1, r1
 8000328:	1003      	asrs	r3, r0, #32
 800032a:	d300      	bcc.n	800032e <__divsi3+0x112>
 800032c:	4240      	negs	r0, r0
 800032e:	4053      	eors	r3, r2
 8000330:	2200      	movs	r2, #0
 8000332:	469c      	mov	ip, r3
 8000334:	0903      	lsrs	r3, r0, #4
 8000336:	428b      	cmp	r3, r1
 8000338:	d32d      	bcc.n	8000396 <__divsi3+0x17a>
 800033a:	0a03      	lsrs	r3, r0, #8
 800033c:	428b      	cmp	r3, r1
 800033e:	d312      	bcc.n	8000366 <__divsi3+0x14a>
 8000340:	22fc      	movs	r2, #252	; 0xfc
 8000342:	0189      	lsls	r1, r1, #6
 8000344:	ba12      	rev	r2, r2
 8000346:	0a03      	lsrs	r3, r0, #8
 8000348:	428b      	cmp	r3, r1
 800034a:	d30c      	bcc.n	8000366 <__divsi3+0x14a>
 800034c:	0189      	lsls	r1, r1, #6
 800034e:	1192      	asrs	r2, r2, #6
 8000350:	428b      	cmp	r3, r1
 8000352:	d308      	bcc.n	8000366 <__divsi3+0x14a>
 8000354:	0189      	lsls	r1, r1, #6
 8000356:	1192      	asrs	r2, r2, #6
 8000358:	428b      	cmp	r3, r1
 800035a:	d304      	bcc.n	8000366 <__divsi3+0x14a>
 800035c:	0189      	lsls	r1, r1, #6
 800035e:	d03a      	beq.n	80003d6 <__divsi3+0x1ba>
 8000360:	1192      	asrs	r2, r2, #6
 8000362:	e000      	b.n	8000366 <__divsi3+0x14a>
 8000364:	0989      	lsrs	r1, r1, #6
 8000366:	09c3      	lsrs	r3, r0, #7
 8000368:	428b      	cmp	r3, r1
 800036a:	d301      	bcc.n	8000370 <__divsi3+0x154>
 800036c:	01cb      	lsls	r3, r1, #7
 800036e:	1ac0      	subs	r0, r0, r3
 8000370:	4152      	adcs	r2, r2
 8000372:	0983      	lsrs	r3, r0, #6
 8000374:	428b      	cmp	r3, r1
 8000376:	d301      	bcc.n	800037c <__divsi3+0x160>
 8000378:	018b      	lsls	r3, r1, #6
 800037a:	1ac0      	subs	r0, r0, r3
 800037c:	4152      	adcs	r2, r2
 800037e:	0943      	lsrs	r3, r0, #5
 8000380:	428b      	cmp	r3, r1
 8000382:	d301      	bcc.n	8000388 <__divsi3+0x16c>
 8000384:	014b      	lsls	r3, r1, #5
 8000386:	1ac0      	subs	r0, r0, r3
 8000388:	4152      	adcs	r2, r2
 800038a:	0903      	lsrs	r3, r0, #4
 800038c:	428b      	cmp	r3, r1
 800038e:	d301      	bcc.n	8000394 <__divsi3+0x178>
 8000390:	010b      	lsls	r3, r1, #4
 8000392:	1ac0      	subs	r0, r0, r3
 8000394:	4152      	adcs	r2, r2
 8000396:	08c3      	lsrs	r3, r0, #3
 8000398:	428b      	cmp	r3, r1
 800039a:	d301      	bcc.n	80003a0 <__divsi3+0x184>
 800039c:	00cb      	lsls	r3, r1, #3
 800039e:	1ac0      	subs	r0, r0, r3
 80003a0:	4152      	adcs	r2, r2
 80003a2:	0883      	lsrs	r3, r0, #2
 80003a4:	428b      	cmp	r3, r1
 80003a6:	d301      	bcc.n	80003ac <__divsi3+0x190>
 80003a8:	008b      	lsls	r3, r1, #2
 80003aa:	1ac0      	subs	r0, r0, r3
 80003ac:	4152      	adcs	r2, r2
 80003ae:	d2d9      	bcs.n	8000364 <__divsi3+0x148>
 80003b0:	0843      	lsrs	r3, r0, #1
 80003b2:	428b      	cmp	r3, r1
 80003b4:	d301      	bcc.n	80003ba <__divsi3+0x19e>
 80003b6:	004b      	lsls	r3, r1, #1
 80003b8:	1ac0      	subs	r0, r0, r3
 80003ba:	4152      	adcs	r2, r2
 80003bc:	1a41      	subs	r1, r0, r1
 80003be:	d200      	bcs.n	80003c2 <__divsi3+0x1a6>
 80003c0:	4601      	mov	r1, r0
 80003c2:	4663      	mov	r3, ip
 80003c4:	4152      	adcs	r2, r2
 80003c6:	105b      	asrs	r3, r3, #1
 80003c8:	4610      	mov	r0, r2
 80003ca:	d301      	bcc.n	80003d0 <__divsi3+0x1b4>
 80003cc:	4240      	negs	r0, r0
 80003ce:	2b00      	cmp	r3, #0
 80003d0:	d500      	bpl.n	80003d4 <__divsi3+0x1b8>
 80003d2:	4249      	negs	r1, r1
 80003d4:	4770      	bx	lr
 80003d6:	4663      	mov	r3, ip
 80003d8:	105b      	asrs	r3, r3, #1
 80003da:	d300      	bcc.n	80003de <__divsi3+0x1c2>
 80003dc:	4240      	negs	r0, r0
 80003de:	b501      	push	{r0, lr}
 80003e0:	2000      	movs	r0, #0
 80003e2:	f000 f805 	bl	80003f0 <__aeabi_idiv0>
 80003e6:	bd02      	pop	{r1, pc}

080003e8 <__aeabi_idivmod>:
 80003e8:	2900      	cmp	r1, #0
 80003ea:	d0f8      	beq.n	80003de <__divsi3+0x1c2>
 80003ec:	e716      	b.n	800021c <__divsi3>
 80003ee:	4770      	bx	lr

080003f0 <__aeabi_idiv0>:
 80003f0:	4770      	bx	lr
 80003f2:	46c0      	nop			; (mov r8, r8)

080003f4 <__aeabi_cdrcmple>:
 80003f4:	4684      	mov	ip, r0
 80003f6:	1c10      	adds	r0, r2, #0
 80003f8:	4662      	mov	r2, ip
 80003fa:	468c      	mov	ip, r1
 80003fc:	1c19      	adds	r1, r3, #0
 80003fe:	4663      	mov	r3, ip
 8000400:	e000      	b.n	8000404 <__aeabi_cdcmpeq>
 8000402:	46c0      	nop			; (mov r8, r8)

08000404 <__aeabi_cdcmpeq>:
 8000404:	b51f      	push	{r0, r1, r2, r3, r4, lr}
 8000406:	f001 f9f5 	bl	80017f4 <__ledf2>
 800040a:	2800      	cmp	r0, #0
 800040c:	d401      	bmi.n	8000412 <__aeabi_cdcmpeq+0xe>
 800040e:	2100      	movs	r1, #0
 8000410:	42c8      	cmn	r0, r1
 8000412:	bd1f      	pop	{r0, r1, r2, r3, r4, pc}

08000414 <__aeabi_dcmpeq>:
 8000414:	b510      	push	{r4, lr}
 8000416:	f001 f94d 	bl	80016b4 <__eqdf2>
 800041a:	4240      	negs	r0, r0
 800041c:	3001      	adds	r0, #1
 800041e:	bd10      	pop	{r4, pc}

08000420 <__aeabi_dcmplt>:
 8000420:	b510      	push	{r4, lr}
 8000422:	f001 f9e7 	bl	80017f4 <__ledf2>
 8000426:	2800      	cmp	r0, #0
 8000428:	db01      	blt.n	800042e <__aeabi_dcmplt+0xe>
 800042a:	2000      	movs	r0, #0
 800042c:	bd10      	pop	{r4, pc}
 800042e:	2001      	movs	r0, #1
 8000430:	bd10      	pop	{r4, pc}
 8000432:	46c0      	nop			; (mov r8, r8)

08000434 <__aeabi_dcmple>:
 8000434:	b510      	push	{r4, lr}
 8000436:	f001 f9dd 	bl	80017f4 <__ledf2>
 800043a:	2800      	cmp	r0, #0
 800043c:	dd01      	ble.n	8000442 <__aeabi_dcmple+0xe>
 800043e:	2000      	movs	r0, #0
 8000440:	bd10      	pop	{r4, pc}
 8000442:	2001      	movs	r0, #1
 8000444:	bd10      	pop	{r4, pc}
 8000446:	46c0      	nop			; (mov r8, r8)

08000448 <__aeabi_dcmpgt>:
 8000448:	b510      	push	{r4, lr}
 800044a:	f001 f96f 	bl	800172c <__gedf2>
 800044e:	2800      	cmp	r0, #0
 8000450:	dc01      	bgt.n	8000456 <__aeabi_dcmpgt+0xe>
 8000452:	2000      	movs	r0, #0
 8000454:	bd10      	pop	{r4, pc}
 8000456:	2001      	movs	r0, #1
 8000458:	bd10      	pop	{r4, pc}
 800045a:	46c0      	nop			; (mov r8, r8)

0800045c <__aeabi_dcmpge>:
 800045c:	b510      	push	{r4, lr}
 800045e:	f001 f965 	bl	800172c <__gedf2>
 8000462:	2800      	cmp	r0, #0
 8000464:	da01      	bge.n	800046a <__aeabi_dcmpge+0xe>
 8000466:	2000      	movs	r0, #0
 8000468:	bd10      	pop	{r4, pc}
 800046a:	2001      	movs	r0, #1
 800046c:	bd10      	pop	{r4, pc}
 800046e:	46c0      	nop			; (mov r8, r8)

08000470 <__aeabi_uldivmod>:
 8000470:	2b00      	cmp	r3, #0
 8000472:	d111      	bne.n	8000498 <__aeabi_uldivmod+0x28>
 8000474:	2a00      	cmp	r2, #0
 8000476:	d10f      	bne.n	8000498 <__aeabi_uldivmod+0x28>
 8000478:	2900      	cmp	r1, #0
 800047a:	d100      	bne.n	800047e <__aeabi_uldivmod+0xe>
 800047c:	2800      	cmp	r0, #0
 800047e:	d002      	beq.n	8000486 <__aeabi_uldivmod+0x16>
 8000480:	2100      	movs	r1, #0
 8000482:	43c9      	mvns	r1, r1
 8000484:	1c08      	adds	r0, r1, #0
 8000486:	b407      	push	{r0, r1, r2}
 8000488:	4802      	ldr	r0, [pc, #8]	; (8000494 <__aeabi_uldivmod+0x24>)
 800048a:	a102      	add	r1, pc, #8	; (adr r1, 8000494 <__aeabi_uldivmod+0x24>)
 800048c:	1840      	adds	r0, r0, r1
 800048e:	9002      	str	r0, [sp, #8]
 8000490:	bd03      	pop	{r0, r1, pc}
 8000492:	46c0      	nop			; (mov r8, r8)
 8000494:	ffffff5d 	.word	0xffffff5d
 8000498:	b403      	push	{r0, r1}
 800049a:	4668      	mov	r0, sp
 800049c:	b501      	push	{r0, lr}
 800049e:	9802      	ldr	r0, [sp, #8]
 80004a0:	f000 f824 	bl	80004ec <__udivmoddi4>
 80004a4:	9b01      	ldr	r3, [sp, #4]
 80004a6:	469e      	mov	lr, r3
 80004a8:	b002      	add	sp, #8
 80004aa:	bc0c      	pop	{r2, r3}
 80004ac:	4770      	bx	lr
 80004ae:	46c0      	nop			; (mov r8, r8)

080004b0 <__aeabi_d2uiz>:
 80004b0:	b570      	push	{r4, r5, r6, lr}
 80004b2:	2200      	movs	r2, #0
 80004b4:	4b0c      	ldr	r3, [pc, #48]	; (80004e8 <__aeabi_d2uiz+0x38>)
 80004b6:	0004      	movs	r4, r0
 80004b8:	000d      	movs	r5, r1
 80004ba:	f7ff ffcf 	bl	800045c <__aeabi_dcmpge>
 80004be:	2800      	cmp	r0, #0
 80004c0:	d104      	bne.n	80004cc <__aeabi_d2uiz+0x1c>
 80004c2:	0020      	movs	r0, r4
 80004c4:	0029      	movs	r1, r5
 80004c6:	f001 ffb7 	bl	8002438 <__aeabi_d2iz>
 80004ca:	bd70      	pop	{r4, r5, r6, pc}
 80004cc:	4b06      	ldr	r3, [pc, #24]	; (80004e8 <__aeabi_d2uiz+0x38>)
 80004ce:	2200      	movs	r2, #0
 80004d0:	0020      	movs	r0, r4
 80004d2:	0029      	movs	r1, r5
 80004d4:	f001 fc68 	bl	8001da8 <__aeabi_dsub>
 80004d8:	f001 ffae 	bl	8002438 <__aeabi_d2iz>
 80004dc:	2380      	movs	r3, #128	; 0x80
 80004de:	061b      	lsls	r3, r3, #24
 80004e0:	469c      	mov	ip, r3
 80004e2:	4460      	add	r0, ip
 80004e4:	e7f1      	b.n	80004ca <__aeabi_d2uiz+0x1a>
 80004e6:	46c0      	nop			; (mov r8, r8)
 80004e8:	41e00000 	.word	0x41e00000

080004ec <__udivmoddi4>:
 80004ec:	b5f0      	push	{r4, r5, r6, r7, lr}
 80004ee:	464f      	mov	r7, r9
 80004f0:	4646      	mov	r6, r8
 80004f2:	46d6      	mov	lr, sl
 80004f4:	b5c0      	push	{r6, r7, lr}
 80004f6:	0004      	movs	r4, r0
 80004f8:	b082      	sub	sp, #8
 80004fa:	000d      	movs	r5, r1
 80004fc:	4691      	mov	r9, r2
 80004fe:	4698      	mov	r8, r3
 8000500:	428b      	cmp	r3, r1
 8000502:	d82f      	bhi.n	8000564 <__udivmoddi4+0x78>
 8000504:	d02c      	beq.n	8000560 <__udivmoddi4+0x74>
 8000506:	4641      	mov	r1, r8
 8000508:	4648      	mov	r0, r9
 800050a:	f002 f8a7 	bl	800265c <__clzdi2>
 800050e:	0029      	movs	r1, r5
 8000510:	0006      	movs	r6, r0
 8000512:	0020      	movs	r0, r4
 8000514:	f002 f8a2 	bl	800265c <__clzdi2>
 8000518:	1a33      	subs	r3, r6, r0
 800051a:	469c      	mov	ip, r3
 800051c:	3b20      	subs	r3, #32
 800051e:	469a      	mov	sl, r3
 8000520:	d500      	bpl.n	8000524 <__udivmoddi4+0x38>
 8000522:	e076      	b.n	8000612 <__udivmoddi4+0x126>
 8000524:	464b      	mov	r3, r9
 8000526:	4652      	mov	r2, sl
 8000528:	4093      	lsls	r3, r2
 800052a:	001f      	movs	r7, r3
 800052c:	464b      	mov	r3, r9
 800052e:	4662      	mov	r2, ip
 8000530:	4093      	lsls	r3, r2
 8000532:	001e      	movs	r6, r3
 8000534:	42af      	cmp	r7, r5
 8000536:	d828      	bhi.n	800058a <__udivmoddi4+0x9e>
 8000538:	d025      	beq.n	8000586 <__udivmoddi4+0x9a>
 800053a:	4653      	mov	r3, sl
 800053c:	1ba4      	subs	r4, r4, r6
 800053e:	41bd      	sbcs	r5, r7
 8000540:	2b00      	cmp	r3, #0
 8000542:	da00      	bge.n	8000546 <__udivmoddi4+0x5a>
 8000544:	e07b      	b.n	800063e <__udivmoddi4+0x152>
 8000546:	2200      	movs	r2, #0
 8000548:	2300      	movs	r3, #0
 800054a:	9200      	str	r2, [sp, #0]
 800054c:	9301      	str	r3, [sp, #4]
 800054e:	2301      	movs	r3, #1
 8000550:	4652      	mov	r2, sl
 8000552:	4093      	lsls	r3, r2
 8000554:	9301      	str	r3, [sp, #4]
 8000556:	2301      	movs	r3, #1
 8000558:	4662      	mov	r2, ip
 800055a:	4093      	lsls	r3, r2
 800055c:	9300      	str	r3, [sp, #0]
 800055e:	e018      	b.n	8000592 <__udivmoddi4+0xa6>
 8000560:	4282      	cmp	r2, r0
 8000562:	d9d0      	bls.n	8000506 <__udivmoddi4+0x1a>
 8000564:	2200      	movs	r2, #0
 8000566:	2300      	movs	r3, #0
 8000568:	9200      	str	r2, [sp, #0]
 800056a:	9301      	str	r3, [sp, #4]
 800056c:	9b0a      	ldr	r3, [sp, #40]	; 0x28
 800056e:	2b00      	cmp	r3, #0
 8000570:	d001      	beq.n	8000576 <__udivmoddi4+0x8a>
 8000572:	601c      	str	r4, [r3, #0]
 8000574:	605d      	str	r5, [r3, #4]
 8000576:	9800      	ldr	r0, [sp, #0]
 8000578:	9901      	ldr	r1, [sp, #4]
 800057a:	b002      	add	sp, #8
 800057c:	bc1c      	pop	{r2, r3, r4}
 800057e:	4690      	mov	r8, r2
 8000580:	4699      	mov	r9, r3
 8000582:	46a2      	mov	sl, r4
 8000584:	bdf0      	pop	{r4, r5, r6, r7, pc}
 8000586:	42a3      	cmp	r3, r4
 8000588:	d9d7      	bls.n	800053a <__udivmoddi4+0x4e>
 800058a:	2200      	movs	r2, #0
 800058c:	2300      	movs	r3, #0
 800058e:	9200      	str	r2, [sp, #0]
 8000590:	9301      	str	r3, [sp, #4]
 8000592:	4663      	mov	r3, ip
 8000594:	2b00      	cmp	r3, #0
 8000596:	d0e9      	beq.n	800056c <__udivmoddi4+0x80>
 8000598:	07fb      	lsls	r3, r7, #31
 800059a:	4698      	mov	r8, r3
 800059c:	4641      	mov	r1, r8
 800059e:	0872      	lsrs	r2, r6, #1
 80005a0:	430a      	orrs	r2, r1
 80005a2:	087b      	lsrs	r3, r7, #1
 80005a4:	4666      	mov	r6, ip
 80005a6:	e00e      	b.n	80005c6 <__udivmoddi4+0xda>
 80005a8:	42ab      	cmp	r3, r5
 80005aa:	d101      	bne.n	80005b0 <__udivmoddi4+0xc4>
 80005ac:	42a2      	cmp	r2, r4
 80005ae:	d80c      	bhi.n	80005ca <__udivmoddi4+0xde>
 80005b0:	1aa4      	subs	r4, r4, r2
 80005b2:	419d      	sbcs	r5, r3
 80005b4:	2001      	movs	r0, #1
 80005b6:	1924      	adds	r4, r4, r4
 80005b8:	416d      	adcs	r5, r5
 80005ba:	2100      	movs	r1, #0
 80005bc:	3e01      	subs	r6, #1
 80005be:	1824      	adds	r4, r4, r0
 80005c0:	414d      	adcs	r5, r1
 80005c2:	2e00      	cmp	r6, #0
 80005c4:	d006      	beq.n	80005d4 <__udivmoddi4+0xe8>
 80005c6:	42ab      	cmp	r3, r5
 80005c8:	d9ee      	bls.n	80005a8 <__udivmoddi4+0xbc>
 80005ca:	3e01      	subs	r6, #1
 80005cc:	1924      	adds	r4, r4, r4
 80005ce:	416d      	adcs	r5, r5
 80005d0:	2e00      	cmp	r6, #0
 80005d2:	d1f8      	bne.n	80005c6 <__udivmoddi4+0xda>
 80005d4:	9800      	ldr	r0, [sp, #0]
 80005d6:	9901      	ldr	r1, [sp, #4]
 80005d8:	4653      	mov	r3, sl
 80005da:	1900      	adds	r0, r0, r4
 80005dc:	4169      	adcs	r1, r5
 80005de:	2b00      	cmp	r3, #0
 80005e0:	db23      	blt.n	800062a <__udivmoddi4+0x13e>
 80005e2:	002b      	movs	r3, r5
 80005e4:	4652      	mov	r2, sl
 80005e6:	40d3      	lsrs	r3, r2
 80005e8:	002a      	movs	r2, r5
 80005ea:	4664      	mov	r4, ip
 80005ec:	40e2      	lsrs	r2, r4
 80005ee:	001c      	movs	r4, r3
 80005f0:	4653      	mov	r3, sl
 80005f2:	0015      	movs	r5, r2
 80005f4:	2b00      	cmp	r3, #0
 80005f6:	db2d      	blt.n	8000654 <__udivmoddi4+0x168>
 80005f8:	0026      	movs	r6, r4
 80005fa:	4657      	mov	r7, sl
 80005fc:	40be      	lsls	r6, r7
 80005fe:	0033      	movs	r3, r6
 8000600:	0026      	movs	r6, r4
 8000602:	4667      	mov	r7, ip
 8000604:	40be      	lsls	r6, r7
 8000606:	0032      	movs	r2, r6
 8000608:	1a80      	subs	r0, r0, r2
 800060a:	4199      	sbcs	r1, r3
 800060c:	9000      	str	r0, [sp, #0]
 800060e:	9101      	str	r1, [sp, #4]
 8000610:	e7ac      	b.n	800056c <__udivmoddi4+0x80>
 8000612:	4662      	mov	r2, ip
 8000614:	2320      	movs	r3, #32
 8000616:	1a9b      	subs	r3, r3, r2
 8000618:	464a      	mov	r2, r9
 800061a:	40da      	lsrs	r2, r3
 800061c:	4661      	mov	r1, ip
 800061e:	0013      	movs	r3, r2
 8000620:	4642      	mov	r2, r8
 8000622:	408a      	lsls	r2, r1
 8000624:	0017      	movs	r7, r2
 8000626:	431f      	orrs	r7, r3
 8000628:	e780      	b.n	800052c <__udivmoddi4+0x40>
 800062a:	4662      	mov	r2, ip
 800062c:	2320      	movs	r3, #32
 800062e:	1a9b      	subs	r3, r3, r2
 8000630:	002a      	movs	r2, r5
 8000632:	4666      	mov	r6, ip
 8000634:	409a      	lsls	r2, r3
 8000636:	0023      	movs	r3, r4
 8000638:	40f3      	lsrs	r3, r6
 800063a:	4313      	orrs	r3, r2
 800063c:	e7d4      	b.n	80005e8 <__udivmoddi4+0xfc>
 800063e:	4662      	mov	r2, ip
 8000640:	2320      	movs	r3, #32
 8000642:	2100      	movs	r1, #0
 8000644:	1a9b      	subs	r3, r3, r2
 8000646:	2200      	movs	r2, #0
 8000648:	9100      	str	r1, [sp, #0]
 800064a:	9201      	str	r2, [sp, #4]
 800064c:	2201      	movs	r2, #1
 800064e:	40da      	lsrs	r2, r3
 8000650:	9201      	str	r2, [sp, #4]
 8000652:	e780      	b.n	8000556 <__udivmoddi4+0x6a>
 8000654:	2320      	movs	r3, #32
 8000656:	4662      	mov	r2, ip
 8000658:	0026      	movs	r6, r4
 800065a:	1a9b      	subs	r3, r3, r2
 800065c:	40de      	lsrs	r6, r3
 800065e:	002f      	movs	r7, r5
 8000660:	46b0      	mov	r8, r6
 8000662:	4666      	mov	r6, ip
 8000664:	40b7      	lsls	r7, r6
 8000666:	4646      	mov	r6, r8
 8000668:	003b      	movs	r3, r7
 800066a:	4333      	orrs	r3, r6
 800066c:	e7c8      	b.n	8000600 <__udivmoddi4+0x114>
 800066e:	46c0      	nop			; (mov r8, r8)

08000670 <__aeabi_fsub>:
 8000670:	b5f8      	push	{r3, r4, r5, r6, r7, lr}
 8000672:	4647      	mov	r7, r8
 8000674:	46ce      	mov	lr, r9
 8000676:	0044      	lsls	r4, r0, #1
 8000678:	0fc2      	lsrs	r2, r0, #31
 800067a:	b580      	push	{r7, lr}
 800067c:	0247      	lsls	r7, r0, #9
 800067e:	0248      	lsls	r0, r1, #9
 8000680:	0a40      	lsrs	r0, r0, #9
 8000682:	4684      	mov	ip, r0
 8000684:	4666      	mov	r6, ip
 8000686:	0048      	lsls	r0, r1, #1
 8000688:	0a7f      	lsrs	r7, r7, #9
 800068a:	0e24      	lsrs	r4, r4, #24
 800068c:	00f6      	lsls	r6, r6, #3
 800068e:	0025      	movs	r5, r4
 8000690:	4690      	mov	r8, r2
 8000692:	00fb      	lsls	r3, r7, #3
 8000694:	0e00      	lsrs	r0, r0, #24
 8000696:	0fc9      	lsrs	r1, r1, #31
 8000698:	46b1      	mov	r9, r6
 800069a:	28ff      	cmp	r0, #255	; 0xff
 800069c:	d100      	bne.n	80006a0 <__aeabi_fsub+0x30>
 800069e:	e085      	b.n	80007ac <__aeabi_fsub+0x13c>
 80006a0:	2601      	movs	r6, #1
 80006a2:	4071      	eors	r1, r6
 80006a4:	1a26      	subs	r6, r4, r0
 80006a6:	4291      	cmp	r1, r2
 80006a8:	d057      	beq.n	800075a <__aeabi_fsub+0xea>
 80006aa:	2e00      	cmp	r6, #0
 80006ac:	dd43      	ble.n	8000736 <__aeabi_fsub+0xc6>
 80006ae:	2800      	cmp	r0, #0
 80006b0:	d000      	beq.n	80006b4 <__aeabi_fsub+0x44>
 80006b2:	e07f      	b.n	80007b4 <__aeabi_fsub+0x144>
 80006b4:	4649      	mov	r1, r9
 80006b6:	2900      	cmp	r1, #0
 80006b8:	d100      	bne.n	80006bc <__aeabi_fsub+0x4c>
 80006ba:	e0aa      	b.n	8000812 <__aeabi_fsub+0x1a2>
 80006bc:	3e01      	subs	r6, #1
 80006be:	2e00      	cmp	r6, #0
 80006c0:	d000      	beq.n	80006c4 <__aeabi_fsub+0x54>
 80006c2:	e0f7      	b.n	80008b4 <__aeabi_fsub+0x244>
 80006c4:	1a5b      	subs	r3, r3, r1
 80006c6:	015a      	lsls	r2, r3, #5
 80006c8:	d400      	bmi.n	80006cc <__aeabi_fsub+0x5c>
 80006ca:	e08b      	b.n	80007e4 <__aeabi_fsub+0x174>
 80006cc:	019b      	lsls	r3, r3, #6
 80006ce:	099c      	lsrs	r4, r3, #6
 80006d0:	0020      	movs	r0, r4
 80006d2:	f001 ffa5 	bl	8002620 <__clzsi2>
 80006d6:	3805      	subs	r0, #5
 80006d8:	4084      	lsls	r4, r0
 80006da:	4285      	cmp	r5, r0
 80006dc:	dd00      	ble.n	80006e0 <__aeabi_fsub+0x70>
 80006de:	e0d3      	b.n	8000888 <__aeabi_fsub+0x218>
 80006e0:	1b45      	subs	r5, r0, r5
 80006e2:	0023      	movs	r3, r4
 80006e4:	2020      	movs	r0, #32
 80006e6:	3501      	adds	r5, #1
 80006e8:	40eb      	lsrs	r3, r5
 80006ea:	1b45      	subs	r5, r0, r5
 80006ec:	40ac      	lsls	r4, r5
 80006ee:	1e62      	subs	r2, r4, #1
 80006f0:	4194      	sbcs	r4, r2
 80006f2:	4323      	orrs	r3, r4
 80006f4:	2407      	movs	r4, #7
 80006f6:	2500      	movs	r5, #0
 80006f8:	401c      	ands	r4, r3
 80006fa:	2201      	movs	r2, #1
 80006fc:	4641      	mov	r1, r8
 80006fe:	400a      	ands	r2, r1
 8000700:	2c00      	cmp	r4, #0
 8000702:	d004      	beq.n	800070e <__aeabi_fsub+0x9e>
 8000704:	210f      	movs	r1, #15
 8000706:	4019      	ands	r1, r3
 8000708:	2904      	cmp	r1, #4
 800070a:	d000      	beq.n	800070e <__aeabi_fsub+0x9e>
 800070c:	3304      	adds	r3, #4
 800070e:	0159      	lsls	r1, r3, #5
 8000710:	d400      	bmi.n	8000714 <__aeabi_fsub+0xa4>
 8000712:	e080      	b.n	8000816 <__aeabi_fsub+0x1a6>
 8000714:	3501      	adds	r5, #1
 8000716:	b2ec      	uxtb	r4, r5
 8000718:	2dff      	cmp	r5, #255	; 0xff
 800071a:	d000      	beq.n	800071e <__aeabi_fsub+0xae>
 800071c:	e0a3      	b.n	8000866 <__aeabi_fsub+0x1f6>
 800071e:	24ff      	movs	r4, #255	; 0xff
 8000720:	2300      	movs	r3, #0
 8000722:	025b      	lsls	r3, r3, #9
 8000724:	05e4      	lsls	r4, r4, #23
 8000726:	0a58      	lsrs	r0, r3, #9
 8000728:	07d2      	lsls	r2, r2, #31
 800072a:	4320      	orrs	r0, r4
 800072c:	4310      	orrs	r0, r2
 800072e:	bc0c      	pop	{r2, r3}
 8000730:	4690      	mov	r8, r2
 8000732:	4699      	mov	r9, r3
 8000734:	bdf8      	pop	{r3, r4, r5, r6, r7, pc}
 8000736:	2e00      	cmp	r6, #0
 8000738:	d174      	bne.n	8000824 <__aeabi_fsub+0x1b4>
 800073a:	1c60      	adds	r0, r4, #1
 800073c:	b2c0      	uxtb	r0, r0
 800073e:	2801      	cmp	r0, #1
 8000740:	dc00      	bgt.n	8000744 <__aeabi_fsub+0xd4>
 8000742:	e0a7      	b.n	8000894 <__aeabi_fsub+0x224>
 8000744:	464a      	mov	r2, r9
 8000746:	1a9c      	subs	r4, r3, r2
 8000748:	0162      	lsls	r2, r4, #5
 800074a:	d500      	bpl.n	800074e <__aeabi_fsub+0xde>
 800074c:	e0b6      	b.n	80008bc <__aeabi_fsub+0x24c>
 800074e:	2c00      	cmp	r4, #0
 8000750:	d1be      	bne.n	80006d0 <__aeabi_fsub+0x60>
 8000752:	2200      	movs	r2, #0
 8000754:	2400      	movs	r4, #0
 8000756:	2300      	movs	r3, #0
 8000758:	e7e3      	b.n	8000722 <__aeabi_fsub+0xb2>
 800075a:	2e00      	cmp	r6, #0
 800075c:	dc00      	bgt.n	8000760 <__aeabi_fsub+0xf0>
 800075e:	e085      	b.n	800086c <__aeabi_fsub+0x1fc>
 8000760:	2800      	cmp	r0, #0
 8000762:	d046      	beq.n	80007f2 <__aeabi_fsub+0x182>
 8000764:	2cff      	cmp	r4, #255	; 0xff
 8000766:	d049      	beq.n	80007fc <__aeabi_fsub+0x18c>
 8000768:	2280      	movs	r2, #128	; 0x80
 800076a:	4648      	mov	r0, r9
 800076c:	04d2      	lsls	r2, r2, #19
 800076e:	4310      	orrs	r0, r2
 8000770:	4681      	mov	r9, r0
 8000772:	2201      	movs	r2, #1
 8000774:	2e1b      	cmp	r6, #27
 8000776:	dc09      	bgt.n	800078c <__aeabi_fsub+0x11c>
 8000778:	2020      	movs	r0, #32
 800077a:	464c      	mov	r4, r9
 800077c:	1b80      	subs	r0, r0, r6
 800077e:	4084      	lsls	r4, r0
 8000780:	464a      	mov	r2, r9
 8000782:	0020      	movs	r0, r4
 8000784:	40f2      	lsrs	r2, r6
 8000786:	1e44      	subs	r4, r0, #1
 8000788:	41a0      	sbcs	r0, r4
 800078a:	4302      	orrs	r2, r0
 800078c:	189b      	adds	r3, r3, r2
 800078e:	015a      	lsls	r2, r3, #5
 8000790:	d528      	bpl.n	80007e4 <__aeabi_fsub+0x174>
 8000792:	3501      	adds	r5, #1
 8000794:	2dff      	cmp	r5, #255	; 0xff
 8000796:	d100      	bne.n	800079a <__aeabi_fsub+0x12a>
 8000798:	e0a8      	b.n	80008ec <__aeabi_fsub+0x27c>
 800079a:	2201      	movs	r2, #1
 800079c:	2407      	movs	r4, #7
 800079e:	4994      	ldr	r1, [pc, #592]	; (80009f0 <__aeabi_fsub+0x380>)
 80007a0:	401a      	ands	r2, r3
 80007a2:	085b      	lsrs	r3, r3, #1
 80007a4:	400b      	ands	r3, r1
 80007a6:	4313      	orrs	r3, r2
 80007a8:	401c      	ands	r4, r3
 80007aa:	e7a6      	b.n	80006fa <__aeabi_fsub+0x8a>
 80007ac:	2e00      	cmp	r6, #0
 80007ae:	d000      	beq.n	80007b2 <__aeabi_fsub+0x142>
 80007b0:	e778      	b.n	80006a4 <__aeabi_fsub+0x34>
 80007b2:	e775      	b.n	80006a0 <__aeabi_fsub+0x30>
 80007b4:	2cff      	cmp	r4, #255	; 0xff
 80007b6:	d054      	beq.n	8000862 <__aeabi_fsub+0x1f2>
 80007b8:	2280      	movs	r2, #128	; 0x80
 80007ba:	4649      	mov	r1, r9
 80007bc:	04d2      	lsls	r2, r2, #19
 80007be:	4311      	orrs	r1, r2
 80007c0:	4689      	mov	r9, r1
 80007c2:	2201      	movs	r2, #1
 80007c4:	2e1b      	cmp	r6, #27
 80007c6:	dc09      	bgt.n	80007dc <__aeabi_fsub+0x16c>
 80007c8:	2120      	movs	r1, #32
 80007ca:	4648      	mov	r0, r9
 80007cc:	1b89      	subs	r1, r1, r6
 80007ce:	4088      	lsls	r0, r1
 80007d0:	464a      	mov	r2, r9
 80007d2:	0001      	movs	r1, r0
 80007d4:	40f2      	lsrs	r2, r6
 80007d6:	1e48      	subs	r0, r1, #1
 80007d8:	4181      	sbcs	r1, r0
 80007da:	430a      	orrs	r2, r1
 80007dc:	1a9b      	subs	r3, r3, r2
 80007de:	015a      	lsls	r2, r3, #5
 80007e0:	d500      	bpl.n	80007e4 <__aeabi_fsub+0x174>
 80007e2:	e773      	b.n	80006cc <__aeabi_fsub+0x5c>
 80007e4:	2201      	movs	r2, #1
 80007e6:	4641      	mov	r1, r8
 80007e8:	400a      	ands	r2, r1
 80007ea:	0759      	lsls	r1, r3, #29
 80007ec:	d000      	beq.n	80007f0 <__aeabi_fsub+0x180>
 80007ee:	e789      	b.n	8000704 <__aeabi_fsub+0x94>
 80007f0:	e011      	b.n	8000816 <__aeabi_fsub+0x1a6>
 80007f2:	4648      	mov	r0, r9
 80007f4:	2800      	cmp	r0, #0
 80007f6:	d158      	bne.n	80008aa <__aeabi_fsub+0x23a>
 80007f8:	2cff      	cmp	r4, #255	; 0xff
 80007fa:	d10c      	bne.n	8000816 <__aeabi_fsub+0x1a6>
 80007fc:	08db      	lsrs	r3, r3, #3
 80007fe:	2b00      	cmp	r3, #0
 8000800:	d100      	bne.n	8000804 <__aeabi_fsub+0x194>
 8000802:	e78c      	b.n	800071e <__aeabi_fsub+0xae>
 8000804:	2080      	movs	r0, #128	; 0x80
 8000806:	03c0      	lsls	r0, r0, #15
 8000808:	4303      	orrs	r3, r0
 800080a:	025b      	lsls	r3, r3, #9
 800080c:	0a5b      	lsrs	r3, r3, #9
 800080e:	24ff      	movs	r4, #255	; 0xff
 8000810:	e787      	b.n	8000722 <__aeabi_fsub+0xb2>
 8000812:	2cff      	cmp	r4, #255	; 0xff
 8000814:	d025      	beq.n	8000862 <__aeabi_fsub+0x1f2>
 8000816:	08db      	lsrs	r3, r3, #3
 8000818:	2dff      	cmp	r5, #255	; 0xff
 800081a:	d0f0      	beq.n	80007fe <__aeabi_fsub+0x18e>
 800081c:	025b      	lsls	r3, r3, #9
 800081e:	0a5b      	lsrs	r3, r3, #9
 8000820:	b2ec      	uxtb	r4, r5
 8000822:	e77e      	b.n	8000722 <__aeabi_fsub+0xb2>
 8000824:	2c00      	cmp	r4, #0
 8000826:	d04d      	beq.n	80008c4 <__aeabi_fsub+0x254>
 8000828:	28ff      	cmp	r0, #255	; 0xff
 800082a:	d018      	beq.n	800085e <__aeabi_fsub+0x1ee>
 800082c:	2480      	movs	r4, #128	; 0x80
 800082e:	04e4      	lsls	r4, r4, #19
 8000830:	4272      	negs	r2, r6
 8000832:	4323      	orrs	r3, r4
 8000834:	2a1b      	cmp	r2, #27
 8000836:	dd00      	ble.n	800083a <__aeabi_fsub+0x1ca>
 8000838:	e0c4      	b.n	80009c4 <__aeabi_fsub+0x354>
 800083a:	001c      	movs	r4, r3
 800083c:	2520      	movs	r5, #32
 800083e:	40d4      	lsrs	r4, r2
 8000840:	1aaa      	subs	r2, r5, r2
 8000842:	4093      	lsls	r3, r2
 8000844:	1e5a      	subs	r2, r3, #1
 8000846:	4193      	sbcs	r3, r2
 8000848:	4323      	orrs	r3, r4
 800084a:	464a      	mov	r2, r9
 800084c:	0005      	movs	r5, r0
 800084e:	1ad3      	subs	r3, r2, r3
 8000850:	4688      	mov	r8, r1
 8000852:	e738      	b.n	80006c6 <__aeabi_fsub+0x56>
 8000854:	1c72      	adds	r2, r6, #1
 8000856:	d0f8      	beq.n	800084a <__aeabi_fsub+0x1da>
 8000858:	43f2      	mvns	r2, r6
 800085a:	28ff      	cmp	r0, #255	; 0xff
 800085c:	d1ea      	bne.n	8000834 <__aeabi_fsub+0x1c4>
 800085e:	000a      	movs	r2, r1
 8000860:	464b      	mov	r3, r9
 8000862:	25ff      	movs	r5, #255	; 0xff
 8000864:	e7d7      	b.n	8000816 <__aeabi_fsub+0x1a6>
 8000866:	019b      	lsls	r3, r3, #6
 8000868:	0a5b      	lsrs	r3, r3, #9
 800086a:	e75a      	b.n	8000722 <__aeabi_fsub+0xb2>
 800086c:	2e00      	cmp	r6, #0
 800086e:	d141      	bne.n	80008f4 <__aeabi_fsub+0x284>
 8000870:	1c65      	adds	r5, r4, #1
 8000872:	b2e9      	uxtb	r1, r5
 8000874:	2901      	cmp	r1, #1
 8000876:	dd45      	ble.n	8000904 <__aeabi_fsub+0x294>
 8000878:	2dff      	cmp	r5, #255	; 0xff
 800087a:	d100      	bne.n	800087e <__aeabi_fsub+0x20e>
 800087c:	e74f      	b.n	800071e <__aeabi_fsub+0xae>
 800087e:	2407      	movs	r4, #7
 8000880:	444b      	add	r3, r9
 8000882:	085b      	lsrs	r3, r3, #1
 8000884:	401c      	ands	r4, r3
 8000886:	e738      	b.n	80006fa <__aeabi_fsub+0x8a>
 8000888:	2207      	movs	r2, #7
 800088a:	4b5a      	ldr	r3, [pc, #360]	; (80009f4 <__aeabi_fsub+0x384>)
 800088c:	1a2d      	subs	r5, r5, r0
 800088e:	4023      	ands	r3, r4
 8000890:	4014      	ands	r4, r2
 8000892:	e732      	b.n	80006fa <__aeabi_fsub+0x8a>
 8000894:	2c00      	cmp	r4, #0
 8000896:	d11d      	bne.n	80008d4 <__aeabi_fsub+0x264>
 8000898:	2b00      	cmp	r3, #0
 800089a:	d17a      	bne.n	8000992 <__aeabi_fsub+0x322>
 800089c:	464b      	mov	r3, r9
 800089e:	2b00      	cmp	r3, #0
 80008a0:	d100      	bne.n	80008a4 <__aeabi_fsub+0x234>
 80008a2:	e091      	b.n	80009c8 <__aeabi_fsub+0x358>
 80008a4:	000a      	movs	r2, r1
 80008a6:	2500      	movs	r5, #0
 80008a8:	e7b5      	b.n	8000816 <__aeabi_fsub+0x1a6>
 80008aa:	3e01      	subs	r6, #1
 80008ac:	2e00      	cmp	r6, #0
 80008ae:	d119      	bne.n	80008e4 <__aeabi_fsub+0x274>
 80008b0:	444b      	add	r3, r9
 80008b2:	e76c      	b.n	800078e <__aeabi_fsub+0x11e>
 80008b4:	2cff      	cmp	r4, #255	; 0xff
 80008b6:	d184      	bne.n	80007c2 <__aeabi_fsub+0x152>
 80008b8:	25ff      	movs	r5, #255	; 0xff
 80008ba:	e7ac      	b.n	8000816 <__aeabi_fsub+0x1a6>
 80008bc:	464a      	mov	r2, r9
 80008be:	4688      	mov	r8, r1
 80008c0:	1ad4      	subs	r4, r2, r3
 80008c2:	e705      	b.n	80006d0 <__aeabi_fsub+0x60>
 80008c4:	2b00      	cmp	r3, #0
 80008c6:	d1c5      	bne.n	8000854 <__aeabi_fsub+0x1e4>
 80008c8:	000a      	movs	r2, r1
 80008ca:	28ff      	cmp	r0, #255	; 0xff
 80008cc:	d0c8      	beq.n	8000860 <__aeabi_fsub+0x1f0>
 80008ce:	0005      	movs	r5, r0
 80008d0:	464b      	mov	r3, r9
 80008d2:	e7a0      	b.n	8000816 <__aeabi_fsub+0x1a6>
 80008d4:	2b00      	cmp	r3, #0
 80008d6:	d149      	bne.n	800096c <__aeabi_fsub+0x2fc>
 80008d8:	464b      	mov	r3, r9
 80008da:	2b00      	cmp	r3, #0
 80008dc:	d077      	beq.n	80009ce <__aeabi_fsub+0x35e>
 80008de:	000a      	movs	r2, r1
 80008e0:	25ff      	movs	r5, #255	; 0xff
 80008e2:	e798      	b.n	8000816 <__aeabi_fsub+0x1a6>
 80008e4:	2cff      	cmp	r4, #255	; 0xff
 80008e6:	d000      	beq.n	80008ea <__aeabi_fsub+0x27a>
 80008e8:	e743      	b.n	8000772 <__aeabi_fsub+0x102>
 80008ea:	e787      	b.n	80007fc <__aeabi_fsub+0x18c>
 80008ec:	000a      	movs	r2, r1
 80008ee:	24ff      	movs	r4, #255	; 0xff
 80008f0:	2300      	movs	r3, #0
 80008f2:	e716      	b.n	8000722 <__aeabi_fsub+0xb2>
 80008f4:	2c00      	cmp	r4, #0
 80008f6:	d115      	bne.n	8000924 <__aeabi_fsub+0x2b4>
 80008f8:	2b00      	cmp	r3, #0
 80008fa:	d157      	bne.n	80009ac <__aeabi_fsub+0x33c>
 80008fc:	28ff      	cmp	r0, #255	; 0xff
 80008fe:	d1e6      	bne.n	80008ce <__aeabi_fsub+0x25e>
 8000900:	464b      	mov	r3, r9
 8000902:	e77b      	b.n	80007fc <__aeabi_fsub+0x18c>
 8000904:	2c00      	cmp	r4, #0
 8000906:	d120      	bne.n	800094a <__aeabi_fsub+0x2da>
 8000908:	2b00      	cmp	r3, #0
 800090a:	d057      	beq.n	80009bc <__aeabi_fsub+0x34c>
 800090c:	4649      	mov	r1, r9
 800090e:	2900      	cmp	r1, #0
 8000910:	d053      	beq.n	80009ba <__aeabi_fsub+0x34a>
 8000912:	444b      	add	r3, r9
 8000914:	015a      	lsls	r2, r3, #5
 8000916:	d568      	bpl.n	80009ea <__aeabi_fsub+0x37a>
 8000918:	2407      	movs	r4, #7
 800091a:	4a36      	ldr	r2, [pc, #216]	; (80009f4 <__aeabi_fsub+0x384>)
 800091c:	401c      	ands	r4, r3
 800091e:	2501      	movs	r5, #1
 8000920:	4013      	ands	r3, r2
 8000922:	e6ea      	b.n	80006fa <__aeabi_fsub+0x8a>
 8000924:	28ff      	cmp	r0, #255	; 0xff
 8000926:	d0eb      	beq.n	8000900 <__aeabi_fsub+0x290>
 8000928:	2280      	movs	r2, #128	; 0x80
 800092a:	04d2      	lsls	r2, r2, #19
 800092c:	4276      	negs	r6, r6
 800092e:	4313      	orrs	r3, r2
 8000930:	2e1b      	cmp	r6, #27
 8000932:	dc53      	bgt.n	80009dc <__aeabi_fsub+0x36c>
 8000934:	2520      	movs	r5, #32
 8000936:	1bad      	subs	r5, r5, r6
 8000938:	001a      	movs	r2, r3
 800093a:	40ab      	lsls	r3, r5
 800093c:	40f2      	lsrs	r2, r6
 800093e:	1e5c      	subs	r4, r3, #1
 8000940:	41a3      	sbcs	r3, r4
 8000942:	4313      	orrs	r3, r2
 8000944:	444b      	add	r3, r9
 8000946:	0005      	movs	r5, r0
 8000948:	e721      	b.n	800078e <__aeabi_fsub+0x11e>
 800094a:	2b00      	cmp	r3, #0
 800094c:	d0d8      	beq.n	8000900 <__aeabi_fsub+0x290>
 800094e:	4649      	mov	r1, r9
 8000950:	2900      	cmp	r1, #0
 8000952:	d100      	bne.n	8000956 <__aeabi_fsub+0x2e6>
 8000954:	e752      	b.n	80007fc <__aeabi_fsub+0x18c>
 8000956:	2180      	movs	r1, #128	; 0x80
 8000958:	03c9      	lsls	r1, r1, #15
 800095a:	420f      	tst	r7, r1
 800095c:	d100      	bne.n	8000960 <__aeabi_fsub+0x2f0>
 800095e:	e74d      	b.n	80007fc <__aeabi_fsub+0x18c>
 8000960:	4660      	mov	r0, ip
 8000962:	4208      	tst	r0, r1
 8000964:	d000      	beq.n	8000968 <__aeabi_fsub+0x2f8>
 8000966:	e749      	b.n	80007fc <__aeabi_fsub+0x18c>
 8000968:	464b      	mov	r3, r9
 800096a:	e747      	b.n	80007fc <__aeabi_fsub+0x18c>
 800096c:	4648      	mov	r0, r9
 800096e:	25ff      	movs	r5, #255	; 0xff
 8000970:	2800      	cmp	r0, #0
 8000972:	d100      	bne.n	8000976 <__aeabi_fsub+0x306>
 8000974:	e74f      	b.n	8000816 <__aeabi_fsub+0x1a6>
 8000976:	2280      	movs	r2, #128	; 0x80
 8000978:	03d2      	lsls	r2, r2, #15
 800097a:	4217      	tst	r7, r2
 800097c:	d004      	beq.n	8000988 <__aeabi_fsub+0x318>
 800097e:	4660      	mov	r0, ip
 8000980:	4210      	tst	r0, r2
 8000982:	d101      	bne.n	8000988 <__aeabi_fsub+0x318>
 8000984:	464b      	mov	r3, r9
 8000986:	4688      	mov	r8, r1
 8000988:	2201      	movs	r2, #1
 800098a:	4641      	mov	r1, r8
 800098c:	25ff      	movs	r5, #255	; 0xff
 800098e:	400a      	ands	r2, r1
 8000990:	e741      	b.n	8000816 <__aeabi_fsub+0x1a6>
 8000992:	4648      	mov	r0, r9
 8000994:	2800      	cmp	r0, #0
 8000996:	d01f      	beq.n	80009d8 <__aeabi_fsub+0x368>
 8000998:	1a1a      	subs	r2, r3, r0
 800099a:	0150      	lsls	r0, r2, #5
 800099c:	d520      	bpl.n	80009e0 <__aeabi_fsub+0x370>
 800099e:	464a      	mov	r2, r9
 80009a0:	2407      	movs	r4, #7
 80009a2:	1ad3      	subs	r3, r2, r3
 80009a4:	401c      	ands	r4, r3
 80009a6:	4688      	mov	r8, r1
 80009a8:	2500      	movs	r5, #0
 80009aa:	e6a6      	b.n	80006fa <__aeabi_fsub+0x8a>
 80009ac:	1c74      	adds	r4, r6, #1
 80009ae:	d0c9      	beq.n	8000944 <__aeabi_fsub+0x2d4>
 80009b0:	43f6      	mvns	r6, r6
 80009b2:	28ff      	cmp	r0, #255	; 0xff
 80009b4:	d1bc      	bne.n	8000930 <__aeabi_fsub+0x2c0>
 80009b6:	464b      	mov	r3, r9
 80009b8:	e720      	b.n	80007fc <__aeabi_fsub+0x18c>
 80009ba:	4699      	mov	r9, r3
 80009bc:	464b      	mov	r3, r9
 80009be:	2500      	movs	r5, #0
 80009c0:	08db      	lsrs	r3, r3, #3
 80009c2:	e72b      	b.n	800081c <__aeabi_fsub+0x1ac>
 80009c4:	2301      	movs	r3, #1
 80009c6:	e740      	b.n	800084a <__aeabi_fsub+0x1da>
 80009c8:	2200      	movs	r2, #0
 80009ca:	2300      	movs	r3, #0
 80009cc:	e6a9      	b.n	8000722 <__aeabi_fsub+0xb2>
 80009ce:	2380      	movs	r3, #128	; 0x80
 80009d0:	2200      	movs	r2, #0
 80009d2:	03db      	lsls	r3, r3, #15
 80009d4:	24ff      	movs	r4, #255	; 0xff
 80009d6:	e6a4      	b.n	8000722 <__aeabi_fsub+0xb2>
 80009d8:	2500      	movs	r5, #0
 80009da:	e71c      	b.n	8000816 <__aeabi_fsub+0x1a6>
 80009dc:	2301      	movs	r3, #1
 80009de:	e7b1      	b.n	8000944 <__aeabi_fsub+0x2d4>
 80009e0:	2a00      	cmp	r2, #0
 80009e2:	d0f1      	beq.n	80009c8 <__aeabi_fsub+0x358>
 80009e4:	0013      	movs	r3, r2
 80009e6:	2500      	movs	r5, #0
 80009e8:	e6fc      	b.n	80007e4 <__aeabi_fsub+0x174>
 80009ea:	2500      	movs	r5, #0
 80009ec:	e6fa      	b.n	80007e4 <__aeabi_fsub+0x174>
 80009ee:	46c0      	nop			; (mov r8, r8)
 80009f0:	7dffffff 	.word	0x7dffffff
 80009f4:	fbffffff 	.word	0xfbffffff

080009f8 <__aeabi_ui2f>:
 80009f8:	b570      	push	{r4, r5, r6, lr}
 80009fa:	1e04      	subs	r4, r0, #0
 80009fc:	d034      	beq.n	8000a68 <__aeabi_ui2f+0x70>
 80009fe:	f001 fe0f 	bl	8002620 <__clzsi2>
 8000a02:	229e      	movs	r2, #158	; 0x9e
 8000a04:	1a12      	subs	r2, r2, r0
 8000a06:	2a96      	cmp	r2, #150	; 0x96
 8000a08:	dc07      	bgt.n	8000a1a <__aeabi_ui2f+0x22>
 8000a0a:	b2d2      	uxtb	r2, r2
 8000a0c:	2808      	cmp	r0, #8
 8000a0e:	dd2e      	ble.n	8000a6e <__aeabi_ui2f+0x76>
 8000a10:	3808      	subs	r0, #8
 8000a12:	4084      	lsls	r4, r0
 8000a14:	0260      	lsls	r0, r4, #9
 8000a16:	0a40      	lsrs	r0, r0, #9
 8000a18:	e021      	b.n	8000a5e <__aeabi_ui2f+0x66>
 8000a1a:	2a99      	cmp	r2, #153	; 0x99
 8000a1c:	dd09      	ble.n	8000a32 <__aeabi_ui2f+0x3a>
 8000a1e:	0003      	movs	r3, r0
 8000a20:	0021      	movs	r1, r4
 8000a22:	331b      	adds	r3, #27
 8000a24:	4099      	lsls	r1, r3
 8000a26:	1e4b      	subs	r3, r1, #1
 8000a28:	4199      	sbcs	r1, r3
 8000a2a:	2305      	movs	r3, #5
 8000a2c:	1a1b      	subs	r3, r3, r0
 8000a2e:	40dc      	lsrs	r4, r3
 8000a30:	430c      	orrs	r4, r1
 8000a32:	2805      	cmp	r0, #5
 8000a34:	dd01      	ble.n	8000a3a <__aeabi_ui2f+0x42>
 8000a36:	1f43      	subs	r3, r0, #5
 8000a38:	409c      	lsls	r4, r3
 8000a3a:	0023      	movs	r3, r4
 8000a3c:	490d      	ldr	r1, [pc, #52]	; (8000a74 <__aeabi_ui2f+0x7c>)
 8000a3e:	400b      	ands	r3, r1
 8000a40:	0765      	lsls	r5, r4, #29
 8000a42:	d009      	beq.n	8000a58 <__aeabi_ui2f+0x60>
 8000a44:	250f      	movs	r5, #15
 8000a46:	402c      	ands	r4, r5
 8000a48:	2c04      	cmp	r4, #4
 8000a4a:	d005      	beq.n	8000a58 <__aeabi_ui2f+0x60>
 8000a4c:	3304      	adds	r3, #4
 8000a4e:	015c      	lsls	r4, r3, #5
 8000a50:	d502      	bpl.n	8000a58 <__aeabi_ui2f+0x60>
 8000a52:	229f      	movs	r2, #159	; 0x9f
 8000a54:	400b      	ands	r3, r1
 8000a56:	1a12      	subs	r2, r2, r0
 8000a58:	019b      	lsls	r3, r3, #6
 8000a5a:	0a58      	lsrs	r0, r3, #9
 8000a5c:	b2d2      	uxtb	r2, r2
 8000a5e:	0240      	lsls	r0, r0, #9
 8000a60:	05d2      	lsls	r2, r2, #23
 8000a62:	0a40      	lsrs	r0, r0, #9
 8000a64:	4310      	orrs	r0, r2
 8000a66:	bd70      	pop	{r4, r5, r6, pc}
 8000a68:	2200      	movs	r2, #0
 8000a6a:	2000      	movs	r0, #0
 8000a6c:	e7f7      	b.n	8000a5e <__aeabi_ui2f+0x66>
 8000a6e:	0260      	lsls	r0, r4, #9
 8000a70:	0a40      	lsrs	r0, r0, #9
 8000a72:	e7f4      	b.n	8000a5e <__aeabi_ui2f+0x66>
 8000a74:	fbffffff 	.word	0xfbffffff

08000a78 <__aeabi_dadd>:
 8000a78:	b5f0      	push	{r4, r5, r6, r7, lr}
 8000a7a:	464f      	mov	r7, r9
 8000a7c:	4646      	mov	r6, r8
 8000a7e:	46d6      	mov	lr, sl
 8000a80:	000c      	movs	r4, r1
 8000a82:	0309      	lsls	r1, r1, #12
 8000a84:	b5c0      	push	{r6, r7, lr}
 8000a86:	0a49      	lsrs	r1, r1, #9
 8000a88:	0f47      	lsrs	r7, r0, #29
 8000a8a:	005e      	lsls	r6, r3, #1
 8000a8c:	4339      	orrs	r1, r7
 8000a8e:	031f      	lsls	r7, r3, #12
 8000a90:	0fdb      	lsrs	r3, r3, #31
 8000a92:	469c      	mov	ip, r3
 8000a94:	0065      	lsls	r5, r4, #1
 8000a96:	0a7b      	lsrs	r3, r7, #9
 8000a98:	0f57      	lsrs	r7, r2, #29
 8000a9a:	431f      	orrs	r7, r3
 8000a9c:	0d6d      	lsrs	r5, r5, #21
 8000a9e:	0fe4      	lsrs	r4, r4, #31
 8000aa0:	0d76      	lsrs	r6, r6, #21
 8000aa2:	46a1      	mov	r9, r4
 8000aa4:	00c0      	lsls	r0, r0, #3
 8000aa6:	46b8      	mov	r8, r7
 8000aa8:	00d2      	lsls	r2, r2, #3
 8000aaa:	1bab      	subs	r3, r5, r6
 8000aac:	4564      	cmp	r4, ip
 8000aae:	d07b      	beq.n	8000ba8 <__aeabi_dadd+0x130>
 8000ab0:	2b00      	cmp	r3, #0
 8000ab2:	dd5f      	ble.n	8000b74 <__aeabi_dadd+0xfc>
 8000ab4:	2e00      	cmp	r6, #0
 8000ab6:	d000      	beq.n	8000aba <__aeabi_dadd+0x42>
 8000ab8:	e0a4      	b.n	8000c04 <__aeabi_dadd+0x18c>
 8000aba:	003e      	movs	r6, r7
 8000abc:	4316      	orrs	r6, r2
 8000abe:	d100      	bne.n	8000ac2 <__aeabi_dadd+0x4a>
 8000ac0:	e112      	b.n	8000ce8 <__aeabi_dadd+0x270>
 8000ac2:	1e5e      	subs	r6, r3, #1
 8000ac4:	2e00      	cmp	r6, #0
 8000ac6:	d000      	beq.n	8000aca <__aeabi_dadd+0x52>
 8000ac8:	e19e      	b.n	8000e08 <__aeabi_dadd+0x390>
 8000aca:	1a87      	subs	r7, r0, r2
 8000acc:	4643      	mov	r3, r8
 8000ace:	42b8      	cmp	r0, r7
 8000ad0:	4180      	sbcs	r0, r0
 8000ad2:	2501      	movs	r5, #1
 8000ad4:	1ac9      	subs	r1, r1, r3
 8000ad6:	4240      	negs	r0, r0
 8000ad8:	1a09      	subs	r1, r1, r0
 8000ada:	020b      	lsls	r3, r1, #8
 8000adc:	d400      	bmi.n	8000ae0 <__aeabi_dadd+0x68>
 8000ade:	e131      	b.n	8000d44 <__aeabi_dadd+0x2cc>
 8000ae0:	0249      	lsls	r1, r1, #9
 8000ae2:	0a4e      	lsrs	r6, r1, #9
 8000ae4:	2e00      	cmp	r6, #0
 8000ae6:	d100      	bne.n	8000aea <__aeabi_dadd+0x72>
 8000ae8:	e16e      	b.n	8000dc8 <__aeabi_dadd+0x350>
 8000aea:	0030      	movs	r0, r6
 8000aec:	f001 fd98 	bl	8002620 <__clzsi2>
 8000af0:	0003      	movs	r3, r0
 8000af2:	3b08      	subs	r3, #8
 8000af4:	2b1f      	cmp	r3, #31
 8000af6:	dd00      	ble.n	8000afa <__aeabi_dadd+0x82>
 8000af8:	e161      	b.n	8000dbe <__aeabi_dadd+0x346>
 8000afa:	2220      	movs	r2, #32
 8000afc:	0039      	movs	r1, r7
 8000afe:	1ad2      	subs	r2, r2, r3
 8000b00:	409e      	lsls	r6, r3
 8000b02:	40d1      	lsrs	r1, r2
 8000b04:	409f      	lsls	r7, r3
 8000b06:	430e      	orrs	r6, r1
 8000b08:	429d      	cmp	r5, r3
 8000b0a:	dd00      	ble.n	8000b0e <__aeabi_dadd+0x96>
 8000b0c:	e151      	b.n	8000db2 <__aeabi_dadd+0x33a>
 8000b0e:	1b5d      	subs	r5, r3, r5
 8000b10:	1c6b      	adds	r3, r5, #1
 8000b12:	2b1f      	cmp	r3, #31
 8000b14:	dd00      	ble.n	8000b18 <__aeabi_dadd+0xa0>
 8000b16:	e17c      	b.n	8000e12 <__aeabi_dadd+0x39a>
 8000b18:	2120      	movs	r1, #32
 8000b1a:	1ac9      	subs	r1, r1, r3
 8000b1c:	003d      	movs	r5, r7
 8000b1e:	0030      	movs	r0, r6
 8000b20:	408f      	lsls	r7, r1
 8000b22:	4088      	lsls	r0, r1
 8000b24:	40dd      	lsrs	r5, r3
 8000b26:	1e79      	subs	r1, r7, #1
 8000b28:	418f      	sbcs	r7, r1
 8000b2a:	0031      	movs	r1, r6
 8000b2c:	2207      	movs	r2, #7
 8000b2e:	4328      	orrs	r0, r5
 8000b30:	40d9      	lsrs	r1, r3
 8000b32:	2500      	movs	r5, #0
 8000b34:	4307      	orrs	r7, r0
 8000b36:	403a      	ands	r2, r7
 8000b38:	2a00      	cmp	r2, #0
 8000b3a:	d009      	beq.n	8000b50 <__aeabi_dadd+0xd8>
 8000b3c:	230f      	movs	r3, #15
 8000b3e:	403b      	ands	r3, r7
 8000b40:	2b04      	cmp	r3, #4
 8000b42:	d005      	beq.n	8000b50 <__aeabi_dadd+0xd8>
 8000b44:	1d3b      	adds	r3, r7, #4
 8000b46:	42bb      	cmp	r3, r7
 8000b48:	41bf      	sbcs	r7, r7
 8000b4a:	427f      	negs	r7, r7
 8000b4c:	19c9      	adds	r1, r1, r7
 8000b4e:	001f      	movs	r7, r3
 8000b50:	020b      	lsls	r3, r1, #8
 8000b52:	d400      	bmi.n	8000b56 <__aeabi_dadd+0xde>
 8000b54:	e226      	b.n	8000fa4 <__aeabi_dadd+0x52c>
 8000b56:	1c6a      	adds	r2, r5, #1
 8000b58:	4bc6      	ldr	r3, [pc, #792]	; (8000e74 <__aeabi_dadd+0x3fc>)
 8000b5a:	0555      	lsls	r5, r2, #21
 8000b5c:	0d6d      	lsrs	r5, r5, #21
 8000b5e:	429a      	cmp	r2, r3
 8000b60:	d100      	bne.n	8000b64 <__aeabi_dadd+0xec>
 8000b62:	e106      	b.n	8000d72 <__aeabi_dadd+0x2fa>
 8000b64:	4ac4      	ldr	r2, [pc, #784]	; (8000e78 <__aeabi_dadd+0x400>)
 8000b66:	08ff      	lsrs	r7, r7, #3
 8000b68:	400a      	ands	r2, r1
 8000b6a:	0753      	lsls	r3, r2, #29
 8000b6c:	0252      	lsls	r2, r2, #9
 8000b6e:	433b      	orrs	r3, r7
 8000b70:	0b12      	lsrs	r2, r2, #12
 8000b72:	e08e      	b.n	8000c92 <__aeabi_dadd+0x21a>
 8000b74:	2b00      	cmp	r3, #0
 8000b76:	d000      	beq.n	8000b7a <__aeabi_dadd+0x102>
 8000b78:	e0b8      	b.n	8000cec <__aeabi_dadd+0x274>
 8000b7a:	1c6b      	adds	r3, r5, #1
 8000b7c:	055b      	lsls	r3, r3, #21
 8000b7e:	0d5b      	lsrs	r3, r3, #21
 8000b80:	2b01      	cmp	r3, #1
 8000b82:	dc00      	bgt.n	8000b86 <__aeabi_dadd+0x10e>
 8000b84:	e130      	b.n	8000de8 <__aeabi_dadd+0x370>
 8000b86:	1a87      	subs	r7, r0, r2
 8000b88:	4643      	mov	r3, r8
 8000b8a:	42b8      	cmp	r0, r7
 8000b8c:	41b6      	sbcs	r6, r6
 8000b8e:	1acb      	subs	r3, r1, r3
 8000b90:	4276      	negs	r6, r6
 8000b92:	1b9e      	subs	r6, r3, r6
 8000b94:	0233      	lsls	r3, r6, #8
 8000b96:	d500      	bpl.n	8000b9a <__aeabi_dadd+0x122>
 8000b98:	e14c      	b.n	8000e34 <__aeabi_dadd+0x3bc>
 8000b9a:	003b      	movs	r3, r7
 8000b9c:	4333      	orrs	r3, r6
 8000b9e:	d1a1      	bne.n	8000ae4 <__aeabi_dadd+0x6c>
 8000ba0:	2200      	movs	r2, #0
 8000ba2:	2400      	movs	r4, #0
 8000ba4:	2500      	movs	r5, #0
 8000ba6:	e070      	b.n	8000c8a <__aeabi_dadd+0x212>
 8000ba8:	2b00      	cmp	r3, #0
 8000baa:	dc00      	bgt.n	8000bae <__aeabi_dadd+0x136>
 8000bac:	e0e5      	b.n	8000d7a <__aeabi_dadd+0x302>
 8000bae:	2e00      	cmp	r6, #0
 8000bb0:	d100      	bne.n	8000bb4 <__aeabi_dadd+0x13c>
 8000bb2:	e083      	b.n	8000cbc <__aeabi_dadd+0x244>
 8000bb4:	4eaf      	ldr	r6, [pc, #700]	; (8000e74 <__aeabi_dadd+0x3fc>)
 8000bb6:	42b5      	cmp	r5, r6
 8000bb8:	d060      	beq.n	8000c7c <__aeabi_dadd+0x204>
 8000bba:	2680      	movs	r6, #128	; 0x80
 8000bbc:	0436      	lsls	r6, r6, #16
 8000bbe:	4337      	orrs	r7, r6
 8000bc0:	46b8      	mov	r8, r7
 8000bc2:	2b38      	cmp	r3, #56	; 0x38
 8000bc4:	dc00      	bgt.n	8000bc8 <__aeabi_dadd+0x150>
 8000bc6:	e13e      	b.n	8000e46 <__aeabi_dadd+0x3ce>
 8000bc8:	4643      	mov	r3, r8
 8000bca:	4313      	orrs	r3, r2
 8000bcc:	001f      	movs	r7, r3
 8000bce:	1e7a      	subs	r2, r7, #1
 8000bd0:	4197      	sbcs	r7, r2
 8000bd2:	183f      	adds	r7, r7, r0
 8000bd4:	4287      	cmp	r7, r0
 8000bd6:	4180      	sbcs	r0, r0
 8000bd8:	4240      	negs	r0, r0
 8000bda:	1809      	adds	r1, r1, r0
 8000bdc:	020b      	lsls	r3, r1, #8
 8000bde:	d400      	bmi.n	8000be2 <__aeabi_dadd+0x16a>
 8000be0:	e0b0      	b.n	8000d44 <__aeabi_dadd+0x2cc>
 8000be2:	4ba4      	ldr	r3, [pc, #656]	; (8000e74 <__aeabi_dadd+0x3fc>)
 8000be4:	3501      	adds	r5, #1
 8000be6:	429d      	cmp	r5, r3
 8000be8:	d100      	bne.n	8000bec <__aeabi_dadd+0x174>
 8000bea:	e0c3      	b.n	8000d74 <__aeabi_dadd+0x2fc>
 8000bec:	4aa2      	ldr	r2, [pc, #648]	; (8000e78 <__aeabi_dadd+0x400>)
 8000bee:	087b      	lsrs	r3, r7, #1
 8000bf0:	400a      	ands	r2, r1
 8000bf2:	2101      	movs	r1, #1
 8000bf4:	400f      	ands	r7, r1
 8000bf6:	431f      	orrs	r7, r3
 8000bf8:	0851      	lsrs	r1, r2, #1
 8000bfa:	07d3      	lsls	r3, r2, #31
 8000bfc:	2207      	movs	r2, #7
 8000bfe:	431f      	orrs	r7, r3
 8000c00:	403a      	ands	r2, r7
 8000c02:	e799      	b.n	8000b38 <__aeabi_dadd+0xc0>
 8000c04:	4e9b      	ldr	r6, [pc, #620]	; (8000e74 <__aeabi_dadd+0x3fc>)
 8000c06:	42b5      	cmp	r5, r6
 8000c08:	d038      	beq.n	8000c7c <__aeabi_dadd+0x204>
 8000c0a:	2680      	movs	r6, #128	; 0x80
 8000c0c:	0436      	lsls	r6, r6, #16
 8000c0e:	4337      	orrs	r7, r6
 8000c10:	46b8      	mov	r8, r7
 8000c12:	2b38      	cmp	r3, #56	; 0x38
 8000c14:	dd00      	ble.n	8000c18 <__aeabi_dadd+0x1a0>
 8000c16:	e0dc      	b.n	8000dd2 <__aeabi_dadd+0x35a>
 8000c18:	2b1f      	cmp	r3, #31
 8000c1a:	dc00      	bgt.n	8000c1e <__aeabi_dadd+0x1a6>
 8000c1c:	e130      	b.n	8000e80 <__aeabi_dadd+0x408>
 8000c1e:	001e      	movs	r6, r3
 8000c20:	4647      	mov	r7, r8
 8000c22:	3e20      	subs	r6, #32
 8000c24:	40f7      	lsrs	r7, r6
 8000c26:	46bc      	mov	ip, r7
 8000c28:	2b20      	cmp	r3, #32
 8000c2a:	d004      	beq.n	8000c36 <__aeabi_dadd+0x1be>
 8000c2c:	2640      	movs	r6, #64	; 0x40
 8000c2e:	1af3      	subs	r3, r6, r3
 8000c30:	4646      	mov	r6, r8
 8000c32:	409e      	lsls	r6, r3
 8000c34:	4332      	orrs	r2, r6
 8000c36:	0017      	movs	r7, r2
 8000c38:	4663      	mov	r3, ip
 8000c3a:	1e7a      	subs	r2, r7, #1
 8000c3c:	4197      	sbcs	r7, r2
 8000c3e:	431f      	orrs	r7, r3
 8000c40:	e0cc      	b.n	8000ddc <__aeabi_dadd+0x364>
 8000c42:	2b00      	cmp	r3, #0
 8000c44:	d100      	bne.n	8000c48 <__aeabi_dadd+0x1d0>
 8000c46:	e204      	b.n	8001052 <__aeabi_dadd+0x5da>
 8000c48:	4643      	mov	r3, r8
 8000c4a:	4313      	orrs	r3, r2
 8000c4c:	d100      	bne.n	8000c50 <__aeabi_dadd+0x1d8>
 8000c4e:	e159      	b.n	8000f04 <__aeabi_dadd+0x48c>
 8000c50:	074b      	lsls	r3, r1, #29
 8000c52:	08c0      	lsrs	r0, r0, #3
 8000c54:	4318      	orrs	r0, r3
 8000c56:	2380      	movs	r3, #128	; 0x80
 8000c58:	08c9      	lsrs	r1, r1, #3
 8000c5a:	031b      	lsls	r3, r3, #12
 8000c5c:	4219      	tst	r1, r3
 8000c5e:	d008      	beq.n	8000c72 <__aeabi_dadd+0x1fa>
 8000c60:	4645      	mov	r5, r8
 8000c62:	08ed      	lsrs	r5, r5, #3
 8000c64:	421d      	tst	r5, r3
 8000c66:	d104      	bne.n	8000c72 <__aeabi_dadd+0x1fa>
 8000c68:	4643      	mov	r3, r8
 8000c6a:	08d0      	lsrs	r0, r2, #3
 8000c6c:	0759      	lsls	r1, r3, #29
 8000c6e:	4308      	orrs	r0, r1
 8000c70:	0029      	movs	r1, r5
 8000c72:	0f42      	lsrs	r2, r0, #29
 8000c74:	00c9      	lsls	r1, r1, #3
 8000c76:	4d7f      	ldr	r5, [pc, #508]	; (8000e74 <__aeabi_dadd+0x3fc>)
 8000c78:	4311      	orrs	r1, r2
 8000c7a:	00c0      	lsls	r0, r0, #3
 8000c7c:	074b      	lsls	r3, r1, #29
 8000c7e:	08ca      	lsrs	r2, r1, #3
 8000c80:	497c      	ldr	r1, [pc, #496]	; (8000e74 <__aeabi_dadd+0x3fc>)
 8000c82:	08c0      	lsrs	r0, r0, #3
 8000c84:	4303      	orrs	r3, r0
 8000c86:	428d      	cmp	r5, r1
 8000c88:	d068      	beq.n	8000d5c <__aeabi_dadd+0x2e4>
 8000c8a:	0312      	lsls	r2, r2, #12
 8000c8c:	056d      	lsls	r5, r5, #21
 8000c8e:	0b12      	lsrs	r2, r2, #12
 8000c90:	0d6d      	lsrs	r5, r5, #21
 8000c92:	2100      	movs	r1, #0
 8000c94:	0312      	lsls	r2, r2, #12
 8000c96:	0018      	movs	r0, r3
 8000c98:	0b13      	lsrs	r3, r2, #12
 8000c9a:	0d0a      	lsrs	r2, r1, #20
 8000c9c:	0512      	lsls	r2, r2, #20
 8000c9e:	431a      	orrs	r2, r3
 8000ca0:	4b76      	ldr	r3, [pc, #472]	; (8000e7c <__aeabi_dadd+0x404>)
 8000ca2:	052d      	lsls	r5, r5, #20
 8000ca4:	4013      	ands	r3, r2
 8000ca6:	432b      	orrs	r3, r5
 8000ca8:	005b      	lsls	r3, r3, #1
 8000caa:	07e4      	lsls	r4, r4, #31
 8000cac:	085b      	lsrs	r3, r3, #1
 8000cae:	4323      	orrs	r3, r4
 8000cb0:	0019      	movs	r1, r3
 8000cb2:	bc1c      	pop	{r2, r3, r4}
 8000cb4:	4690      	mov	r8, r2
 8000cb6:	4699      	mov	r9, r3
 8000cb8:	46a2      	mov	sl, r4
 8000cba:	bdf0      	pop	{r4, r5, r6, r7, pc}
 8000cbc:	003e      	movs	r6, r7
 8000cbe:	4316      	orrs	r6, r2
 8000cc0:	d012      	beq.n	8000ce8 <__aeabi_dadd+0x270>
 8000cc2:	1e5e      	subs	r6, r3, #1
 8000cc4:	2e00      	cmp	r6, #0
 8000cc6:	d000      	beq.n	8000cca <__aeabi_dadd+0x252>
 8000cc8:	e100      	b.n	8000ecc <__aeabi_dadd+0x454>
 8000cca:	1887      	adds	r7, r0, r2
 8000ccc:	4287      	cmp	r7, r0
 8000cce:	4180      	sbcs	r0, r0
 8000cd0:	4441      	add	r1, r8
 8000cd2:	4240      	negs	r0, r0
 8000cd4:	1809      	adds	r1, r1, r0
 8000cd6:	2501      	movs	r5, #1
 8000cd8:	020b      	lsls	r3, r1, #8
 8000cda:	d533      	bpl.n	8000d44 <__aeabi_dadd+0x2cc>
 8000cdc:	2502      	movs	r5, #2
 8000cde:	e785      	b.n	8000bec <__aeabi_dadd+0x174>
 8000ce0:	4664      	mov	r4, ip
 8000ce2:	0033      	movs	r3, r6
 8000ce4:	4641      	mov	r1, r8
 8000ce6:	0010      	movs	r0, r2
 8000ce8:	001d      	movs	r5, r3
 8000cea:	e7c7      	b.n	8000c7c <__aeabi_dadd+0x204>
 8000cec:	2d00      	cmp	r5, #0
 8000cee:	d000      	beq.n	8000cf2 <__aeabi_dadd+0x27a>
 8000cf0:	e0da      	b.n	8000ea8 <__aeabi_dadd+0x430>
 8000cf2:	000c      	movs	r4, r1
 8000cf4:	4304      	orrs	r4, r0
 8000cf6:	d0f3      	beq.n	8000ce0 <__aeabi_dadd+0x268>
 8000cf8:	1c5c      	adds	r4, r3, #1
 8000cfa:	d100      	bne.n	8000cfe <__aeabi_dadd+0x286>
 8000cfc:	e19f      	b.n	800103e <__aeabi_dadd+0x5c6>
 8000cfe:	4c5d      	ldr	r4, [pc, #372]	; (8000e74 <__aeabi_dadd+0x3fc>)
 8000d00:	42a6      	cmp	r6, r4
 8000d02:	d100      	bne.n	8000d06 <__aeabi_dadd+0x28e>
 8000d04:	e12f      	b.n	8000f66 <__aeabi_dadd+0x4ee>
 8000d06:	43db      	mvns	r3, r3
 8000d08:	2b38      	cmp	r3, #56	; 0x38
 8000d0a:	dd00      	ble.n	8000d0e <__aeabi_dadd+0x296>
 8000d0c:	e166      	b.n	8000fdc <__aeabi_dadd+0x564>
 8000d0e:	2b1f      	cmp	r3, #31
 8000d10:	dd00      	ble.n	8000d14 <__aeabi_dadd+0x29c>
 8000d12:	e183      	b.n	800101c <__aeabi_dadd+0x5a4>
 8000d14:	2420      	movs	r4, #32
 8000d16:	0005      	movs	r5, r0
 8000d18:	1ae4      	subs	r4, r4, r3
 8000d1a:	000f      	movs	r7, r1
 8000d1c:	40dd      	lsrs	r5, r3
 8000d1e:	40d9      	lsrs	r1, r3
 8000d20:	40a0      	lsls	r0, r4
 8000d22:	4643      	mov	r3, r8
 8000d24:	40a7      	lsls	r7, r4
 8000d26:	1a5b      	subs	r3, r3, r1
 8000d28:	1e44      	subs	r4, r0, #1
 8000d2a:	41a0      	sbcs	r0, r4
 8000d2c:	4698      	mov	r8, r3
 8000d2e:	432f      	orrs	r7, r5
 8000d30:	4338      	orrs	r0, r7
 8000d32:	1a17      	subs	r7, r2, r0
 8000d34:	42ba      	cmp	r2, r7
 8000d36:	4192      	sbcs	r2, r2
 8000d38:	4643      	mov	r3, r8
 8000d3a:	4252      	negs	r2, r2
 8000d3c:	1a99      	subs	r1, r3, r2
 8000d3e:	4664      	mov	r4, ip
 8000d40:	0035      	movs	r5, r6
 8000d42:	e6ca      	b.n	8000ada <__aeabi_dadd+0x62>
 8000d44:	2207      	movs	r2, #7
 8000d46:	403a      	ands	r2, r7
 8000d48:	2a00      	cmp	r2, #0
 8000d4a:	d000      	beq.n	8000d4e <__aeabi_dadd+0x2d6>
 8000d4c:	e6f6      	b.n	8000b3c <__aeabi_dadd+0xc4>
 8000d4e:	074b      	lsls	r3, r1, #29
 8000d50:	08ca      	lsrs	r2, r1, #3
 8000d52:	4948      	ldr	r1, [pc, #288]	; (8000e74 <__aeabi_dadd+0x3fc>)
 8000d54:	08ff      	lsrs	r7, r7, #3
 8000d56:	433b      	orrs	r3, r7
 8000d58:	428d      	cmp	r5, r1
 8000d5a:	d196      	bne.n	8000c8a <__aeabi_dadd+0x212>
 8000d5c:	0019      	movs	r1, r3
 8000d5e:	4311      	orrs	r1, r2
 8000d60:	d100      	bne.n	8000d64 <__aeabi_dadd+0x2ec>
 8000d62:	e19e      	b.n	80010a2 <__aeabi_dadd+0x62a>
 8000d64:	2180      	movs	r1, #128	; 0x80
 8000d66:	0309      	lsls	r1, r1, #12
 8000d68:	430a      	orrs	r2, r1
 8000d6a:	0312      	lsls	r2, r2, #12
 8000d6c:	0b12      	lsrs	r2, r2, #12
 8000d6e:	4d41      	ldr	r5, [pc, #260]	; (8000e74 <__aeabi_dadd+0x3fc>)
 8000d70:	e78f      	b.n	8000c92 <__aeabi_dadd+0x21a>
 8000d72:	0015      	movs	r5, r2
 8000d74:	2200      	movs	r2, #0
 8000d76:	2300      	movs	r3, #0
 8000d78:	e78b      	b.n	8000c92 <__aeabi_dadd+0x21a>
 8000d7a:	2b00      	cmp	r3, #0
 8000d7c:	d000      	beq.n	8000d80 <__aeabi_dadd+0x308>
 8000d7e:	e0c7      	b.n	8000f10 <__aeabi_dadd+0x498>
 8000d80:	1c6b      	adds	r3, r5, #1
 8000d82:	055f      	lsls	r7, r3, #21
 8000d84:	0d7f      	lsrs	r7, r7, #21
 8000d86:	2f01      	cmp	r7, #1
 8000d88:	dc00      	bgt.n	8000d8c <__aeabi_dadd+0x314>
 8000d8a:	e0f1      	b.n	8000f70 <__aeabi_dadd+0x4f8>
 8000d8c:	4d39      	ldr	r5, [pc, #228]	; (8000e74 <__aeabi_dadd+0x3fc>)
 8000d8e:	42ab      	cmp	r3, r5
 8000d90:	d100      	bne.n	8000d94 <__aeabi_dadd+0x31c>
 8000d92:	e0b9      	b.n	8000f08 <__aeabi_dadd+0x490>
 8000d94:	1885      	adds	r5, r0, r2
 8000d96:	000a      	movs	r2, r1
 8000d98:	4285      	cmp	r5, r0
 8000d9a:	4189      	sbcs	r1, r1
 8000d9c:	4442      	add	r2, r8
 8000d9e:	4249      	negs	r1, r1
 8000da0:	1851      	adds	r1, r2, r1
 8000da2:	2207      	movs	r2, #7
 8000da4:	07cf      	lsls	r7, r1, #31
 8000da6:	086d      	lsrs	r5, r5, #1
 8000da8:	432f      	orrs	r7, r5
 8000daa:	0849      	lsrs	r1, r1, #1
 8000dac:	403a      	ands	r2, r7
 8000dae:	001d      	movs	r5, r3
 8000db0:	e6c2      	b.n	8000b38 <__aeabi_dadd+0xc0>
 8000db2:	2207      	movs	r2, #7
 8000db4:	4930      	ldr	r1, [pc, #192]	; (8000e78 <__aeabi_dadd+0x400>)
 8000db6:	1aed      	subs	r5, r5, r3
 8000db8:	4031      	ands	r1, r6
 8000dba:	403a      	ands	r2, r7
 8000dbc:	e6bc      	b.n	8000b38 <__aeabi_dadd+0xc0>
 8000dbe:	003e      	movs	r6, r7
 8000dc0:	3828      	subs	r0, #40	; 0x28
 8000dc2:	4086      	lsls	r6, r0
 8000dc4:	2700      	movs	r7, #0
 8000dc6:	e69f      	b.n	8000b08 <__aeabi_dadd+0x90>
 8000dc8:	0038      	movs	r0, r7
 8000dca:	f001 fc29 	bl	8002620 <__clzsi2>
 8000dce:	3020      	adds	r0, #32
 8000dd0:	e68e      	b.n	8000af0 <__aeabi_dadd+0x78>
 8000dd2:	4643      	mov	r3, r8
 8000dd4:	4313      	orrs	r3, r2
 8000dd6:	001f      	movs	r7, r3
 8000dd8:	1e7a      	subs	r2, r7, #1
 8000dda:	4197      	sbcs	r7, r2
 8000ddc:	1bc7      	subs	r7, r0, r7
 8000dde:	42b8      	cmp	r0, r7
 8000de0:	4180      	sbcs	r0, r0
 8000de2:	4240      	negs	r0, r0
 8000de4:	1a09      	subs	r1, r1, r0
 8000de6:	e678      	b.n	8000ada <__aeabi_dadd+0x62>
 8000de8:	000e      	movs	r6, r1
 8000dea:	003b      	movs	r3, r7
 8000dec:	4306      	orrs	r6, r0
 8000dee:	4313      	orrs	r3, r2
 8000df0:	2d00      	cmp	r5, #0
 8000df2:	d161      	bne.n	8000eb8 <__aeabi_dadd+0x440>
 8000df4:	2e00      	cmp	r6, #0
 8000df6:	d000      	beq.n	8000dfa <__aeabi_dadd+0x382>
 8000df8:	e0f4      	b.n	8000fe4 <__aeabi_dadd+0x56c>
 8000dfa:	2b00      	cmp	r3, #0
 8000dfc:	d100      	bne.n	8000e00 <__aeabi_dadd+0x388>
 8000dfe:	e11b      	b.n	8001038 <__aeabi_dadd+0x5c0>
 8000e00:	4664      	mov	r4, ip
 8000e02:	0039      	movs	r1, r7
 8000e04:	0010      	movs	r0, r2
 8000e06:	e739      	b.n	8000c7c <__aeabi_dadd+0x204>
 8000e08:	4f1a      	ldr	r7, [pc, #104]	; (8000e74 <__aeabi_dadd+0x3fc>)
 8000e0a:	42bb      	cmp	r3, r7
 8000e0c:	d07a      	beq.n	8000f04 <__aeabi_dadd+0x48c>
 8000e0e:	0033      	movs	r3, r6
 8000e10:	e6ff      	b.n	8000c12 <__aeabi_dadd+0x19a>
 8000e12:	0030      	movs	r0, r6
 8000e14:	3d1f      	subs	r5, #31
 8000e16:	40e8      	lsrs	r0, r5
 8000e18:	2b20      	cmp	r3, #32
 8000e1a:	d003      	beq.n	8000e24 <__aeabi_dadd+0x3ac>
 8000e1c:	2140      	movs	r1, #64	; 0x40
 8000e1e:	1acb      	subs	r3, r1, r3
 8000e20:	409e      	lsls	r6, r3
 8000e22:	4337      	orrs	r7, r6
 8000e24:	1e7b      	subs	r3, r7, #1
 8000e26:	419f      	sbcs	r7, r3
 8000e28:	2207      	movs	r2, #7
 8000e2a:	4307      	orrs	r7, r0
 8000e2c:	403a      	ands	r2, r7
 8000e2e:	2100      	movs	r1, #0
 8000e30:	2500      	movs	r5, #0
 8000e32:	e789      	b.n	8000d48 <__aeabi_dadd+0x2d0>
 8000e34:	1a17      	subs	r7, r2, r0
 8000e36:	4643      	mov	r3, r8
 8000e38:	42ba      	cmp	r2, r7
 8000e3a:	41b6      	sbcs	r6, r6
 8000e3c:	1a59      	subs	r1, r3, r1
 8000e3e:	4276      	negs	r6, r6
 8000e40:	1b8e      	subs	r6, r1, r6
 8000e42:	4664      	mov	r4, ip
 8000e44:	e64e      	b.n	8000ae4 <__aeabi_dadd+0x6c>
 8000e46:	2b1f      	cmp	r3, #31
 8000e48:	dd00      	ble.n	8000e4c <__aeabi_dadd+0x3d4>
 8000e4a:	e0ad      	b.n	8000fa8 <__aeabi_dadd+0x530>
 8000e4c:	2620      	movs	r6, #32
 8000e4e:	4647      	mov	r7, r8
 8000e50:	1af6      	subs	r6, r6, r3
 8000e52:	40b7      	lsls	r7, r6
 8000e54:	46b9      	mov	r9, r7
 8000e56:	0017      	movs	r7, r2
 8000e58:	46b2      	mov	sl, r6
 8000e5a:	40df      	lsrs	r7, r3
 8000e5c:	464e      	mov	r6, r9
 8000e5e:	433e      	orrs	r6, r7
 8000e60:	0037      	movs	r7, r6
 8000e62:	4656      	mov	r6, sl
 8000e64:	40b2      	lsls	r2, r6
 8000e66:	1e56      	subs	r6, r2, #1
 8000e68:	41b2      	sbcs	r2, r6
 8000e6a:	4317      	orrs	r7, r2
 8000e6c:	4642      	mov	r2, r8
 8000e6e:	40da      	lsrs	r2, r3
 8000e70:	1889      	adds	r1, r1, r2
 8000e72:	e6ae      	b.n	8000bd2 <__aeabi_dadd+0x15a>
 8000e74:	000007ff 	.word	0x000007ff
 8000e78:	ff7fffff 	.word	0xff7fffff
 8000e7c:	800fffff 	.word	0x800fffff
 8000e80:	2620      	movs	r6, #32
 8000e82:	4647      	mov	r7, r8
 8000e84:	1af6      	subs	r6, r6, r3
 8000e86:	40b7      	lsls	r7, r6
 8000e88:	46b9      	mov	r9, r7
 8000e8a:	0017      	movs	r7, r2
 8000e8c:	46b2      	mov	sl, r6
 8000e8e:	40df      	lsrs	r7, r3
 8000e90:	464e      	mov	r6, r9
 8000e92:	433e      	orrs	r6, r7
 8000e94:	0037      	movs	r7, r6
 8000e96:	4656      	mov	r6, sl
 8000e98:	40b2      	lsls	r2, r6
 8000e9a:	1e56      	subs	r6, r2, #1
 8000e9c:	41b2      	sbcs	r2, r6
 8000e9e:	4317      	orrs	r7, r2
 8000ea0:	4642      	mov	r2, r8
 8000ea2:	40da      	lsrs	r2, r3
 8000ea4:	1a89      	subs	r1, r1, r2
 8000ea6:	e799      	b.n	8000ddc <__aeabi_dadd+0x364>
 8000ea8:	4c7f      	ldr	r4, [pc, #508]	; (80010a8 <__aeabi_dadd+0x630>)
 8000eaa:	42a6      	cmp	r6, r4
 8000eac:	d05b      	beq.n	8000f66 <__aeabi_dadd+0x4ee>
 8000eae:	2480      	movs	r4, #128	; 0x80
 8000eb0:	0424      	lsls	r4, r4, #16
 8000eb2:	425b      	negs	r3, r3
 8000eb4:	4321      	orrs	r1, r4
 8000eb6:	e727      	b.n	8000d08 <__aeabi_dadd+0x290>
 8000eb8:	2e00      	cmp	r6, #0
 8000eba:	d10c      	bne.n	8000ed6 <__aeabi_dadd+0x45e>
 8000ebc:	2b00      	cmp	r3, #0
 8000ebe:	d100      	bne.n	8000ec2 <__aeabi_dadd+0x44a>
 8000ec0:	e0cb      	b.n	800105a <__aeabi_dadd+0x5e2>
 8000ec2:	4664      	mov	r4, ip
 8000ec4:	0039      	movs	r1, r7
 8000ec6:	0010      	movs	r0, r2
 8000ec8:	4d77      	ldr	r5, [pc, #476]	; (80010a8 <__aeabi_dadd+0x630>)
 8000eca:	e6d7      	b.n	8000c7c <__aeabi_dadd+0x204>
 8000ecc:	4f76      	ldr	r7, [pc, #472]	; (80010a8 <__aeabi_dadd+0x630>)
 8000ece:	42bb      	cmp	r3, r7
 8000ed0:	d018      	beq.n	8000f04 <__aeabi_dadd+0x48c>
 8000ed2:	0033      	movs	r3, r6
 8000ed4:	e675      	b.n	8000bc2 <__aeabi_dadd+0x14a>
 8000ed6:	2b00      	cmp	r3, #0
 8000ed8:	d014      	beq.n	8000f04 <__aeabi_dadd+0x48c>
 8000eda:	074b      	lsls	r3, r1, #29
 8000edc:	08c0      	lsrs	r0, r0, #3
 8000ede:	4318      	orrs	r0, r3
 8000ee0:	2380      	movs	r3, #128	; 0x80
 8000ee2:	08c9      	lsrs	r1, r1, #3
 8000ee4:	031b      	lsls	r3, r3, #12
 8000ee6:	4219      	tst	r1, r3
 8000ee8:	d007      	beq.n	8000efa <__aeabi_dadd+0x482>
 8000eea:	08fc      	lsrs	r4, r7, #3
 8000eec:	421c      	tst	r4, r3
 8000eee:	d104      	bne.n	8000efa <__aeabi_dadd+0x482>
 8000ef0:	0779      	lsls	r1, r7, #29
 8000ef2:	08d0      	lsrs	r0, r2, #3
 8000ef4:	4308      	orrs	r0, r1
 8000ef6:	46e1      	mov	r9, ip
 8000ef8:	0021      	movs	r1, r4
 8000efa:	464c      	mov	r4, r9
 8000efc:	0f42      	lsrs	r2, r0, #29
 8000efe:	00c9      	lsls	r1, r1, #3
 8000f00:	4311      	orrs	r1, r2
 8000f02:	00c0      	lsls	r0, r0, #3
 8000f04:	4d68      	ldr	r5, [pc, #416]	; (80010a8 <__aeabi_dadd+0x630>)
 8000f06:	e6b9      	b.n	8000c7c <__aeabi_dadd+0x204>
 8000f08:	001d      	movs	r5, r3
 8000f0a:	2200      	movs	r2, #0
 8000f0c:	2300      	movs	r3, #0
 8000f0e:	e6c0      	b.n	8000c92 <__aeabi_dadd+0x21a>
 8000f10:	2d00      	cmp	r5, #0
 8000f12:	d15b      	bne.n	8000fcc <__aeabi_dadd+0x554>
 8000f14:	000d      	movs	r5, r1
 8000f16:	4305      	orrs	r5, r0
 8000f18:	d100      	bne.n	8000f1c <__aeabi_dadd+0x4a4>
 8000f1a:	e6e2      	b.n	8000ce2 <__aeabi_dadd+0x26a>
 8000f1c:	1c5d      	adds	r5, r3, #1
 8000f1e:	d100      	bne.n	8000f22 <__aeabi_dadd+0x4aa>
 8000f20:	e0b0      	b.n	8001084 <__aeabi_dadd+0x60c>
 8000f22:	4d61      	ldr	r5, [pc, #388]	; (80010a8 <__aeabi_dadd+0x630>)
 8000f24:	42ae      	cmp	r6, r5
 8000f26:	d01f      	beq.n	8000f68 <__aeabi_dadd+0x4f0>
 8000f28:	43db      	mvns	r3, r3
 8000f2a:	2b38      	cmp	r3, #56	; 0x38
 8000f2c:	dc71      	bgt.n	8001012 <__aeabi_dadd+0x59a>
 8000f2e:	2b1f      	cmp	r3, #31
 8000f30:	dd00      	ble.n	8000f34 <__aeabi_dadd+0x4bc>
 8000f32:	e096      	b.n	8001062 <__aeabi_dadd+0x5ea>
 8000f34:	2520      	movs	r5, #32
 8000f36:	000f      	movs	r7, r1
 8000f38:	1aed      	subs	r5, r5, r3
 8000f3a:	40af      	lsls	r7, r5
 8000f3c:	46b9      	mov	r9, r7
 8000f3e:	0007      	movs	r7, r0
 8000f40:	46aa      	mov	sl, r5
 8000f42:	40df      	lsrs	r7, r3
 8000f44:	464d      	mov	r5, r9
 8000f46:	433d      	orrs	r5, r7
 8000f48:	002f      	movs	r7, r5
 8000f4a:	4655      	mov	r5, sl
 8000f4c:	40a8      	lsls	r0, r5
 8000f4e:	40d9      	lsrs	r1, r3
 8000f50:	1e45      	subs	r5, r0, #1
 8000f52:	41a8      	sbcs	r0, r5
 8000f54:	4488      	add	r8, r1
 8000f56:	4307      	orrs	r7, r0
 8000f58:	18bf      	adds	r7, r7, r2
 8000f5a:	4297      	cmp	r7, r2
 8000f5c:	4192      	sbcs	r2, r2
 8000f5e:	4251      	negs	r1, r2
 8000f60:	4441      	add	r1, r8
 8000f62:	0035      	movs	r5, r6
 8000f64:	e63a      	b.n	8000bdc <__aeabi_dadd+0x164>
 8000f66:	4664      	mov	r4, ip
 8000f68:	0035      	movs	r5, r6
 8000f6a:	4641      	mov	r1, r8
 8000f6c:	0010      	movs	r0, r2
 8000f6e:	e685      	b.n	8000c7c <__aeabi_dadd+0x204>
 8000f70:	000b      	movs	r3, r1
 8000f72:	4303      	orrs	r3, r0
 8000f74:	2d00      	cmp	r5, #0
 8000f76:	d000      	beq.n	8000f7a <__aeabi_dadd+0x502>
 8000f78:	e663      	b.n	8000c42 <__aeabi_dadd+0x1ca>
 8000f7a:	2b00      	cmp	r3, #0
 8000f7c:	d0f5      	beq.n	8000f6a <__aeabi_dadd+0x4f2>
 8000f7e:	4643      	mov	r3, r8
 8000f80:	4313      	orrs	r3, r2
 8000f82:	d100      	bne.n	8000f86 <__aeabi_dadd+0x50e>
 8000f84:	e67a      	b.n	8000c7c <__aeabi_dadd+0x204>
 8000f86:	1887      	adds	r7, r0, r2
 8000f88:	4287      	cmp	r7, r0
 8000f8a:	4180      	sbcs	r0, r0
 8000f8c:	2207      	movs	r2, #7
 8000f8e:	4441      	add	r1, r8
 8000f90:	4240      	negs	r0, r0
 8000f92:	1809      	adds	r1, r1, r0
 8000f94:	403a      	ands	r2, r7
 8000f96:	020b      	lsls	r3, r1, #8
 8000f98:	d400      	bmi.n	8000f9c <__aeabi_dadd+0x524>
 8000f9a:	e6d5      	b.n	8000d48 <__aeabi_dadd+0x2d0>
 8000f9c:	4b43      	ldr	r3, [pc, #268]	; (80010ac <__aeabi_dadd+0x634>)
 8000f9e:	3501      	adds	r5, #1
 8000fa0:	4019      	ands	r1, r3
 8000fa2:	e5c9      	b.n	8000b38 <__aeabi_dadd+0xc0>
 8000fa4:	0038      	movs	r0, r7
 8000fa6:	e669      	b.n	8000c7c <__aeabi_dadd+0x204>
 8000fa8:	001e      	movs	r6, r3
 8000faa:	4647      	mov	r7, r8
 8000fac:	3e20      	subs	r6, #32
 8000fae:	40f7      	lsrs	r7, r6
 8000fb0:	46bc      	mov	ip, r7
 8000fb2:	2b20      	cmp	r3, #32
 8000fb4:	d004      	beq.n	8000fc0 <__aeabi_dadd+0x548>
 8000fb6:	2640      	movs	r6, #64	; 0x40
 8000fb8:	1af3      	subs	r3, r6, r3
 8000fba:	4646      	mov	r6, r8
 8000fbc:	409e      	lsls	r6, r3
 8000fbe:	4332      	orrs	r2, r6
 8000fc0:	0017      	movs	r7, r2
 8000fc2:	4663      	mov	r3, ip
 8000fc4:	1e7a      	subs	r2, r7, #1
 8000fc6:	4197      	sbcs	r7, r2
 8000fc8:	431f      	orrs	r7, r3
 8000fca:	e602      	b.n	8000bd2 <__aeabi_dadd+0x15a>
 8000fcc:	4d36      	ldr	r5, [pc, #216]	; (80010a8 <__aeabi_dadd+0x630>)
 8000fce:	42ae      	cmp	r6, r5
 8000fd0:	d0ca      	beq.n	8000f68 <__aeabi_dadd+0x4f0>
 8000fd2:	2580      	movs	r5, #128	; 0x80
 8000fd4:	042d      	lsls	r5, r5, #16
 8000fd6:	425b      	negs	r3, r3
 8000fd8:	4329      	orrs	r1, r5
 8000fda:	e7a6      	b.n	8000f2a <__aeabi_dadd+0x4b2>
 8000fdc:	4308      	orrs	r0, r1
 8000fde:	1e41      	subs	r1, r0, #1
 8000fe0:	4188      	sbcs	r0, r1
 8000fe2:	e6a6      	b.n	8000d32 <__aeabi_dadd+0x2ba>
 8000fe4:	2b00      	cmp	r3, #0
 8000fe6:	d100      	bne.n	8000fea <__aeabi_dadd+0x572>
 8000fe8:	e648      	b.n	8000c7c <__aeabi_dadd+0x204>
 8000fea:	1a87      	subs	r7, r0, r2
 8000fec:	4643      	mov	r3, r8
 8000fee:	42b8      	cmp	r0, r7
 8000ff0:	41b6      	sbcs	r6, r6
 8000ff2:	1acb      	subs	r3, r1, r3
 8000ff4:	4276      	negs	r6, r6
 8000ff6:	1b9e      	subs	r6, r3, r6
 8000ff8:	0233      	lsls	r3, r6, #8
 8000ffa:	d54b      	bpl.n	8001094 <__aeabi_dadd+0x61c>
 8000ffc:	1a17      	subs	r7, r2, r0
 8000ffe:	4643      	mov	r3, r8
 8001000:	42ba      	cmp	r2, r7
 8001002:	4192      	sbcs	r2, r2
 8001004:	1a59      	subs	r1, r3, r1
 8001006:	4252      	negs	r2, r2
 8001008:	1a89      	subs	r1, r1, r2
 800100a:	2207      	movs	r2, #7
 800100c:	4664      	mov	r4, ip
 800100e:	403a      	ands	r2, r7
 8001010:	e592      	b.n	8000b38 <__aeabi_dadd+0xc0>
 8001012:	4301      	orrs	r1, r0
 8001014:	000f      	movs	r7, r1
 8001016:	1e79      	subs	r1, r7, #1
 8001018:	418f      	sbcs	r7, r1
 800101a:	e79d      	b.n	8000f58 <__aeabi_dadd+0x4e0>
 800101c:	001c      	movs	r4, r3
 800101e:	000f      	movs	r7, r1
 8001020:	3c20      	subs	r4, #32
 8001022:	40e7      	lsrs	r7, r4
 8001024:	2b20      	cmp	r3, #32
 8001026:	d003      	beq.n	8001030 <__aeabi_dadd+0x5b8>
 8001028:	2440      	movs	r4, #64	; 0x40
 800102a:	1ae3      	subs	r3, r4, r3
 800102c:	4099      	lsls	r1, r3
 800102e:	4308      	orrs	r0, r1
 8001030:	1e41      	subs	r1, r0, #1
 8001032:	4188      	sbcs	r0, r1
 8001034:	4338      	orrs	r0, r7
 8001036:	e67c      	b.n	8000d32 <__aeabi_dadd+0x2ba>
 8001038:	2200      	movs	r2, #0
 800103a:	2400      	movs	r4, #0
 800103c:	e625      	b.n	8000c8a <__aeabi_dadd+0x212>
 800103e:	1a17      	subs	r7, r2, r0
 8001040:	4643      	mov	r3, r8
 8001042:	42ba      	cmp	r2, r7
 8001044:	4192      	sbcs	r2, r2
 8001046:	1a59      	subs	r1, r3, r1
 8001048:	4252      	negs	r2, r2
 800104a:	1a89      	subs	r1, r1, r2
 800104c:	4664      	mov	r4, ip
 800104e:	0035      	movs	r5, r6
 8001050:	e543      	b.n	8000ada <__aeabi_dadd+0x62>
 8001052:	4641      	mov	r1, r8
 8001054:	0010      	movs	r0, r2
 8001056:	4d14      	ldr	r5, [pc, #80]	; (80010a8 <__aeabi_dadd+0x630>)
 8001058:	e610      	b.n	8000c7c <__aeabi_dadd+0x204>
 800105a:	2280      	movs	r2, #128	; 0x80
 800105c:	2400      	movs	r4, #0
 800105e:	0312      	lsls	r2, r2, #12
 8001060:	e680      	b.n	8000d64 <__aeabi_dadd+0x2ec>
 8001062:	001d      	movs	r5, r3
 8001064:	000f      	movs	r7, r1
 8001066:	3d20      	subs	r5, #32
 8001068:	40ef      	lsrs	r7, r5
 800106a:	46bc      	mov	ip, r7
 800106c:	2b20      	cmp	r3, #32
 800106e:	d003      	beq.n	8001078 <__aeabi_dadd+0x600>
 8001070:	2540      	movs	r5, #64	; 0x40
 8001072:	1aeb      	subs	r3, r5, r3
 8001074:	4099      	lsls	r1, r3
 8001076:	4308      	orrs	r0, r1
 8001078:	0007      	movs	r7, r0
 800107a:	4663      	mov	r3, ip
 800107c:	1e78      	subs	r0, r7, #1
 800107e:	4187      	sbcs	r7, r0
 8001080:	431f      	orrs	r7, r3
 8001082:	e769      	b.n	8000f58 <__aeabi_dadd+0x4e0>
 8001084:	1887      	adds	r7, r0, r2
 8001086:	4297      	cmp	r7, r2
 8001088:	419b      	sbcs	r3, r3
 800108a:	4441      	add	r1, r8
 800108c:	425b      	negs	r3, r3
 800108e:	18c9      	adds	r1, r1, r3
 8001090:	0035      	movs	r5, r6
 8001092:	e5a3      	b.n	8000bdc <__aeabi_dadd+0x164>
 8001094:	003b      	movs	r3, r7
 8001096:	4333      	orrs	r3, r6
 8001098:	d0ce      	beq.n	8001038 <__aeabi_dadd+0x5c0>
 800109a:	2207      	movs	r2, #7
 800109c:	0031      	movs	r1, r6
 800109e:	403a      	ands	r2, r7
 80010a0:	e652      	b.n	8000d48 <__aeabi_dadd+0x2d0>
 80010a2:	2300      	movs	r3, #0
 80010a4:	001a      	movs	r2, r3
 80010a6:	e5f4      	b.n	8000c92 <__aeabi_dadd+0x21a>
 80010a8:	000007ff 	.word	0x000007ff
 80010ac:	ff7fffff 	.word	0xff7fffff

080010b0 <__aeabi_ddiv>:
 80010b0:	b5f0      	push	{r4, r5, r6, r7, lr}
 80010b2:	4657      	mov	r7, sl
 80010b4:	46de      	mov	lr, fp
 80010b6:	464e      	mov	r6, r9
 80010b8:	4645      	mov	r5, r8
 80010ba:	b5e0      	push	{r5, r6, r7, lr}
 80010bc:	4683      	mov	fp, r0
 80010be:	0007      	movs	r7, r0
 80010c0:	030e      	lsls	r6, r1, #12
 80010c2:	0048      	lsls	r0, r1, #1
 80010c4:	b085      	sub	sp, #20
 80010c6:	4692      	mov	sl, r2
 80010c8:	001c      	movs	r4, r3
 80010ca:	0b36      	lsrs	r6, r6, #12
 80010cc:	0d40      	lsrs	r0, r0, #21
 80010ce:	0fcd      	lsrs	r5, r1, #31
 80010d0:	2800      	cmp	r0, #0
 80010d2:	d100      	bne.n	80010d6 <__aeabi_ddiv+0x26>
 80010d4:	e09d      	b.n	8001212 <__aeabi_ddiv+0x162>
 80010d6:	4b95      	ldr	r3, [pc, #596]	; (800132c <__aeabi_ddiv+0x27c>)
 80010d8:	4298      	cmp	r0, r3
 80010da:	d039      	beq.n	8001150 <__aeabi_ddiv+0xa0>
 80010dc:	2380      	movs	r3, #128	; 0x80
 80010de:	00f6      	lsls	r6, r6, #3
 80010e0:	041b      	lsls	r3, r3, #16
 80010e2:	431e      	orrs	r6, r3
 80010e4:	4a92      	ldr	r2, [pc, #584]	; (8001330 <__aeabi_ddiv+0x280>)
 80010e6:	0f7b      	lsrs	r3, r7, #29
 80010e8:	4333      	orrs	r3, r6
 80010ea:	4699      	mov	r9, r3
 80010ec:	4694      	mov	ip, r2
 80010ee:	0003      	movs	r3, r0
 80010f0:	4463      	add	r3, ip
 80010f2:	9300      	str	r3, [sp, #0]
 80010f4:	2300      	movs	r3, #0
 80010f6:	2600      	movs	r6, #0
 80010f8:	00ff      	lsls	r7, r7, #3
 80010fa:	9302      	str	r3, [sp, #8]
 80010fc:	0323      	lsls	r3, r4, #12
 80010fe:	0b1b      	lsrs	r3, r3, #12
 8001100:	4698      	mov	r8, r3
 8001102:	0063      	lsls	r3, r4, #1
 8001104:	0fe4      	lsrs	r4, r4, #31
 8001106:	4652      	mov	r2, sl
 8001108:	0d5b      	lsrs	r3, r3, #21
 800110a:	9401      	str	r4, [sp, #4]
 800110c:	d100      	bne.n	8001110 <__aeabi_ddiv+0x60>
 800110e:	e0b3      	b.n	8001278 <__aeabi_ddiv+0x1c8>
 8001110:	4986      	ldr	r1, [pc, #536]	; (800132c <__aeabi_ddiv+0x27c>)
 8001112:	428b      	cmp	r3, r1
 8001114:	d100      	bne.n	8001118 <__aeabi_ddiv+0x68>
 8001116:	e09e      	b.n	8001256 <__aeabi_ddiv+0x1a6>
 8001118:	4642      	mov	r2, r8
 800111a:	00d1      	lsls	r1, r2, #3
 800111c:	2280      	movs	r2, #128	; 0x80
 800111e:	0412      	lsls	r2, r2, #16
 8001120:	430a      	orrs	r2, r1
 8001122:	4651      	mov	r1, sl
 8001124:	0f49      	lsrs	r1, r1, #29
 8001126:	4311      	orrs	r1, r2
 8001128:	468b      	mov	fp, r1
 800112a:	4981      	ldr	r1, [pc, #516]	; (8001330 <__aeabi_ddiv+0x280>)
 800112c:	4652      	mov	r2, sl
 800112e:	468c      	mov	ip, r1
 8001130:	9900      	ldr	r1, [sp, #0]
 8001132:	4463      	add	r3, ip
 8001134:	1acb      	subs	r3, r1, r3
 8001136:	2100      	movs	r1, #0
 8001138:	00d2      	lsls	r2, r2, #3
 800113a:	9300      	str	r3, [sp, #0]
 800113c:	002b      	movs	r3, r5
 800113e:	4063      	eors	r3, r4
 8001140:	469a      	mov	sl, r3
 8001142:	2e0f      	cmp	r6, #15
 8001144:	d900      	bls.n	8001148 <__aeabi_ddiv+0x98>
 8001146:	e105      	b.n	8001354 <__aeabi_ddiv+0x2a4>
 8001148:	4b7a      	ldr	r3, [pc, #488]	; (8001334 <__aeabi_ddiv+0x284>)
 800114a:	00b6      	lsls	r6, r6, #2
 800114c:	599b      	ldr	r3, [r3, r6]
 800114e:	469f      	mov	pc, r3
 8001150:	465b      	mov	r3, fp
 8001152:	4333      	orrs	r3, r6
 8001154:	4699      	mov	r9, r3
 8001156:	d000      	beq.n	800115a <__aeabi_ddiv+0xaa>
 8001158:	e0b8      	b.n	80012cc <__aeabi_ddiv+0x21c>
 800115a:	2302      	movs	r3, #2
 800115c:	2608      	movs	r6, #8
 800115e:	2700      	movs	r7, #0
 8001160:	9000      	str	r0, [sp, #0]
 8001162:	9302      	str	r3, [sp, #8]
 8001164:	e7ca      	b.n	80010fc <__aeabi_ddiv+0x4c>
 8001166:	46cb      	mov	fp, r9
 8001168:	003a      	movs	r2, r7
 800116a:	9902      	ldr	r1, [sp, #8]
 800116c:	9501      	str	r5, [sp, #4]
 800116e:	9b01      	ldr	r3, [sp, #4]
 8001170:	469a      	mov	sl, r3
 8001172:	2902      	cmp	r1, #2
 8001174:	d027      	beq.n	80011c6 <__aeabi_ddiv+0x116>
 8001176:	2903      	cmp	r1, #3
 8001178:	d100      	bne.n	800117c <__aeabi_ddiv+0xcc>
 800117a:	e280      	b.n	800167e <__aeabi_ddiv+0x5ce>
 800117c:	2901      	cmp	r1, #1
 800117e:	d044      	beq.n	800120a <__aeabi_ddiv+0x15a>
 8001180:	496d      	ldr	r1, [pc, #436]	; (8001338 <__aeabi_ddiv+0x288>)
 8001182:	9b00      	ldr	r3, [sp, #0]
 8001184:	468c      	mov	ip, r1
 8001186:	4463      	add	r3, ip
 8001188:	001c      	movs	r4, r3
 800118a:	2c00      	cmp	r4, #0
 800118c:	dd38      	ble.n	8001200 <__aeabi_ddiv+0x150>
 800118e:	0753      	lsls	r3, r2, #29
 8001190:	d000      	beq.n	8001194 <__aeabi_ddiv+0xe4>
 8001192:	e213      	b.n	80015bc <__aeabi_ddiv+0x50c>
 8001194:	08d2      	lsrs	r2, r2, #3
 8001196:	465b      	mov	r3, fp
 8001198:	01db      	lsls	r3, r3, #7
 800119a:	d509      	bpl.n	80011b0 <__aeabi_ddiv+0x100>
 800119c:	4659      	mov	r1, fp
 800119e:	4b67      	ldr	r3, [pc, #412]	; (800133c <__aeabi_ddiv+0x28c>)
 80011a0:	4019      	ands	r1, r3
 80011a2:	468b      	mov	fp, r1
 80011a4:	2180      	movs	r1, #128	; 0x80
 80011a6:	00c9      	lsls	r1, r1, #3
 80011a8:	468c      	mov	ip, r1
 80011aa:	9b00      	ldr	r3, [sp, #0]
 80011ac:	4463      	add	r3, ip
 80011ae:	001c      	movs	r4, r3
 80011b0:	4b63      	ldr	r3, [pc, #396]	; (8001340 <__aeabi_ddiv+0x290>)
 80011b2:	429c      	cmp	r4, r3
 80011b4:	dc07      	bgt.n	80011c6 <__aeabi_ddiv+0x116>
 80011b6:	465b      	mov	r3, fp
 80011b8:	0564      	lsls	r4, r4, #21
 80011ba:	075f      	lsls	r7, r3, #29
 80011bc:	025b      	lsls	r3, r3, #9
 80011be:	4317      	orrs	r7, r2
 80011c0:	0b1b      	lsrs	r3, r3, #12
 80011c2:	0d62      	lsrs	r2, r4, #21
 80011c4:	e002      	b.n	80011cc <__aeabi_ddiv+0x11c>
 80011c6:	2300      	movs	r3, #0
 80011c8:	2700      	movs	r7, #0
 80011ca:	4a58      	ldr	r2, [pc, #352]	; (800132c <__aeabi_ddiv+0x27c>)
 80011cc:	2100      	movs	r1, #0
 80011ce:	031b      	lsls	r3, r3, #12
 80011d0:	0b1c      	lsrs	r4, r3, #12
 80011d2:	0d0b      	lsrs	r3, r1, #20
 80011d4:	051b      	lsls	r3, r3, #20
 80011d6:	4323      	orrs	r3, r4
 80011d8:	0514      	lsls	r4, r2, #20
 80011da:	4a5a      	ldr	r2, [pc, #360]	; (8001344 <__aeabi_ddiv+0x294>)
 80011dc:	0038      	movs	r0, r7
 80011de:	4013      	ands	r3, r2
 80011e0:	431c      	orrs	r4, r3
 80011e2:	4653      	mov	r3, sl
 80011e4:	0064      	lsls	r4, r4, #1
 80011e6:	07db      	lsls	r3, r3, #31
 80011e8:	0864      	lsrs	r4, r4, #1
 80011ea:	431c      	orrs	r4, r3
 80011ec:	0021      	movs	r1, r4
 80011ee:	b005      	add	sp, #20
 80011f0:	bc3c      	pop	{r2, r3, r4, r5}
 80011f2:	4690      	mov	r8, r2
 80011f4:	4699      	mov	r9, r3
 80011f6:	46a2      	mov	sl, r4
 80011f8:	46ab      	mov	fp, r5
 80011fa:	bdf0      	pop	{r4, r5, r6, r7, pc}
 80011fc:	2201      	movs	r2, #1
 80011fe:	4252      	negs	r2, r2
 8001200:	2301      	movs	r3, #1
 8001202:	1b1b      	subs	r3, r3, r4
 8001204:	2b38      	cmp	r3, #56	; 0x38
 8001206:	dc00      	bgt.n	800120a <__aeabi_ddiv+0x15a>
 8001208:	e1ad      	b.n	8001566 <__aeabi_ddiv+0x4b6>
 800120a:	2200      	movs	r2, #0
 800120c:	2300      	movs	r3, #0
 800120e:	2700      	movs	r7, #0
 8001210:	e7dc      	b.n	80011cc <__aeabi_ddiv+0x11c>
 8001212:	465b      	mov	r3, fp
 8001214:	4333      	orrs	r3, r6
 8001216:	4699      	mov	r9, r3
 8001218:	d05e      	beq.n	80012d8 <__aeabi_ddiv+0x228>
 800121a:	2e00      	cmp	r6, #0
 800121c:	d100      	bne.n	8001220 <__aeabi_ddiv+0x170>
 800121e:	e18a      	b.n	8001536 <__aeabi_ddiv+0x486>
 8001220:	0030      	movs	r0, r6
 8001222:	f001 f9fd 	bl	8002620 <__clzsi2>
 8001226:	0003      	movs	r3, r0
 8001228:	3b0b      	subs	r3, #11
 800122a:	2b1c      	cmp	r3, #28
 800122c:	dd00      	ble.n	8001230 <__aeabi_ddiv+0x180>
 800122e:	e17b      	b.n	8001528 <__aeabi_ddiv+0x478>
 8001230:	221d      	movs	r2, #29
 8001232:	1ad3      	subs	r3, r2, r3
 8001234:	465a      	mov	r2, fp
 8001236:	0001      	movs	r1, r0
 8001238:	40da      	lsrs	r2, r3
 800123a:	3908      	subs	r1, #8
 800123c:	408e      	lsls	r6, r1
 800123e:	0013      	movs	r3, r2
 8001240:	465f      	mov	r7, fp
 8001242:	4333      	orrs	r3, r6
 8001244:	4699      	mov	r9, r3
 8001246:	408f      	lsls	r7, r1
 8001248:	4b3f      	ldr	r3, [pc, #252]	; (8001348 <__aeabi_ddiv+0x298>)
 800124a:	2600      	movs	r6, #0
 800124c:	1a1b      	subs	r3, r3, r0
 800124e:	9300      	str	r3, [sp, #0]
 8001250:	2300      	movs	r3, #0
 8001252:	9302      	str	r3, [sp, #8]
 8001254:	e752      	b.n	80010fc <__aeabi_ddiv+0x4c>
 8001256:	4641      	mov	r1, r8
 8001258:	4653      	mov	r3, sl
 800125a:	430b      	orrs	r3, r1
 800125c:	493b      	ldr	r1, [pc, #236]	; (800134c <__aeabi_ddiv+0x29c>)
 800125e:	469b      	mov	fp, r3
 8001260:	468c      	mov	ip, r1
 8001262:	9b00      	ldr	r3, [sp, #0]
 8001264:	4463      	add	r3, ip
 8001266:	9300      	str	r3, [sp, #0]
 8001268:	465b      	mov	r3, fp
 800126a:	2b00      	cmp	r3, #0
 800126c:	d13b      	bne.n	80012e6 <__aeabi_ddiv+0x236>
 800126e:	2302      	movs	r3, #2
 8001270:	2200      	movs	r2, #0
 8001272:	431e      	orrs	r6, r3
 8001274:	2102      	movs	r1, #2
 8001276:	e761      	b.n	800113c <__aeabi_ddiv+0x8c>
 8001278:	4643      	mov	r3, r8
 800127a:	4313      	orrs	r3, r2
 800127c:	469b      	mov	fp, r3
 800127e:	d037      	beq.n	80012f0 <__aeabi_ddiv+0x240>
 8001280:	4643      	mov	r3, r8
 8001282:	2b00      	cmp	r3, #0
 8001284:	d100      	bne.n	8001288 <__aeabi_ddiv+0x1d8>
 8001286:	e162      	b.n	800154e <__aeabi_ddiv+0x49e>
 8001288:	4640      	mov	r0, r8
 800128a:	f001 f9c9 	bl	8002620 <__clzsi2>
 800128e:	0003      	movs	r3, r0
 8001290:	3b0b      	subs	r3, #11
 8001292:	2b1c      	cmp	r3, #28
 8001294:	dd00      	ble.n	8001298 <__aeabi_ddiv+0x1e8>
 8001296:	e153      	b.n	8001540 <__aeabi_ddiv+0x490>
 8001298:	0002      	movs	r2, r0
 800129a:	4641      	mov	r1, r8
 800129c:	3a08      	subs	r2, #8
 800129e:	4091      	lsls	r1, r2
 80012a0:	4688      	mov	r8, r1
 80012a2:	211d      	movs	r1, #29
 80012a4:	1acb      	subs	r3, r1, r3
 80012a6:	4651      	mov	r1, sl
 80012a8:	40d9      	lsrs	r1, r3
 80012aa:	000b      	movs	r3, r1
 80012ac:	4641      	mov	r1, r8
 80012ae:	430b      	orrs	r3, r1
 80012b0:	469b      	mov	fp, r3
 80012b2:	4653      	mov	r3, sl
 80012b4:	4093      	lsls	r3, r2
 80012b6:	001a      	movs	r2, r3
 80012b8:	9b00      	ldr	r3, [sp, #0]
 80012ba:	4925      	ldr	r1, [pc, #148]	; (8001350 <__aeabi_ddiv+0x2a0>)
 80012bc:	469c      	mov	ip, r3
 80012be:	4460      	add	r0, ip
 80012c0:	0003      	movs	r3, r0
 80012c2:	468c      	mov	ip, r1
 80012c4:	4463      	add	r3, ip
 80012c6:	9300      	str	r3, [sp, #0]
 80012c8:	2100      	movs	r1, #0
 80012ca:	e737      	b.n	800113c <__aeabi_ddiv+0x8c>
 80012cc:	2303      	movs	r3, #3
 80012ce:	46b1      	mov	r9, r6
 80012d0:	9000      	str	r0, [sp, #0]
 80012d2:	260c      	movs	r6, #12
 80012d4:	9302      	str	r3, [sp, #8]
 80012d6:	e711      	b.n	80010fc <__aeabi_ddiv+0x4c>
 80012d8:	2300      	movs	r3, #0
 80012da:	9300      	str	r3, [sp, #0]
 80012dc:	3301      	adds	r3, #1
 80012de:	2604      	movs	r6, #4
 80012e0:	2700      	movs	r7, #0
 80012e2:	9302      	str	r3, [sp, #8]
 80012e4:	e70a      	b.n	80010fc <__aeabi_ddiv+0x4c>
 80012e6:	2303      	movs	r3, #3
 80012e8:	46c3      	mov	fp, r8
 80012ea:	431e      	orrs	r6, r3
 80012ec:	2103      	movs	r1, #3
 80012ee:	e725      	b.n	800113c <__aeabi_ddiv+0x8c>
 80012f0:	3301      	adds	r3, #1
 80012f2:	431e      	orrs	r6, r3
 80012f4:	2200      	movs	r2, #0
 80012f6:	2101      	movs	r1, #1
 80012f8:	e720      	b.n	800113c <__aeabi_ddiv+0x8c>
 80012fa:	2300      	movs	r3, #0
 80012fc:	469a      	mov	sl, r3
 80012fe:	2380      	movs	r3, #128	; 0x80
 8001300:	2700      	movs	r7, #0
 8001302:	031b      	lsls	r3, r3, #12
 8001304:	4a09      	ldr	r2, [pc, #36]	; (800132c <__aeabi_ddiv+0x27c>)
 8001306:	e761      	b.n	80011cc <__aeabi_ddiv+0x11c>
 8001308:	2380      	movs	r3, #128	; 0x80
 800130a:	4649      	mov	r1, r9
 800130c:	031b      	lsls	r3, r3, #12
 800130e:	4219      	tst	r1, r3
 8001310:	d100      	bne.n	8001314 <__aeabi_ddiv+0x264>
 8001312:	e0e2      	b.n	80014da <__aeabi_ddiv+0x42a>
 8001314:	4659      	mov	r1, fp
 8001316:	4219      	tst	r1, r3
 8001318:	d000      	beq.n	800131c <__aeabi_ddiv+0x26c>
 800131a:	e0de      	b.n	80014da <__aeabi_ddiv+0x42a>
 800131c:	430b      	orrs	r3, r1
 800131e:	031b      	lsls	r3, r3, #12
 8001320:	0017      	movs	r7, r2
 8001322:	0b1b      	lsrs	r3, r3, #12
 8001324:	46a2      	mov	sl, r4
 8001326:	4a01      	ldr	r2, [pc, #4]	; (800132c <__aeabi_ddiv+0x27c>)
 8001328:	e750      	b.n	80011cc <__aeabi_ddiv+0x11c>
 800132a:	46c0      	nop			; (mov r8, r8)
 800132c:	000007ff 	.word	0x000007ff
 8001330:	fffffc01 	.word	0xfffffc01
 8001334:	0801a8f0 	.word	0x0801a8f0
 8001338:	000003ff 	.word	0x000003ff
 800133c:	feffffff 	.word	0xfeffffff
 8001340:	000007fe 	.word	0x000007fe
 8001344:	800fffff 	.word	0x800fffff
 8001348:	fffffc0d 	.word	0xfffffc0d
 800134c:	fffff801 	.word	0xfffff801
 8001350:	000003f3 	.word	0x000003f3
 8001354:	45d9      	cmp	r9, fp
 8001356:	d900      	bls.n	800135a <__aeabi_ddiv+0x2aa>
 8001358:	e0cb      	b.n	80014f2 <__aeabi_ddiv+0x442>
 800135a:	d100      	bne.n	800135e <__aeabi_ddiv+0x2ae>
 800135c:	e0c6      	b.n	80014ec <__aeabi_ddiv+0x43c>
 800135e:	003c      	movs	r4, r7
 8001360:	4648      	mov	r0, r9
 8001362:	2700      	movs	r7, #0
 8001364:	9b00      	ldr	r3, [sp, #0]
 8001366:	3b01      	subs	r3, #1
 8001368:	9300      	str	r3, [sp, #0]
 800136a:	465b      	mov	r3, fp
 800136c:	0e16      	lsrs	r6, r2, #24
 800136e:	021b      	lsls	r3, r3, #8
 8001370:	431e      	orrs	r6, r3
 8001372:	0213      	lsls	r3, r2, #8
 8001374:	4698      	mov	r8, r3
 8001376:	0433      	lsls	r3, r6, #16
 8001378:	0c1b      	lsrs	r3, r3, #16
 800137a:	4699      	mov	r9, r3
 800137c:	0c31      	lsrs	r1, r6, #16
 800137e:	9101      	str	r1, [sp, #4]
 8001380:	f7fe ff48 	bl	8000214 <__aeabi_uidivmod>
 8001384:	464a      	mov	r2, r9
 8001386:	4342      	muls	r2, r0
 8001388:	040b      	lsls	r3, r1, #16
 800138a:	0c21      	lsrs	r1, r4, #16
 800138c:	0005      	movs	r5, r0
 800138e:	4319      	orrs	r1, r3
 8001390:	428a      	cmp	r2, r1
 8001392:	d907      	bls.n	80013a4 <__aeabi_ddiv+0x2f4>
 8001394:	1989      	adds	r1, r1, r6
 8001396:	3d01      	subs	r5, #1
 8001398:	428e      	cmp	r6, r1
 800139a:	d803      	bhi.n	80013a4 <__aeabi_ddiv+0x2f4>
 800139c:	428a      	cmp	r2, r1
 800139e:	d901      	bls.n	80013a4 <__aeabi_ddiv+0x2f4>
 80013a0:	1e85      	subs	r5, r0, #2
 80013a2:	1989      	adds	r1, r1, r6
 80013a4:	1a88      	subs	r0, r1, r2
 80013a6:	9901      	ldr	r1, [sp, #4]
 80013a8:	f7fe ff34 	bl	8000214 <__aeabi_uidivmod>
 80013ac:	0409      	lsls	r1, r1, #16
 80013ae:	468c      	mov	ip, r1
 80013b0:	464a      	mov	r2, r9
 80013b2:	0421      	lsls	r1, r4, #16
 80013b4:	4664      	mov	r4, ip
 80013b6:	4342      	muls	r2, r0
 80013b8:	0c09      	lsrs	r1, r1, #16
 80013ba:	0003      	movs	r3, r0
 80013bc:	4321      	orrs	r1, r4
 80013be:	428a      	cmp	r2, r1
 80013c0:	d904      	bls.n	80013cc <__aeabi_ddiv+0x31c>
 80013c2:	1989      	adds	r1, r1, r6
 80013c4:	3b01      	subs	r3, #1
 80013c6:	428e      	cmp	r6, r1
 80013c8:	d800      	bhi.n	80013cc <__aeabi_ddiv+0x31c>
 80013ca:	e0f1      	b.n	80015b0 <__aeabi_ddiv+0x500>
 80013cc:	042d      	lsls	r5, r5, #16
 80013ce:	431d      	orrs	r5, r3
 80013d0:	46ab      	mov	fp, r5
 80013d2:	4643      	mov	r3, r8
 80013d4:	1a89      	subs	r1, r1, r2
 80013d6:	4642      	mov	r2, r8
 80013d8:	0c28      	lsrs	r0, r5, #16
 80013da:	0412      	lsls	r2, r2, #16
 80013dc:	0c1d      	lsrs	r5, r3, #16
 80013de:	465b      	mov	r3, fp
 80013e0:	0c14      	lsrs	r4, r2, #16
 80013e2:	0022      	movs	r2, r4
 80013e4:	041b      	lsls	r3, r3, #16
 80013e6:	0c1b      	lsrs	r3, r3, #16
 80013e8:	435a      	muls	r2, r3
 80013ea:	9403      	str	r4, [sp, #12]
 80013ec:	436b      	muls	r3, r5
 80013ee:	4344      	muls	r4, r0
 80013f0:	9502      	str	r5, [sp, #8]
 80013f2:	4368      	muls	r0, r5
 80013f4:	191b      	adds	r3, r3, r4
 80013f6:	0c15      	lsrs	r5, r2, #16
 80013f8:	18eb      	adds	r3, r5, r3
 80013fa:	429c      	cmp	r4, r3
 80013fc:	d903      	bls.n	8001406 <__aeabi_ddiv+0x356>
 80013fe:	2480      	movs	r4, #128	; 0x80
 8001400:	0264      	lsls	r4, r4, #9
 8001402:	46a4      	mov	ip, r4
 8001404:	4460      	add	r0, ip
 8001406:	0c1c      	lsrs	r4, r3, #16
 8001408:	0415      	lsls	r5, r2, #16
 800140a:	041b      	lsls	r3, r3, #16
 800140c:	0c2d      	lsrs	r5, r5, #16
 800140e:	1820      	adds	r0, r4, r0
 8001410:	195d      	adds	r5, r3, r5
 8001412:	4281      	cmp	r1, r0
 8001414:	d377      	bcc.n	8001506 <__aeabi_ddiv+0x456>
 8001416:	d073      	beq.n	8001500 <__aeabi_ddiv+0x450>
 8001418:	1a0c      	subs	r4, r1, r0
 800141a:	4aa2      	ldr	r2, [pc, #648]	; (80016a4 <__aeabi_ddiv+0x5f4>)
 800141c:	1b7d      	subs	r5, r7, r5
 800141e:	42af      	cmp	r7, r5
 8001420:	41bf      	sbcs	r7, r7
 8001422:	4694      	mov	ip, r2
 8001424:	9b00      	ldr	r3, [sp, #0]
 8001426:	427f      	negs	r7, r7
 8001428:	4463      	add	r3, ip
 800142a:	1be0      	subs	r0, r4, r7
 800142c:	001c      	movs	r4, r3
 800142e:	4286      	cmp	r6, r0
 8001430:	d100      	bne.n	8001434 <__aeabi_ddiv+0x384>
 8001432:	e0db      	b.n	80015ec <__aeabi_ddiv+0x53c>
 8001434:	9901      	ldr	r1, [sp, #4]
 8001436:	f7fe feed 	bl	8000214 <__aeabi_uidivmod>
 800143a:	464a      	mov	r2, r9
 800143c:	4342      	muls	r2, r0
 800143e:	040b      	lsls	r3, r1, #16
 8001440:	0c29      	lsrs	r1, r5, #16
 8001442:	0007      	movs	r7, r0
 8001444:	4319      	orrs	r1, r3
 8001446:	428a      	cmp	r2, r1
 8001448:	d907      	bls.n	800145a <__aeabi_ddiv+0x3aa>
 800144a:	1989      	adds	r1, r1, r6
 800144c:	3f01      	subs	r7, #1
 800144e:	428e      	cmp	r6, r1
 8001450:	d803      	bhi.n	800145a <__aeabi_ddiv+0x3aa>
 8001452:	428a      	cmp	r2, r1
 8001454:	d901      	bls.n	800145a <__aeabi_ddiv+0x3aa>
 8001456:	1e87      	subs	r7, r0, #2
 8001458:	1989      	adds	r1, r1, r6
 800145a:	1a88      	subs	r0, r1, r2
 800145c:	9901      	ldr	r1, [sp, #4]
 800145e:	f7fe fed9 	bl	8000214 <__aeabi_uidivmod>
 8001462:	0409      	lsls	r1, r1, #16
 8001464:	464a      	mov	r2, r9
 8001466:	4689      	mov	r9, r1
 8001468:	0429      	lsls	r1, r5, #16
 800146a:	464d      	mov	r5, r9
 800146c:	4342      	muls	r2, r0
 800146e:	0c09      	lsrs	r1, r1, #16
 8001470:	0003      	movs	r3, r0
 8001472:	4329      	orrs	r1, r5
 8001474:	428a      	cmp	r2, r1
 8001476:	d907      	bls.n	8001488 <__aeabi_ddiv+0x3d8>
 8001478:	1989      	adds	r1, r1, r6
 800147a:	3b01      	subs	r3, #1
 800147c:	428e      	cmp	r6, r1
 800147e:	d803      	bhi.n	8001488 <__aeabi_ddiv+0x3d8>
 8001480:	428a      	cmp	r2, r1
 8001482:	d901      	bls.n	8001488 <__aeabi_ddiv+0x3d8>
 8001484:	1e83      	subs	r3, r0, #2
 8001486:	1989      	adds	r1, r1, r6
 8001488:	043f      	lsls	r7, r7, #16
 800148a:	1a89      	subs	r1, r1, r2
 800148c:	003a      	movs	r2, r7
 800148e:	9f03      	ldr	r7, [sp, #12]
 8001490:	431a      	orrs	r2, r3
 8001492:	0038      	movs	r0, r7
 8001494:	0413      	lsls	r3, r2, #16
 8001496:	0c1b      	lsrs	r3, r3, #16
 8001498:	4358      	muls	r0, r3
 800149a:	4681      	mov	r9, r0
 800149c:	9802      	ldr	r0, [sp, #8]
 800149e:	0c15      	lsrs	r5, r2, #16
 80014a0:	436f      	muls	r7, r5
 80014a2:	4343      	muls	r3, r0
 80014a4:	4345      	muls	r5, r0
 80014a6:	4648      	mov	r0, r9
 80014a8:	0c00      	lsrs	r0, r0, #16
 80014aa:	4684      	mov	ip, r0
 80014ac:	19db      	adds	r3, r3, r7
 80014ae:	4463      	add	r3, ip
 80014b0:	429f      	cmp	r7, r3
 80014b2:	d903      	bls.n	80014bc <__aeabi_ddiv+0x40c>
 80014b4:	2080      	movs	r0, #128	; 0x80
 80014b6:	0240      	lsls	r0, r0, #9
 80014b8:	4684      	mov	ip, r0
 80014ba:	4465      	add	r5, ip
 80014bc:	4648      	mov	r0, r9
 80014be:	0c1f      	lsrs	r7, r3, #16
 80014c0:	0400      	lsls	r0, r0, #16
 80014c2:	041b      	lsls	r3, r3, #16
 80014c4:	0c00      	lsrs	r0, r0, #16
 80014c6:	197d      	adds	r5, r7, r5
 80014c8:	1818      	adds	r0, r3, r0
 80014ca:	42a9      	cmp	r1, r5
 80014cc:	d200      	bcs.n	80014d0 <__aeabi_ddiv+0x420>
 80014ce:	e084      	b.n	80015da <__aeabi_ddiv+0x52a>
 80014d0:	d100      	bne.n	80014d4 <__aeabi_ddiv+0x424>
 80014d2:	e07f      	b.n	80015d4 <__aeabi_ddiv+0x524>
 80014d4:	2301      	movs	r3, #1
 80014d6:	431a      	orrs	r2, r3
 80014d8:	e657      	b.n	800118a <__aeabi_ddiv+0xda>
 80014da:	2380      	movs	r3, #128	; 0x80
 80014dc:	464a      	mov	r2, r9
 80014de:	031b      	lsls	r3, r3, #12
 80014e0:	4313      	orrs	r3, r2
 80014e2:	031b      	lsls	r3, r3, #12
 80014e4:	0b1b      	lsrs	r3, r3, #12
 80014e6:	46aa      	mov	sl, r5
 80014e8:	4a6f      	ldr	r2, [pc, #444]	; (80016a8 <__aeabi_ddiv+0x5f8>)
 80014ea:	e66f      	b.n	80011cc <__aeabi_ddiv+0x11c>
 80014ec:	42ba      	cmp	r2, r7
 80014ee:	d900      	bls.n	80014f2 <__aeabi_ddiv+0x442>
 80014f0:	e735      	b.n	800135e <__aeabi_ddiv+0x2ae>
 80014f2:	464b      	mov	r3, r9
 80014f4:	07dc      	lsls	r4, r3, #31
 80014f6:	0858      	lsrs	r0, r3, #1
 80014f8:	087b      	lsrs	r3, r7, #1
 80014fa:	431c      	orrs	r4, r3
 80014fc:	07ff      	lsls	r7, r7, #31
 80014fe:	e734      	b.n	800136a <__aeabi_ddiv+0x2ba>
 8001500:	2400      	movs	r4, #0
 8001502:	42af      	cmp	r7, r5
 8001504:	d289      	bcs.n	800141a <__aeabi_ddiv+0x36a>
 8001506:	4447      	add	r7, r8
 8001508:	4547      	cmp	r7, r8
 800150a:	41a4      	sbcs	r4, r4
 800150c:	465b      	mov	r3, fp
 800150e:	4264      	negs	r4, r4
 8001510:	19a4      	adds	r4, r4, r6
 8001512:	1864      	adds	r4, r4, r1
 8001514:	3b01      	subs	r3, #1
 8001516:	42a6      	cmp	r6, r4
 8001518:	d21e      	bcs.n	8001558 <__aeabi_ddiv+0x4a8>
 800151a:	42a0      	cmp	r0, r4
 800151c:	d86d      	bhi.n	80015fa <__aeabi_ddiv+0x54a>
 800151e:	d100      	bne.n	8001522 <__aeabi_ddiv+0x472>
 8001520:	e0b6      	b.n	8001690 <__aeabi_ddiv+0x5e0>
 8001522:	1a24      	subs	r4, r4, r0
 8001524:	469b      	mov	fp, r3
 8001526:	e778      	b.n	800141a <__aeabi_ddiv+0x36a>
 8001528:	0003      	movs	r3, r0
 800152a:	465a      	mov	r2, fp
 800152c:	3b28      	subs	r3, #40	; 0x28
 800152e:	409a      	lsls	r2, r3
 8001530:	2700      	movs	r7, #0
 8001532:	4691      	mov	r9, r2
 8001534:	e688      	b.n	8001248 <__aeabi_ddiv+0x198>
 8001536:	4658      	mov	r0, fp
 8001538:	f001 f872 	bl	8002620 <__clzsi2>
 800153c:	3020      	adds	r0, #32
 800153e:	e672      	b.n	8001226 <__aeabi_ddiv+0x176>
 8001540:	0003      	movs	r3, r0
 8001542:	4652      	mov	r2, sl
 8001544:	3b28      	subs	r3, #40	; 0x28
 8001546:	409a      	lsls	r2, r3
 8001548:	4693      	mov	fp, r2
 800154a:	2200      	movs	r2, #0
 800154c:	e6b4      	b.n	80012b8 <__aeabi_ddiv+0x208>
 800154e:	4650      	mov	r0, sl
 8001550:	f001 f866 	bl	8002620 <__clzsi2>
 8001554:	3020      	adds	r0, #32
 8001556:	e69a      	b.n	800128e <__aeabi_ddiv+0x1de>
 8001558:	42a6      	cmp	r6, r4
 800155a:	d1e2      	bne.n	8001522 <__aeabi_ddiv+0x472>
 800155c:	45b8      	cmp	r8, r7
 800155e:	d9dc      	bls.n	800151a <__aeabi_ddiv+0x46a>
 8001560:	1a34      	subs	r4, r6, r0
 8001562:	469b      	mov	fp, r3
 8001564:	e759      	b.n	800141a <__aeabi_ddiv+0x36a>
 8001566:	2b1f      	cmp	r3, #31
 8001568:	dc65      	bgt.n	8001636 <__aeabi_ddiv+0x586>
 800156a:	4c50      	ldr	r4, [pc, #320]	; (80016ac <__aeabi_ddiv+0x5fc>)
 800156c:	9900      	ldr	r1, [sp, #0]
 800156e:	46a4      	mov	ip, r4
 8001570:	465c      	mov	r4, fp
 8001572:	4461      	add	r1, ip
 8001574:	0008      	movs	r0, r1
 8001576:	408c      	lsls	r4, r1
 8001578:	0011      	movs	r1, r2
 800157a:	4082      	lsls	r2, r0
 800157c:	40d9      	lsrs	r1, r3
 800157e:	1e50      	subs	r0, r2, #1
 8001580:	4182      	sbcs	r2, r0
 8001582:	430c      	orrs	r4, r1
 8001584:	4314      	orrs	r4, r2
 8001586:	465a      	mov	r2, fp
 8001588:	40da      	lsrs	r2, r3
 800158a:	0013      	movs	r3, r2
 800158c:	0762      	lsls	r2, r4, #29
 800158e:	d009      	beq.n	80015a4 <__aeabi_ddiv+0x4f4>
 8001590:	220f      	movs	r2, #15
 8001592:	4022      	ands	r2, r4
 8001594:	2a04      	cmp	r2, #4
 8001596:	d005      	beq.n	80015a4 <__aeabi_ddiv+0x4f4>
 8001598:	0022      	movs	r2, r4
 800159a:	1d14      	adds	r4, r2, #4
 800159c:	4294      	cmp	r4, r2
 800159e:	4189      	sbcs	r1, r1
 80015a0:	4249      	negs	r1, r1
 80015a2:	185b      	adds	r3, r3, r1
 80015a4:	021a      	lsls	r2, r3, #8
 80015a6:	d562      	bpl.n	800166e <__aeabi_ddiv+0x5be>
 80015a8:	2201      	movs	r2, #1
 80015aa:	2300      	movs	r3, #0
 80015ac:	2700      	movs	r7, #0
 80015ae:	e60d      	b.n	80011cc <__aeabi_ddiv+0x11c>
 80015b0:	428a      	cmp	r2, r1
 80015b2:	d800      	bhi.n	80015b6 <__aeabi_ddiv+0x506>
 80015b4:	e70a      	b.n	80013cc <__aeabi_ddiv+0x31c>
 80015b6:	1e83      	subs	r3, r0, #2
 80015b8:	1989      	adds	r1, r1, r6
 80015ba:	e707      	b.n	80013cc <__aeabi_ddiv+0x31c>
 80015bc:	230f      	movs	r3, #15
 80015be:	4013      	ands	r3, r2
 80015c0:	2b04      	cmp	r3, #4
 80015c2:	d100      	bne.n	80015c6 <__aeabi_ddiv+0x516>
 80015c4:	e5e6      	b.n	8001194 <__aeabi_ddiv+0xe4>
 80015c6:	1d17      	adds	r7, r2, #4
 80015c8:	4297      	cmp	r7, r2
 80015ca:	4192      	sbcs	r2, r2
 80015cc:	4253      	negs	r3, r2
 80015ce:	449b      	add	fp, r3
 80015d0:	08fa      	lsrs	r2, r7, #3
 80015d2:	e5e0      	b.n	8001196 <__aeabi_ddiv+0xe6>
 80015d4:	2800      	cmp	r0, #0
 80015d6:	d100      	bne.n	80015da <__aeabi_ddiv+0x52a>
 80015d8:	e5d7      	b.n	800118a <__aeabi_ddiv+0xda>
 80015da:	1871      	adds	r1, r6, r1
 80015dc:	1e53      	subs	r3, r2, #1
 80015de:	42b1      	cmp	r1, r6
 80015e0:	d327      	bcc.n	8001632 <__aeabi_ddiv+0x582>
 80015e2:	42a9      	cmp	r1, r5
 80015e4:	d315      	bcc.n	8001612 <__aeabi_ddiv+0x562>
 80015e6:	d058      	beq.n	800169a <__aeabi_ddiv+0x5ea>
 80015e8:	001a      	movs	r2, r3
 80015ea:	e773      	b.n	80014d4 <__aeabi_ddiv+0x424>
 80015ec:	2b00      	cmp	r3, #0
 80015ee:	dc00      	bgt.n	80015f2 <__aeabi_ddiv+0x542>
 80015f0:	e604      	b.n	80011fc <__aeabi_ddiv+0x14c>
 80015f2:	2301      	movs	r3, #1
 80015f4:	2200      	movs	r2, #0
 80015f6:	449b      	add	fp, r3
 80015f8:	e5cd      	b.n	8001196 <__aeabi_ddiv+0xe6>
 80015fa:	2302      	movs	r3, #2
 80015fc:	4447      	add	r7, r8
 80015fe:	4547      	cmp	r7, r8
 8001600:	4189      	sbcs	r1, r1
 8001602:	425b      	negs	r3, r3
 8001604:	469c      	mov	ip, r3
 8001606:	4249      	negs	r1, r1
 8001608:	1989      	adds	r1, r1, r6
 800160a:	190c      	adds	r4, r1, r4
 800160c:	44e3      	add	fp, ip
 800160e:	1a24      	subs	r4, r4, r0
 8001610:	e703      	b.n	800141a <__aeabi_ddiv+0x36a>
 8001612:	4643      	mov	r3, r8
 8001614:	005f      	lsls	r7, r3, #1
 8001616:	4547      	cmp	r7, r8
 8001618:	419b      	sbcs	r3, r3
 800161a:	46b8      	mov	r8, r7
 800161c:	425b      	negs	r3, r3
 800161e:	199e      	adds	r6, r3, r6
 8001620:	3a02      	subs	r2, #2
 8001622:	1989      	adds	r1, r1, r6
 8001624:	42a9      	cmp	r1, r5
 8001626:	d000      	beq.n	800162a <__aeabi_ddiv+0x57a>
 8001628:	e754      	b.n	80014d4 <__aeabi_ddiv+0x424>
 800162a:	4540      	cmp	r0, r8
 800162c:	d000      	beq.n	8001630 <__aeabi_ddiv+0x580>
 800162e:	e751      	b.n	80014d4 <__aeabi_ddiv+0x424>
 8001630:	e5ab      	b.n	800118a <__aeabi_ddiv+0xda>
 8001632:	001a      	movs	r2, r3
 8001634:	e7f6      	b.n	8001624 <__aeabi_ddiv+0x574>
 8001636:	211f      	movs	r1, #31
 8001638:	465f      	mov	r7, fp
 800163a:	4249      	negs	r1, r1
 800163c:	1b0c      	subs	r4, r1, r4
 800163e:	40e7      	lsrs	r7, r4
 8001640:	2b20      	cmp	r3, #32
 8001642:	d007      	beq.n	8001654 <__aeabi_ddiv+0x5a4>
 8001644:	491a      	ldr	r1, [pc, #104]	; (80016b0 <__aeabi_ddiv+0x600>)
 8001646:	9b00      	ldr	r3, [sp, #0]
 8001648:	468c      	mov	ip, r1
 800164a:	4463      	add	r3, ip
 800164c:	0018      	movs	r0, r3
 800164e:	465b      	mov	r3, fp
 8001650:	4083      	lsls	r3, r0
 8001652:	431a      	orrs	r2, r3
 8001654:	1e50      	subs	r0, r2, #1
 8001656:	4182      	sbcs	r2, r0
 8001658:	433a      	orrs	r2, r7
 800165a:	2707      	movs	r7, #7
 800165c:	2300      	movs	r3, #0
 800165e:	4017      	ands	r7, r2
 8001660:	d009      	beq.n	8001676 <__aeabi_ddiv+0x5c6>
 8001662:	210f      	movs	r1, #15
 8001664:	2300      	movs	r3, #0
 8001666:	4011      	ands	r1, r2
 8001668:	0014      	movs	r4, r2
 800166a:	2904      	cmp	r1, #4
 800166c:	d195      	bne.n	800159a <__aeabi_ddiv+0x4ea>
 800166e:	0022      	movs	r2, r4
 8001670:	075f      	lsls	r7, r3, #29
 8001672:	025b      	lsls	r3, r3, #9
 8001674:	0b1b      	lsrs	r3, r3, #12
 8001676:	08d2      	lsrs	r2, r2, #3
 8001678:	4317      	orrs	r7, r2
 800167a:	2200      	movs	r2, #0
 800167c:	e5a6      	b.n	80011cc <__aeabi_ddiv+0x11c>
 800167e:	2380      	movs	r3, #128	; 0x80
 8001680:	4659      	mov	r1, fp
 8001682:	031b      	lsls	r3, r3, #12
 8001684:	430b      	orrs	r3, r1
 8001686:	031b      	lsls	r3, r3, #12
 8001688:	0017      	movs	r7, r2
 800168a:	0b1b      	lsrs	r3, r3, #12
 800168c:	4a06      	ldr	r2, [pc, #24]	; (80016a8 <__aeabi_ddiv+0x5f8>)
 800168e:	e59d      	b.n	80011cc <__aeabi_ddiv+0x11c>
 8001690:	42bd      	cmp	r5, r7
 8001692:	d8b2      	bhi.n	80015fa <__aeabi_ddiv+0x54a>
 8001694:	469b      	mov	fp, r3
 8001696:	2400      	movs	r4, #0
 8001698:	e6bf      	b.n	800141a <__aeabi_ddiv+0x36a>
 800169a:	4580      	cmp	r8, r0
 800169c:	d3b9      	bcc.n	8001612 <__aeabi_ddiv+0x562>
 800169e:	001a      	movs	r2, r3
 80016a0:	e7c3      	b.n	800162a <__aeabi_ddiv+0x57a>
 80016a2:	46c0      	nop			; (mov r8, r8)
 80016a4:	000003ff 	.word	0x000003ff
 80016a8:	000007ff 	.word	0x000007ff
 80016ac:	0000041e 	.word	0x0000041e
 80016b0:	0000043e 	.word	0x0000043e

080016b4 <__eqdf2>:
 80016b4:	b5f0      	push	{r4, r5, r6, r7, lr}
 80016b6:	464f      	mov	r7, r9
 80016b8:	4646      	mov	r6, r8
 80016ba:	46d6      	mov	lr, sl
 80016bc:	4684      	mov	ip, r0
 80016be:	b5c0      	push	{r6, r7, lr}
 80016c0:	4680      	mov	r8, r0
 80016c2:	4e19      	ldr	r6, [pc, #100]	; (8001728 <__eqdf2+0x74>)
 80016c4:	0318      	lsls	r0, r3, #12
 80016c6:	030f      	lsls	r7, r1, #12
 80016c8:	004d      	lsls	r5, r1, #1
 80016ca:	0b00      	lsrs	r0, r0, #12
 80016cc:	005c      	lsls	r4, r3, #1
 80016ce:	4682      	mov	sl, r0
 80016d0:	0b3f      	lsrs	r7, r7, #12
 80016d2:	0d6d      	lsrs	r5, r5, #21
 80016d4:	0fc9      	lsrs	r1, r1, #31
 80016d6:	4691      	mov	r9, r2
 80016d8:	0d64      	lsrs	r4, r4, #21
 80016da:	0fdb      	lsrs	r3, r3, #31
 80016dc:	2001      	movs	r0, #1
 80016de:	42b5      	cmp	r5, r6
 80016e0:	d00a      	beq.n	80016f8 <__eqdf2+0x44>
 80016e2:	42b4      	cmp	r4, r6
 80016e4:	d003      	beq.n	80016ee <__eqdf2+0x3a>
 80016e6:	42a5      	cmp	r5, r4
 80016e8:	d101      	bne.n	80016ee <__eqdf2+0x3a>
 80016ea:	4557      	cmp	r7, sl
 80016ec:	d00c      	beq.n	8001708 <__eqdf2+0x54>
 80016ee:	bc1c      	pop	{r2, r3, r4}
 80016f0:	4690      	mov	r8, r2
 80016f2:	4699      	mov	r9, r3
 80016f4:	46a2      	mov	sl, r4
 80016f6:	bdf0      	pop	{r4, r5, r6, r7, pc}
 80016f8:	4666      	mov	r6, ip
 80016fa:	433e      	orrs	r6, r7
 80016fc:	d1f7      	bne.n	80016ee <__eqdf2+0x3a>
 80016fe:	42ac      	cmp	r4, r5
 8001700:	d1f5      	bne.n	80016ee <__eqdf2+0x3a>
 8001702:	4654      	mov	r4, sl
 8001704:	4314      	orrs	r4, r2
 8001706:	d1f2      	bne.n	80016ee <__eqdf2+0x3a>
 8001708:	2001      	movs	r0, #1
 800170a:	45c8      	cmp	r8, r9
 800170c:	d1ef      	bne.n	80016ee <__eqdf2+0x3a>
 800170e:	4299      	cmp	r1, r3
 8001710:	d007      	beq.n	8001722 <__eqdf2+0x6e>
 8001712:	2d00      	cmp	r5, #0
 8001714:	d1eb      	bne.n	80016ee <__eqdf2+0x3a>
 8001716:	4663      	mov	r3, ip
 8001718:	431f      	orrs	r7, r3
 800171a:	0038      	movs	r0, r7
 800171c:	1e47      	subs	r7, r0, #1
 800171e:	41b8      	sbcs	r0, r7
 8001720:	e7e5      	b.n	80016ee <__eqdf2+0x3a>
 8001722:	2000      	movs	r0, #0
 8001724:	e7e3      	b.n	80016ee <__eqdf2+0x3a>
 8001726:	46c0      	nop			; (mov r8, r8)
 8001728:	000007ff 	.word	0x000007ff

0800172c <__gedf2>:
 800172c:	b5f0      	push	{r4, r5, r6, r7, lr}
 800172e:	464f      	mov	r7, r9
 8001730:	4646      	mov	r6, r8
 8001732:	46d6      	mov	lr, sl
 8001734:	004d      	lsls	r5, r1, #1
 8001736:	b5c0      	push	{r6, r7, lr}
 8001738:	030e      	lsls	r6, r1, #12
 800173a:	0fc9      	lsrs	r1, r1, #31
 800173c:	468a      	mov	sl, r1
 800173e:	492c      	ldr	r1, [pc, #176]	; (80017f0 <__gedf2+0xc4>)
 8001740:	031f      	lsls	r7, r3, #12
 8001742:	005c      	lsls	r4, r3, #1
 8001744:	4680      	mov	r8, r0
 8001746:	0b36      	lsrs	r6, r6, #12
 8001748:	0d6d      	lsrs	r5, r5, #21
 800174a:	4691      	mov	r9, r2
 800174c:	0b3f      	lsrs	r7, r7, #12
 800174e:	0d64      	lsrs	r4, r4, #21
 8001750:	0fdb      	lsrs	r3, r3, #31
 8001752:	428d      	cmp	r5, r1
 8001754:	d01e      	beq.n	8001794 <__gedf2+0x68>
 8001756:	428c      	cmp	r4, r1
 8001758:	d016      	beq.n	8001788 <__gedf2+0x5c>
 800175a:	2d00      	cmp	r5, #0
 800175c:	d11e      	bne.n	800179c <__gedf2+0x70>
 800175e:	4330      	orrs	r0, r6
 8001760:	4684      	mov	ip, r0
 8001762:	2c00      	cmp	r4, #0
 8001764:	d101      	bne.n	800176a <__gedf2+0x3e>
 8001766:	433a      	orrs	r2, r7
 8001768:	d023      	beq.n	80017b2 <__gedf2+0x86>
 800176a:	4662      	mov	r2, ip
 800176c:	2a00      	cmp	r2, #0
 800176e:	d01a      	beq.n	80017a6 <__gedf2+0x7a>
 8001770:	459a      	cmp	sl, r3
 8001772:	d029      	beq.n	80017c8 <__gedf2+0x9c>
 8001774:	4651      	mov	r1, sl
 8001776:	2002      	movs	r0, #2
 8001778:	3901      	subs	r1, #1
 800177a:	4008      	ands	r0, r1
 800177c:	3801      	subs	r0, #1
 800177e:	bc1c      	pop	{r2, r3, r4}
 8001780:	4690      	mov	r8, r2
 8001782:	4699      	mov	r9, r3
 8001784:	46a2      	mov	sl, r4
 8001786:	bdf0      	pop	{r4, r5, r6, r7, pc}
 8001788:	0039      	movs	r1, r7
 800178a:	4311      	orrs	r1, r2
 800178c:	d0e5      	beq.n	800175a <__gedf2+0x2e>
 800178e:	2002      	movs	r0, #2
 8001790:	4240      	negs	r0, r0
 8001792:	e7f4      	b.n	800177e <__gedf2+0x52>
 8001794:	4330      	orrs	r0, r6
 8001796:	d1fa      	bne.n	800178e <__gedf2+0x62>
 8001798:	42ac      	cmp	r4, r5
 800179a:	d00f      	beq.n	80017bc <__gedf2+0x90>
 800179c:	2c00      	cmp	r4, #0
 800179e:	d10f      	bne.n	80017c0 <__gedf2+0x94>
 80017a0:	433a      	orrs	r2, r7
 80017a2:	d0e7      	beq.n	8001774 <__gedf2+0x48>
 80017a4:	e00c      	b.n	80017c0 <__gedf2+0x94>
 80017a6:	2201      	movs	r2, #1
 80017a8:	3b01      	subs	r3, #1
 80017aa:	4393      	bics	r3, r2
 80017ac:	0018      	movs	r0, r3
 80017ae:	3001      	adds	r0, #1
 80017b0:	e7e5      	b.n	800177e <__gedf2+0x52>
 80017b2:	4663      	mov	r3, ip
 80017b4:	2000      	movs	r0, #0
 80017b6:	2b00      	cmp	r3, #0
 80017b8:	d0e1      	beq.n	800177e <__gedf2+0x52>
 80017ba:	e7db      	b.n	8001774 <__gedf2+0x48>
 80017bc:	433a      	orrs	r2, r7
 80017be:	d1e6      	bne.n	800178e <__gedf2+0x62>
 80017c0:	459a      	cmp	sl, r3
 80017c2:	d1d7      	bne.n	8001774 <__gedf2+0x48>
 80017c4:	42a5      	cmp	r5, r4
 80017c6:	dcd5      	bgt.n	8001774 <__gedf2+0x48>
 80017c8:	42a5      	cmp	r5, r4
 80017ca:	db05      	blt.n	80017d8 <__gedf2+0xac>
 80017cc:	42be      	cmp	r6, r7
 80017ce:	d8d1      	bhi.n	8001774 <__gedf2+0x48>
 80017d0:	d008      	beq.n	80017e4 <__gedf2+0xb8>
 80017d2:	2000      	movs	r0, #0
 80017d4:	42be      	cmp	r6, r7
 80017d6:	d2d2      	bcs.n	800177e <__gedf2+0x52>
 80017d8:	4650      	mov	r0, sl
 80017da:	2301      	movs	r3, #1
 80017dc:	3801      	subs	r0, #1
 80017de:	4398      	bics	r0, r3
 80017e0:	3001      	adds	r0, #1
 80017e2:	e7cc      	b.n	800177e <__gedf2+0x52>
 80017e4:	45c8      	cmp	r8, r9
 80017e6:	d8c5      	bhi.n	8001774 <__gedf2+0x48>
 80017e8:	2000      	movs	r0, #0
 80017ea:	45c8      	cmp	r8, r9
 80017ec:	d3f4      	bcc.n	80017d8 <__gedf2+0xac>
 80017ee:	e7c6      	b.n	800177e <__gedf2+0x52>
 80017f0:	000007ff 	.word	0x000007ff

080017f4 <__ledf2>:
 80017f4:	b5f0      	push	{r4, r5, r6, r7, lr}
 80017f6:	464f      	mov	r7, r9
 80017f8:	4646      	mov	r6, r8
 80017fa:	46d6      	mov	lr, sl
 80017fc:	004d      	lsls	r5, r1, #1
 80017fe:	b5c0      	push	{r6, r7, lr}
 8001800:	030e      	lsls	r6, r1, #12
 8001802:	0fc9      	lsrs	r1, r1, #31
 8001804:	468a      	mov	sl, r1
 8001806:	492e      	ldr	r1, [pc, #184]	; (80018c0 <__ledf2+0xcc>)
 8001808:	031f      	lsls	r7, r3, #12
 800180a:	005c      	lsls	r4, r3, #1
 800180c:	4680      	mov	r8, r0
 800180e:	0b36      	lsrs	r6, r6, #12
 8001810:	0d6d      	lsrs	r5, r5, #21
 8001812:	4691      	mov	r9, r2
 8001814:	0b3f      	lsrs	r7, r7, #12
 8001816:	0d64      	lsrs	r4, r4, #21
 8001818:	0fdb      	lsrs	r3, r3, #31
 800181a:	428d      	cmp	r5, r1
 800181c:	d018      	beq.n	8001850 <__ledf2+0x5c>
 800181e:	428c      	cmp	r4, r1
 8001820:	d011      	beq.n	8001846 <__ledf2+0x52>
 8001822:	2d00      	cmp	r5, #0
 8001824:	d118      	bne.n	8001858 <__ledf2+0x64>
 8001826:	4330      	orrs	r0, r6
 8001828:	4684      	mov	ip, r0
 800182a:	2c00      	cmp	r4, #0
 800182c:	d11e      	bne.n	800186c <__ledf2+0x78>
 800182e:	433a      	orrs	r2, r7
 8001830:	d11c      	bne.n	800186c <__ledf2+0x78>
 8001832:	4663      	mov	r3, ip
 8001834:	2000      	movs	r0, #0
 8001836:	2b00      	cmp	r3, #0
 8001838:	d030      	beq.n	800189c <__ledf2+0xa8>
 800183a:	4651      	mov	r1, sl
 800183c:	2002      	movs	r0, #2
 800183e:	3901      	subs	r1, #1
 8001840:	4008      	ands	r0, r1
 8001842:	3801      	subs	r0, #1
 8001844:	e02a      	b.n	800189c <__ledf2+0xa8>
 8001846:	0039      	movs	r1, r7
 8001848:	4311      	orrs	r1, r2
 800184a:	d0ea      	beq.n	8001822 <__ledf2+0x2e>
 800184c:	2002      	movs	r0, #2
 800184e:	e025      	b.n	800189c <__ledf2+0xa8>
 8001850:	4330      	orrs	r0, r6
 8001852:	d1fb      	bne.n	800184c <__ledf2+0x58>
 8001854:	42ac      	cmp	r4, r5
 8001856:	d026      	beq.n	80018a6 <__ledf2+0xb2>
 8001858:	2c00      	cmp	r4, #0
 800185a:	d126      	bne.n	80018aa <__ledf2+0xb6>
 800185c:	433a      	orrs	r2, r7
 800185e:	d124      	bne.n	80018aa <__ledf2+0xb6>
 8001860:	4651      	mov	r1, sl
 8001862:	2002      	movs	r0, #2
 8001864:	3901      	subs	r1, #1
 8001866:	4008      	ands	r0, r1
 8001868:	3801      	subs	r0, #1
 800186a:	e017      	b.n	800189c <__ledf2+0xa8>
 800186c:	4662      	mov	r2, ip
 800186e:	2a00      	cmp	r2, #0
 8001870:	d00f      	beq.n	8001892 <__ledf2+0x9e>
 8001872:	459a      	cmp	sl, r3
 8001874:	d1e1      	bne.n	800183a <__ledf2+0x46>
 8001876:	42a5      	cmp	r5, r4
 8001878:	db05      	blt.n	8001886 <__ledf2+0x92>
 800187a:	42be      	cmp	r6, r7
 800187c:	d8dd      	bhi.n	800183a <__ledf2+0x46>
 800187e:	d019      	beq.n	80018b4 <__ledf2+0xc0>
 8001880:	2000      	movs	r0, #0
 8001882:	42be      	cmp	r6, r7
 8001884:	d20a      	bcs.n	800189c <__ledf2+0xa8>
 8001886:	4650      	mov	r0, sl
 8001888:	2301      	movs	r3, #1
 800188a:	3801      	subs	r0, #1
 800188c:	4398      	bics	r0, r3
 800188e:	3001      	adds	r0, #1
 8001890:	e004      	b.n	800189c <__ledf2+0xa8>
 8001892:	2201      	movs	r2, #1
 8001894:	3b01      	subs	r3, #1
 8001896:	4393      	bics	r3, r2
 8001898:	0018      	movs	r0, r3
 800189a:	3001      	adds	r0, #1
 800189c:	bc1c      	pop	{r2, r3, r4}
 800189e:	4690      	mov	r8, r2
 80018a0:	4699      	mov	r9, r3
 80018a2:	46a2      	mov	sl, r4
 80018a4:	bdf0      	pop	{r4, r5, r6, r7, pc}
 80018a6:	433a      	orrs	r2, r7
 80018a8:	d1d0      	bne.n	800184c <__ledf2+0x58>
 80018aa:	459a      	cmp	sl, r3
 80018ac:	d1c5      	bne.n	800183a <__ledf2+0x46>
 80018ae:	42a5      	cmp	r5, r4
 80018b0:	dcc3      	bgt.n	800183a <__ledf2+0x46>
 80018b2:	e7e0      	b.n	8001876 <__ledf2+0x82>
 80018b4:	45c8      	cmp	r8, r9
 80018b6:	d8c0      	bhi.n	800183a <__ledf2+0x46>
 80018b8:	2000      	movs	r0, #0
 80018ba:	45c8      	cmp	r8, r9
 80018bc:	d3e3      	bcc.n	8001886 <__ledf2+0x92>
 80018be:	e7ed      	b.n	800189c <__ledf2+0xa8>
 80018c0:	000007ff 	.word	0x000007ff

080018c4 <__aeabi_dmul>:
 80018c4:	b5f0      	push	{r4, r5, r6, r7, lr}
 80018c6:	4657      	mov	r7, sl
 80018c8:	46de      	mov	lr, fp
 80018ca:	464e      	mov	r6, r9
 80018cc:	4645      	mov	r5, r8
 80018ce:	b5e0      	push	{r5, r6, r7, lr}
 80018d0:	4683      	mov	fp, r0
 80018d2:	0006      	movs	r6, r0
 80018d4:	030f      	lsls	r7, r1, #12
 80018d6:	0048      	lsls	r0, r1, #1
 80018d8:	b087      	sub	sp, #28
 80018da:	4692      	mov	sl, r2
 80018dc:	001d      	movs	r5, r3
 80018de:	0b3f      	lsrs	r7, r7, #12
 80018e0:	0d40      	lsrs	r0, r0, #21
 80018e2:	0fcc      	lsrs	r4, r1, #31
 80018e4:	2800      	cmp	r0, #0
 80018e6:	d100      	bne.n	80018ea <__aeabi_dmul+0x26>
 80018e8:	e06f      	b.n	80019ca <__aeabi_dmul+0x106>
 80018ea:	4bde      	ldr	r3, [pc, #888]	; (8001c64 <__aeabi_dmul+0x3a0>)
 80018ec:	4298      	cmp	r0, r3
 80018ee:	d038      	beq.n	8001962 <__aeabi_dmul+0x9e>
 80018f0:	2380      	movs	r3, #128	; 0x80
 80018f2:	00ff      	lsls	r7, r7, #3
 80018f4:	041b      	lsls	r3, r3, #16
 80018f6:	431f      	orrs	r7, r3
 80018f8:	0f73      	lsrs	r3, r6, #29
 80018fa:	433b      	orrs	r3, r7
 80018fc:	9301      	str	r3, [sp, #4]
 80018fe:	4bda      	ldr	r3, [pc, #872]	; (8001c68 <__aeabi_dmul+0x3a4>)
 8001900:	2700      	movs	r7, #0
 8001902:	4699      	mov	r9, r3
 8001904:	2300      	movs	r3, #0
 8001906:	469b      	mov	fp, r3
 8001908:	00f6      	lsls	r6, r6, #3
 800190a:	4481      	add	r9, r0
 800190c:	032b      	lsls	r3, r5, #12
 800190e:	0069      	lsls	r1, r5, #1
 8001910:	0b1b      	lsrs	r3, r3, #12
 8001912:	4652      	mov	r2, sl
 8001914:	4698      	mov	r8, r3
 8001916:	0d49      	lsrs	r1, r1, #21
 8001918:	0fed      	lsrs	r5, r5, #31
 800191a:	2900      	cmp	r1, #0
 800191c:	d100      	bne.n	8001920 <__aeabi_dmul+0x5c>
 800191e:	e085      	b.n	8001a2c <__aeabi_dmul+0x168>
 8001920:	4bd0      	ldr	r3, [pc, #832]	; (8001c64 <__aeabi_dmul+0x3a0>)
 8001922:	4299      	cmp	r1, r3
 8001924:	d100      	bne.n	8001928 <__aeabi_dmul+0x64>
 8001926:	e073      	b.n	8001a10 <__aeabi_dmul+0x14c>
 8001928:	4643      	mov	r3, r8
 800192a:	00da      	lsls	r2, r3, #3
 800192c:	2380      	movs	r3, #128	; 0x80
 800192e:	041b      	lsls	r3, r3, #16
 8001930:	4313      	orrs	r3, r2
 8001932:	4652      	mov	r2, sl
 8001934:	48cc      	ldr	r0, [pc, #816]	; (8001c68 <__aeabi_dmul+0x3a4>)
 8001936:	0f52      	lsrs	r2, r2, #29
 8001938:	4684      	mov	ip, r0
 800193a:	4313      	orrs	r3, r2
 800193c:	4652      	mov	r2, sl
 800193e:	2000      	movs	r0, #0
 8001940:	4461      	add	r1, ip
 8001942:	00d2      	lsls	r2, r2, #3
 8001944:	4489      	add	r9, r1
 8001946:	0021      	movs	r1, r4
 8001948:	4069      	eors	r1, r5
 800194a:	9100      	str	r1, [sp, #0]
 800194c:	468c      	mov	ip, r1
 800194e:	2101      	movs	r1, #1
 8001950:	4449      	add	r1, r9
 8001952:	468a      	mov	sl, r1
 8001954:	2f0f      	cmp	r7, #15
 8001956:	d900      	bls.n	800195a <__aeabi_dmul+0x96>
 8001958:	e090      	b.n	8001a7c <__aeabi_dmul+0x1b8>
 800195a:	49c4      	ldr	r1, [pc, #784]	; (8001c6c <__aeabi_dmul+0x3a8>)
 800195c:	00bf      	lsls	r7, r7, #2
 800195e:	59cf      	ldr	r7, [r1, r7]
 8001960:	46bf      	mov	pc, r7
 8001962:	465b      	mov	r3, fp
 8001964:	433b      	orrs	r3, r7
 8001966:	9301      	str	r3, [sp, #4]
 8001968:	d000      	beq.n	800196c <__aeabi_dmul+0xa8>
 800196a:	e16a      	b.n	8001c42 <__aeabi_dmul+0x37e>
 800196c:	2302      	movs	r3, #2
 800196e:	2708      	movs	r7, #8
 8001970:	2600      	movs	r6, #0
 8001972:	4681      	mov	r9, r0
 8001974:	469b      	mov	fp, r3
 8001976:	e7c9      	b.n	800190c <__aeabi_dmul+0x48>
 8001978:	0032      	movs	r2, r6
 800197a:	4658      	mov	r0, fp
 800197c:	9b01      	ldr	r3, [sp, #4]
 800197e:	4661      	mov	r1, ip
 8001980:	9100      	str	r1, [sp, #0]
 8001982:	2802      	cmp	r0, #2
 8001984:	d100      	bne.n	8001988 <__aeabi_dmul+0xc4>
 8001986:	e075      	b.n	8001a74 <__aeabi_dmul+0x1b0>
 8001988:	2803      	cmp	r0, #3
 800198a:	d100      	bne.n	800198e <__aeabi_dmul+0xca>
 800198c:	e1fe      	b.n	8001d8c <__aeabi_dmul+0x4c8>
 800198e:	2801      	cmp	r0, #1
 8001990:	d000      	beq.n	8001994 <__aeabi_dmul+0xd0>
 8001992:	e12c      	b.n	8001bee <__aeabi_dmul+0x32a>
 8001994:	2300      	movs	r3, #0
 8001996:	2700      	movs	r7, #0
 8001998:	2600      	movs	r6, #0
 800199a:	2500      	movs	r5, #0
 800199c:	033f      	lsls	r7, r7, #12
 800199e:	0d2a      	lsrs	r2, r5, #20
 80019a0:	0b3f      	lsrs	r7, r7, #12
 80019a2:	48b3      	ldr	r0, [pc, #716]	; (8001c70 <__aeabi_dmul+0x3ac>)
 80019a4:	0512      	lsls	r2, r2, #20
 80019a6:	433a      	orrs	r2, r7
 80019a8:	4002      	ands	r2, r0
 80019aa:	051b      	lsls	r3, r3, #20
 80019ac:	4313      	orrs	r3, r2
 80019ae:	9a00      	ldr	r2, [sp, #0]
 80019b0:	005b      	lsls	r3, r3, #1
 80019b2:	07d1      	lsls	r1, r2, #31
 80019b4:	085b      	lsrs	r3, r3, #1
 80019b6:	430b      	orrs	r3, r1
 80019b8:	0030      	movs	r0, r6
 80019ba:	0019      	movs	r1, r3
 80019bc:	b007      	add	sp, #28
 80019be:	bc3c      	pop	{r2, r3, r4, r5}
 80019c0:	4690      	mov	r8, r2
 80019c2:	4699      	mov	r9, r3
 80019c4:	46a2      	mov	sl, r4
 80019c6:	46ab      	mov	fp, r5
 80019c8:	bdf0      	pop	{r4, r5, r6, r7, pc}
 80019ca:	465b      	mov	r3, fp
 80019cc:	433b      	orrs	r3, r7
 80019ce:	9301      	str	r3, [sp, #4]
 80019d0:	d100      	bne.n	80019d4 <__aeabi_dmul+0x110>
 80019d2:	e12f      	b.n	8001c34 <__aeabi_dmul+0x370>
 80019d4:	2f00      	cmp	r7, #0
 80019d6:	d100      	bne.n	80019da <__aeabi_dmul+0x116>
 80019d8:	e1a5      	b.n	8001d26 <__aeabi_dmul+0x462>
 80019da:	0038      	movs	r0, r7
 80019dc:	f000 fe20 	bl	8002620 <__clzsi2>
 80019e0:	0003      	movs	r3, r0
 80019e2:	3b0b      	subs	r3, #11
 80019e4:	2b1c      	cmp	r3, #28
 80019e6:	dd00      	ble.n	80019ea <__aeabi_dmul+0x126>
 80019e8:	e196      	b.n	8001d18 <__aeabi_dmul+0x454>
 80019ea:	221d      	movs	r2, #29
 80019ec:	1ad3      	subs	r3, r2, r3
 80019ee:	465a      	mov	r2, fp
 80019f0:	0001      	movs	r1, r0
 80019f2:	40da      	lsrs	r2, r3
 80019f4:	465e      	mov	r6, fp
 80019f6:	3908      	subs	r1, #8
 80019f8:	408f      	lsls	r7, r1
 80019fa:	0013      	movs	r3, r2
 80019fc:	408e      	lsls	r6, r1
 80019fe:	433b      	orrs	r3, r7
 8001a00:	9301      	str	r3, [sp, #4]
 8001a02:	4b9c      	ldr	r3, [pc, #624]	; (8001c74 <__aeabi_dmul+0x3b0>)
 8001a04:	2700      	movs	r7, #0
 8001a06:	1a1b      	subs	r3, r3, r0
 8001a08:	4699      	mov	r9, r3
 8001a0a:	2300      	movs	r3, #0
 8001a0c:	469b      	mov	fp, r3
 8001a0e:	e77d      	b.n	800190c <__aeabi_dmul+0x48>
 8001a10:	4641      	mov	r1, r8
 8001a12:	4653      	mov	r3, sl
 8001a14:	430b      	orrs	r3, r1
 8001a16:	4993      	ldr	r1, [pc, #588]	; (8001c64 <__aeabi_dmul+0x3a0>)
 8001a18:	468c      	mov	ip, r1
 8001a1a:	44e1      	add	r9, ip
 8001a1c:	2b00      	cmp	r3, #0
 8001a1e:	d000      	beq.n	8001a22 <__aeabi_dmul+0x15e>
 8001a20:	e11a      	b.n	8001c58 <__aeabi_dmul+0x394>
 8001a22:	2202      	movs	r2, #2
 8001a24:	2002      	movs	r0, #2
 8001a26:	4317      	orrs	r7, r2
 8001a28:	2200      	movs	r2, #0
 8001a2a:	e78c      	b.n	8001946 <__aeabi_dmul+0x82>
 8001a2c:	4313      	orrs	r3, r2
 8001a2e:	d100      	bne.n	8001a32 <__aeabi_dmul+0x16e>
 8001a30:	e10d      	b.n	8001c4e <__aeabi_dmul+0x38a>
 8001a32:	4643      	mov	r3, r8
 8001a34:	2b00      	cmp	r3, #0
 8001a36:	d100      	bne.n	8001a3a <__aeabi_dmul+0x176>
 8001a38:	e181      	b.n	8001d3e <__aeabi_dmul+0x47a>
 8001a3a:	4640      	mov	r0, r8
 8001a3c:	f000 fdf0 	bl	8002620 <__clzsi2>
 8001a40:	0002      	movs	r2, r0
 8001a42:	3a0b      	subs	r2, #11
 8001a44:	2a1c      	cmp	r2, #28
 8001a46:	dd00      	ble.n	8001a4a <__aeabi_dmul+0x186>
 8001a48:	e172      	b.n	8001d30 <__aeabi_dmul+0x46c>
 8001a4a:	0001      	movs	r1, r0
 8001a4c:	4643      	mov	r3, r8
 8001a4e:	3908      	subs	r1, #8
 8001a50:	408b      	lsls	r3, r1
 8001a52:	4698      	mov	r8, r3
 8001a54:	231d      	movs	r3, #29
 8001a56:	1a9a      	subs	r2, r3, r2
 8001a58:	4653      	mov	r3, sl
 8001a5a:	40d3      	lsrs	r3, r2
 8001a5c:	001a      	movs	r2, r3
 8001a5e:	4643      	mov	r3, r8
 8001a60:	4313      	orrs	r3, r2
 8001a62:	4652      	mov	r2, sl
 8001a64:	408a      	lsls	r2, r1
 8001a66:	4649      	mov	r1, r9
 8001a68:	1a08      	subs	r0, r1, r0
 8001a6a:	4982      	ldr	r1, [pc, #520]	; (8001c74 <__aeabi_dmul+0x3b0>)
 8001a6c:	4689      	mov	r9, r1
 8001a6e:	4481      	add	r9, r0
 8001a70:	2000      	movs	r0, #0
 8001a72:	e768      	b.n	8001946 <__aeabi_dmul+0x82>
 8001a74:	4b7b      	ldr	r3, [pc, #492]	; (8001c64 <__aeabi_dmul+0x3a0>)
 8001a76:	2700      	movs	r7, #0
 8001a78:	2600      	movs	r6, #0
 8001a7a:	e78e      	b.n	800199a <__aeabi_dmul+0xd6>
 8001a7c:	0c14      	lsrs	r4, r2, #16
 8001a7e:	0412      	lsls	r2, r2, #16
 8001a80:	0c12      	lsrs	r2, r2, #16
 8001a82:	0011      	movs	r1, r2
 8001a84:	0c37      	lsrs	r7, r6, #16
 8001a86:	0436      	lsls	r6, r6, #16
 8001a88:	0c35      	lsrs	r5, r6, #16
 8001a8a:	4379      	muls	r1, r7
 8001a8c:	0028      	movs	r0, r5
 8001a8e:	468c      	mov	ip, r1
 8001a90:	002e      	movs	r6, r5
 8001a92:	4360      	muls	r0, r4
 8001a94:	4460      	add	r0, ip
 8001a96:	4683      	mov	fp, r0
 8001a98:	4356      	muls	r6, r2
 8001a9a:	0021      	movs	r1, r4
 8001a9c:	0c30      	lsrs	r0, r6, #16
 8001a9e:	4680      	mov	r8, r0
 8001aa0:	4658      	mov	r0, fp
 8001aa2:	4379      	muls	r1, r7
 8001aa4:	4440      	add	r0, r8
 8001aa6:	9102      	str	r1, [sp, #8]
 8001aa8:	4584      	cmp	ip, r0
 8001aaa:	d906      	bls.n	8001aba <__aeabi_dmul+0x1f6>
 8001aac:	4688      	mov	r8, r1
 8001aae:	2180      	movs	r1, #128	; 0x80
 8001ab0:	0249      	lsls	r1, r1, #9
 8001ab2:	468c      	mov	ip, r1
 8001ab4:	44e0      	add	r8, ip
 8001ab6:	4641      	mov	r1, r8
 8001ab8:	9102      	str	r1, [sp, #8]
 8001aba:	0436      	lsls	r6, r6, #16
 8001abc:	0c01      	lsrs	r1, r0, #16
 8001abe:	0c36      	lsrs	r6, r6, #16
 8001ac0:	0400      	lsls	r0, r0, #16
 8001ac2:	468b      	mov	fp, r1
 8001ac4:	1981      	adds	r1, r0, r6
 8001ac6:	0c1e      	lsrs	r6, r3, #16
 8001ac8:	041b      	lsls	r3, r3, #16
 8001aca:	0c1b      	lsrs	r3, r3, #16
 8001acc:	9103      	str	r1, [sp, #12]
 8001ace:	0019      	movs	r1, r3
 8001ad0:	4379      	muls	r1, r7
 8001ad2:	468c      	mov	ip, r1
 8001ad4:	0028      	movs	r0, r5
 8001ad6:	4375      	muls	r5, r6
 8001ad8:	4465      	add	r5, ip
 8001ada:	46a8      	mov	r8, r5
 8001adc:	4358      	muls	r0, r3
 8001ade:	0c05      	lsrs	r5, r0, #16
 8001ae0:	4445      	add	r5, r8
 8001ae2:	4377      	muls	r7, r6
 8001ae4:	42a9      	cmp	r1, r5
 8001ae6:	d903      	bls.n	8001af0 <__aeabi_dmul+0x22c>
 8001ae8:	2180      	movs	r1, #128	; 0x80
 8001aea:	0249      	lsls	r1, r1, #9
 8001aec:	468c      	mov	ip, r1
 8001aee:	4467      	add	r7, ip
 8001af0:	0c29      	lsrs	r1, r5, #16
 8001af2:	468c      	mov	ip, r1
 8001af4:	0039      	movs	r1, r7
 8001af6:	0400      	lsls	r0, r0, #16
 8001af8:	0c00      	lsrs	r0, r0, #16
 8001afa:	042d      	lsls	r5, r5, #16
 8001afc:	182d      	adds	r5, r5, r0
 8001afe:	4461      	add	r1, ip
 8001b00:	44ab      	add	fp, r5
 8001b02:	9105      	str	r1, [sp, #20]
 8001b04:	4659      	mov	r1, fp
 8001b06:	9104      	str	r1, [sp, #16]
 8001b08:	9901      	ldr	r1, [sp, #4]
 8001b0a:	040f      	lsls	r7, r1, #16
 8001b0c:	0c3f      	lsrs	r7, r7, #16
 8001b0e:	0c08      	lsrs	r0, r1, #16
 8001b10:	0039      	movs	r1, r7
 8001b12:	4351      	muls	r1, r2
 8001b14:	4342      	muls	r2, r0
 8001b16:	4690      	mov	r8, r2
 8001b18:	0002      	movs	r2, r0
 8001b1a:	468c      	mov	ip, r1
 8001b1c:	0c09      	lsrs	r1, r1, #16
 8001b1e:	468b      	mov	fp, r1
 8001b20:	4362      	muls	r2, r4
 8001b22:	437c      	muls	r4, r7
 8001b24:	4444      	add	r4, r8
 8001b26:	445c      	add	r4, fp
 8001b28:	45a0      	cmp	r8, r4
 8001b2a:	d903      	bls.n	8001b34 <__aeabi_dmul+0x270>
 8001b2c:	2180      	movs	r1, #128	; 0x80
 8001b2e:	0249      	lsls	r1, r1, #9
 8001b30:	4688      	mov	r8, r1
 8001b32:	4442      	add	r2, r8
 8001b34:	0c21      	lsrs	r1, r4, #16
 8001b36:	4688      	mov	r8, r1
 8001b38:	4661      	mov	r1, ip
 8001b3a:	0409      	lsls	r1, r1, #16
 8001b3c:	0c09      	lsrs	r1, r1, #16
 8001b3e:	468c      	mov	ip, r1
 8001b40:	0039      	movs	r1, r7
 8001b42:	4359      	muls	r1, r3
 8001b44:	4343      	muls	r3, r0
 8001b46:	4370      	muls	r0, r6
 8001b48:	437e      	muls	r6, r7
 8001b4a:	0c0f      	lsrs	r7, r1, #16
 8001b4c:	18f6      	adds	r6, r6, r3
 8001b4e:	0424      	lsls	r4, r4, #16
 8001b50:	19be      	adds	r6, r7, r6
 8001b52:	4464      	add	r4, ip
 8001b54:	4442      	add	r2, r8
 8001b56:	468c      	mov	ip, r1
 8001b58:	42b3      	cmp	r3, r6
 8001b5a:	d903      	bls.n	8001b64 <__aeabi_dmul+0x2a0>
 8001b5c:	2380      	movs	r3, #128	; 0x80
 8001b5e:	025b      	lsls	r3, r3, #9
 8001b60:	4698      	mov	r8, r3
 8001b62:	4440      	add	r0, r8
 8001b64:	9b02      	ldr	r3, [sp, #8]
 8001b66:	4661      	mov	r1, ip
 8001b68:	4698      	mov	r8, r3
 8001b6a:	9b04      	ldr	r3, [sp, #16]
 8001b6c:	0437      	lsls	r7, r6, #16
 8001b6e:	4443      	add	r3, r8
 8001b70:	469b      	mov	fp, r3
 8001b72:	45ab      	cmp	fp, r5
 8001b74:	41ad      	sbcs	r5, r5
 8001b76:	426b      	negs	r3, r5
 8001b78:	040d      	lsls	r5, r1, #16
 8001b7a:	9905      	ldr	r1, [sp, #20]
 8001b7c:	0c2d      	lsrs	r5, r5, #16
 8001b7e:	468c      	mov	ip, r1
 8001b80:	197f      	adds	r7, r7, r5
 8001b82:	4467      	add	r7, ip
 8001b84:	18fd      	adds	r5, r7, r3
 8001b86:	46a8      	mov	r8, r5
 8001b88:	465d      	mov	r5, fp
 8001b8a:	192d      	adds	r5, r5, r4
 8001b8c:	42a5      	cmp	r5, r4
 8001b8e:	41a4      	sbcs	r4, r4
 8001b90:	4693      	mov	fp, r2
 8001b92:	4264      	negs	r4, r4
 8001b94:	46a4      	mov	ip, r4
 8001b96:	44c3      	add	fp, r8
 8001b98:	44dc      	add	ip, fp
 8001b9a:	428f      	cmp	r7, r1
 8001b9c:	41bf      	sbcs	r7, r7
 8001b9e:	4598      	cmp	r8, r3
 8001ba0:	419b      	sbcs	r3, r3
 8001ba2:	4593      	cmp	fp, r2
 8001ba4:	4192      	sbcs	r2, r2
 8001ba6:	45a4      	cmp	ip, r4
 8001ba8:	41a4      	sbcs	r4, r4
 8001baa:	425b      	negs	r3, r3
 8001bac:	427f      	negs	r7, r7
 8001bae:	431f      	orrs	r7, r3
 8001bb0:	0c36      	lsrs	r6, r6, #16
 8001bb2:	4252      	negs	r2, r2
 8001bb4:	4264      	negs	r4, r4
 8001bb6:	19bf      	adds	r7, r7, r6
 8001bb8:	4322      	orrs	r2, r4
 8001bba:	18bf      	adds	r7, r7, r2
 8001bbc:	4662      	mov	r2, ip
 8001bbe:	1838      	adds	r0, r7, r0
 8001bc0:	0243      	lsls	r3, r0, #9
 8001bc2:	0dd2      	lsrs	r2, r2, #23
 8001bc4:	9903      	ldr	r1, [sp, #12]
 8001bc6:	4313      	orrs	r3, r2
 8001bc8:	026a      	lsls	r2, r5, #9
 8001bca:	430a      	orrs	r2, r1
 8001bcc:	1e50      	subs	r0, r2, #1
 8001bce:	4182      	sbcs	r2, r0
 8001bd0:	4661      	mov	r1, ip
 8001bd2:	0ded      	lsrs	r5, r5, #23
 8001bd4:	432a      	orrs	r2, r5
 8001bd6:	024e      	lsls	r6, r1, #9
 8001bd8:	4332      	orrs	r2, r6
 8001bda:	01d9      	lsls	r1, r3, #7
 8001bdc:	d400      	bmi.n	8001be0 <__aeabi_dmul+0x31c>
 8001bde:	e0b3      	b.n	8001d48 <__aeabi_dmul+0x484>
 8001be0:	2601      	movs	r6, #1
 8001be2:	0850      	lsrs	r0, r2, #1
 8001be4:	4032      	ands	r2, r6
 8001be6:	4302      	orrs	r2, r0
 8001be8:	07de      	lsls	r6, r3, #31
 8001bea:	4332      	orrs	r2, r6
 8001bec:	085b      	lsrs	r3, r3, #1
 8001bee:	4c22      	ldr	r4, [pc, #136]	; (8001c78 <__aeabi_dmul+0x3b4>)
 8001bf0:	4454      	add	r4, sl
 8001bf2:	2c00      	cmp	r4, #0
 8001bf4:	dd62      	ble.n	8001cbc <__aeabi_dmul+0x3f8>
 8001bf6:	0751      	lsls	r1, r2, #29
 8001bf8:	d009      	beq.n	8001c0e <__aeabi_dmul+0x34a>
 8001bfa:	200f      	movs	r0, #15
 8001bfc:	4010      	ands	r0, r2
 8001bfe:	2804      	cmp	r0, #4
 8001c00:	d005      	beq.n	8001c0e <__aeabi_dmul+0x34a>
 8001c02:	1d10      	adds	r0, r2, #4
 8001c04:	4290      	cmp	r0, r2
 8001c06:	4192      	sbcs	r2, r2
 8001c08:	4252      	negs	r2, r2
 8001c0a:	189b      	adds	r3, r3, r2
 8001c0c:	0002      	movs	r2, r0
 8001c0e:	01d9      	lsls	r1, r3, #7
 8001c10:	d504      	bpl.n	8001c1c <__aeabi_dmul+0x358>
 8001c12:	2480      	movs	r4, #128	; 0x80
 8001c14:	4819      	ldr	r0, [pc, #100]	; (8001c7c <__aeabi_dmul+0x3b8>)
 8001c16:	00e4      	lsls	r4, r4, #3
 8001c18:	4003      	ands	r3, r0
 8001c1a:	4454      	add	r4, sl
 8001c1c:	4818      	ldr	r0, [pc, #96]	; (8001c80 <__aeabi_dmul+0x3bc>)
 8001c1e:	4284      	cmp	r4, r0
 8001c20:	dd00      	ble.n	8001c24 <__aeabi_dmul+0x360>
 8001c22:	e727      	b.n	8001a74 <__aeabi_dmul+0x1b0>
 8001c24:	075e      	lsls	r6, r3, #29
 8001c26:	025b      	lsls	r3, r3, #9
 8001c28:	08d2      	lsrs	r2, r2, #3
 8001c2a:	0b1f      	lsrs	r7, r3, #12
 8001c2c:	0563      	lsls	r3, r4, #21
 8001c2e:	4316      	orrs	r6, r2
 8001c30:	0d5b      	lsrs	r3, r3, #21
 8001c32:	e6b2      	b.n	800199a <__aeabi_dmul+0xd6>
 8001c34:	2300      	movs	r3, #0
 8001c36:	4699      	mov	r9, r3
 8001c38:	3301      	adds	r3, #1
 8001c3a:	2704      	movs	r7, #4
 8001c3c:	2600      	movs	r6, #0
 8001c3e:	469b      	mov	fp, r3
 8001c40:	e664      	b.n	800190c <__aeabi_dmul+0x48>
 8001c42:	2303      	movs	r3, #3
 8001c44:	9701      	str	r7, [sp, #4]
 8001c46:	4681      	mov	r9, r0
 8001c48:	270c      	movs	r7, #12
 8001c4a:	469b      	mov	fp, r3
 8001c4c:	e65e      	b.n	800190c <__aeabi_dmul+0x48>
 8001c4e:	2201      	movs	r2, #1
 8001c50:	2001      	movs	r0, #1
 8001c52:	4317      	orrs	r7, r2
 8001c54:	2200      	movs	r2, #0
 8001c56:	e676      	b.n	8001946 <__aeabi_dmul+0x82>
 8001c58:	2303      	movs	r3, #3
 8001c5a:	2003      	movs	r0, #3
 8001c5c:	431f      	orrs	r7, r3
 8001c5e:	4643      	mov	r3, r8
 8001c60:	e671      	b.n	8001946 <__aeabi_dmul+0x82>
 8001c62:	46c0      	nop			; (mov r8, r8)
 8001c64:	000007ff 	.word	0x000007ff
 8001c68:	fffffc01 	.word	0xfffffc01
 8001c6c:	0801a930 	.word	0x0801a930
 8001c70:	800fffff 	.word	0x800fffff
 8001c74:	fffffc0d 	.word	0xfffffc0d
 8001c78:	000003ff 	.word	0x000003ff
 8001c7c:	feffffff 	.word	0xfeffffff
 8001c80:	000007fe 	.word	0x000007fe
 8001c84:	2300      	movs	r3, #0
 8001c86:	2780      	movs	r7, #128	; 0x80
 8001c88:	9300      	str	r3, [sp, #0]
 8001c8a:	033f      	lsls	r7, r7, #12
 8001c8c:	2600      	movs	r6, #0
 8001c8e:	4b43      	ldr	r3, [pc, #268]	; (8001d9c <__aeabi_dmul+0x4d8>)
 8001c90:	e683      	b.n	800199a <__aeabi_dmul+0xd6>
 8001c92:	9b01      	ldr	r3, [sp, #4]
 8001c94:	0032      	movs	r2, r6
 8001c96:	46a4      	mov	ip, r4
 8001c98:	4658      	mov	r0, fp
 8001c9a:	e670      	b.n	800197e <__aeabi_dmul+0xba>
 8001c9c:	46ac      	mov	ip, r5
 8001c9e:	e66e      	b.n	800197e <__aeabi_dmul+0xba>
 8001ca0:	2780      	movs	r7, #128	; 0x80
 8001ca2:	9901      	ldr	r1, [sp, #4]
 8001ca4:	033f      	lsls	r7, r7, #12
 8001ca6:	4239      	tst	r1, r7
 8001ca8:	d02d      	beq.n	8001d06 <__aeabi_dmul+0x442>
 8001caa:	423b      	tst	r3, r7
 8001cac:	d12b      	bne.n	8001d06 <__aeabi_dmul+0x442>
 8001cae:	431f      	orrs	r7, r3
 8001cb0:	033f      	lsls	r7, r7, #12
 8001cb2:	0b3f      	lsrs	r7, r7, #12
 8001cb4:	9500      	str	r5, [sp, #0]
 8001cb6:	0016      	movs	r6, r2
 8001cb8:	4b38      	ldr	r3, [pc, #224]	; (8001d9c <__aeabi_dmul+0x4d8>)
 8001cba:	e66e      	b.n	800199a <__aeabi_dmul+0xd6>
 8001cbc:	2501      	movs	r5, #1
 8001cbe:	1b2d      	subs	r5, r5, r4
 8001cc0:	2d38      	cmp	r5, #56	; 0x38
 8001cc2:	dd00      	ble.n	8001cc6 <__aeabi_dmul+0x402>
 8001cc4:	e666      	b.n	8001994 <__aeabi_dmul+0xd0>
 8001cc6:	2d1f      	cmp	r5, #31
 8001cc8:	dc40      	bgt.n	8001d4c <__aeabi_dmul+0x488>
 8001cca:	4835      	ldr	r0, [pc, #212]	; (8001da0 <__aeabi_dmul+0x4dc>)
 8001ccc:	001c      	movs	r4, r3
 8001cce:	4450      	add	r0, sl
 8001cd0:	0016      	movs	r6, r2
 8001cd2:	4082      	lsls	r2, r0
 8001cd4:	4084      	lsls	r4, r0
 8001cd6:	40ee      	lsrs	r6, r5
 8001cd8:	1e50      	subs	r0, r2, #1
 8001cda:	4182      	sbcs	r2, r0
 8001cdc:	4334      	orrs	r4, r6
 8001cde:	4314      	orrs	r4, r2
 8001ce0:	40eb      	lsrs	r3, r5
 8001ce2:	0762      	lsls	r2, r4, #29
 8001ce4:	d009      	beq.n	8001cfa <__aeabi_dmul+0x436>
 8001ce6:	220f      	movs	r2, #15
 8001ce8:	4022      	ands	r2, r4
 8001cea:	2a04      	cmp	r2, #4
 8001cec:	d005      	beq.n	8001cfa <__aeabi_dmul+0x436>
 8001cee:	0022      	movs	r2, r4
 8001cf0:	1d14      	adds	r4, r2, #4
 8001cf2:	4294      	cmp	r4, r2
 8001cf4:	4180      	sbcs	r0, r0
 8001cf6:	4240      	negs	r0, r0
 8001cf8:	181b      	adds	r3, r3, r0
 8001cfa:	021a      	lsls	r2, r3, #8
 8001cfc:	d53e      	bpl.n	8001d7c <__aeabi_dmul+0x4b8>
 8001cfe:	2301      	movs	r3, #1
 8001d00:	2700      	movs	r7, #0
 8001d02:	2600      	movs	r6, #0
 8001d04:	e649      	b.n	800199a <__aeabi_dmul+0xd6>
 8001d06:	2780      	movs	r7, #128	; 0x80
 8001d08:	9b01      	ldr	r3, [sp, #4]
 8001d0a:	033f      	lsls	r7, r7, #12
 8001d0c:	431f      	orrs	r7, r3
 8001d0e:	033f      	lsls	r7, r7, #12
 8001d10:	0b3f      	lsrs	r7, r7, #12
 8001d12:	9400      	str	r4, [sp, #0]
 8001d14:	4b21      	ldr	r3, [pc, #132]	; (8001d9c <__aeabi_dmul+0x4d8>)
 8001d16:	e640      	b.n	800199a <__aeabi_dmul+0xd6>
 8001d18:	0003      	movs	r3, r0
 8001d1a:	465a      	mov	r2, fp
 8001d1c:	3b28      	subs	r3, #40	; 0x28
 8001d1e:	409a      	lsls	r2, r3
 8001d20:	2600      	movs	r6, #0
 8001d22:	9201      	str	r2, [sp, #4]
 8001d24:	e66d      	b.n	8001a02 <__aeabi_dmul+0x13e>
 8001d26:	4658      	mov	r0, fp
 8001d28:	f000 fc7a 	bl	8002620 <__clzsi2>
 8001d2c:	3020      	adds	r0, #32
 8001d2e:	e657      	b.n	80019e0 <__aeabi_dmul+0x11c>
 8001d30:	0003      	movs	r3, r0
 8001d32:	4652      	mov	r2, sl
 8001d34:	3b28      	subs	r3, #40	; 0x28
 8001d36:	409a      	lsls	r2, r3
 8001d38:	0013      	movs	r3, r2
 8001d3a:	2200      	movs	r2, #0
 8001d3c:	e693      	b.n	8001a66 <__aeabi_dmul+0x1a2>
 8001d3e:	4650      	mov	r0, sl
 8001d40:	f000 fc6e 	bl	8002620 <__clzsi2>
 8001d44:	3020      	adds	r0, #32
 8001d46:	e67b      	b.n	8001a40 <__aeabi_dmul+0x17c>
 8001d48:	46ca      	mov	sl, r9
 8001d4a:	e750      	b.n	8001bee <__aeabi_dmul+0x32a>
 8001d4c:	201f      	movs	r0, #31
 8001d4e:	001e      	movs	r6, r3
 8001d50:	4240      	negs	r0, r0
 8001d52:	1b04      	subs	r4, r0, r4
 8001d54:	40e6      	lsrs	r6, r4
 8001d56:	2d20      	cmp	r5, #32
 8001d58:	d003      	beq.n	8001d62 <__aeabi_dmul+0x49e>
 8001d5a:	4c12      	ldr	r4, [pc, #72]	; (8001da4 <__aeabi_dmul+0x4e0>)
 8001d5c:	4454      	add	r4, sl
 8001d5e:	40a3      	lsls	r3, r4
 8001d60:	431a      	orrs	r2, r3
 8001d62:	1e50      	subs	r0, r2, #1
 8001d64:	4182      	sbcs	r2, r0
 8001d66:	4332      	orrs	r2, r6
 8001d68:	2607      	movs	r6, #7
 8001d6a:	2700      	movs	r7, #0
 8001d6c:	4016      	ands	r6, r2
 8001d6e:	d009      	beq.n	8001d84 <__aeabi_dmul+0x4c0>
 8001d70:	200f      	movs	r0, #15
 8001d72:	2300      	movs	r3, #0
 8001d74:	4010      	ands	r0, r2
 8001d76:	0014      	movs	r4, r2
 8001d78:	2804      	cmp	r0, #4
 8001d7a:	d1b9      	bne.n	8001cf0 <__aeabi_dmul+0x42c>
 8001d7c:	0022      	movs	r2, r4
 8001d7e:	075e      	lsls	r6, r3, #29
 8001d80:	025b      	lsls	r3, r3, #9
 8001d82:	0b1f      	lsrs	r7, r3, #12
 8001d84:	08d2      	lsrs	r2, r2, #3
 8001d86:	4316      	orrs	r6, r2
 8001d88:	2300      	movs	r3, #0
 8001d8a:	e606      	b.n	800199a <__aeabi_dmul+0xd6>
 8001d8c:	2780      	movs	r7, #128	; 0x80
 8001d8e:	033f      	lsls	r7, r7, #12
 8001d90:	431f      	orrs	r7, r3
 8001d92:	033f      	lsls	r7, r7, #12
 8001d94:	0b3f      	lsrs	r7, r7, #12
 8001d96:	0016      	movs	r6, r2
 8001d98:	4b00      	ldr	r3, [pc, #0]	; (8001d9c <__aeabi_dmul+0x4d8>)
 8001d9a:	e5fe      	b.n	800199a <__aeabi_dmul+0xd6>
 8001d9c:	000007ff 	.word	0x000007ff
 8001da0:	0000041e 	.word	0x0000041e
 8001da4:	0000043e 	.word	0x0000043e

08001da8 <__aeabi_dsub>:
 8001da8:	b5f8      	push	{r3, r4, r5, r6, r7, lr}
 8001daa:	4657      	mov	r7, sl
 8001dac:	464e      	mov	r6, r9
 8001dae:	4645      	mov	r5, r8
 8001db0:	46de      	mov	lr, fp
 8001db2:	000c      	movs	r4, r1
 8001db4:	0309      	lsls	r1, r1, #12
 8001db6:	b5e0      	push	{r5, r6, r7, lr}
 8001db8:	0a49      	lsrs	r1, r1, #9
 8001dba:	0f46      	lsrs	r6, r0, #29
 8001dbc:	005f      	lsls	r7, r3, #1
 8001dbe:	4331      	orrs	r1, r6
 8001dc0:	031e      	lsls	r6, r3, #12
 8001dc2:	0fdb      	lsrs	r3, r3, #31
 8001dc4:	0a76      	lsrs	r6, r6, #9
 8001dc6:	469b      	mov	fp, r3
 8001dc8:	0f53      	lsrs	r3, r2, #29
 8001dca:	4333      	orrs	r3, r6
 8001dcc:	4ec8      	ldr	r6, [pc, #800]	; (80020f0 <__aeabi_dsub+0x348>)
 8001dce:	0065      	lsls	r5, r4, #1
 8001dd0:	00c0      	lsls	r0, r0, #3
 8001dd2:	0fe4      	lsrs	r4, r4, #31
 8001dd4:	00d2      	lsls	r2, r2, #3
 8001dd6:	0d6d      	lsrs	r5, r5, #21
 8001dd8:	46a2      	mov	sl, r4
 8001dda:	4681      	mov	r9, r0
 8001ddc:	0d7f      	lsrs	r7, r7, #21
 8001dde:	469c      	mov	ip, r3
 8001de0:	4690      	mov	r8, r2
 8001de2:	42b7      	cmp	r7, r6
 8001de4:	d100      	bne.n	8001de8 <__aeabi_dsub+0x40>
 8001de6:	e0b9      	b.n	8001f5c <__aeabi_dsub+0x1b4>
 8001de8:	465b      	mov	r3, fp
 8001dea:	2601      	movs	r6, #1
 8001dec:	4073      	eors	r3, r6
 8001dee:	469b      	mov	fp, r3
 8001df0:	1bee      	subs	r6, r5, r7
 8001df2:	45a3      	cmp	fp, r4
 8001df4:	d100      	bne.n	8001df8 <__aeabi_dsub+0x50>
 8001df6:	e083      	b.n	8001f00 <__aeabi_dsub+0x158>
 8001df8:	2e00      	cmp	r6, #0
 8001dfa:	dd63      	ble.n	8001ec4 <__aeabi_dsub+0x11c>
 8001dfc:	2f00      	cmp	r7, #0
 8001dfe:	d000      	beq.n	8001e02 <__aeabi_dsub+0x5a>
 8001e00:	e0b1      	b.n	8001f66 <__aeabi_dsub+0x1be>
 8001e02:	4663      	mov	r3, ip
 8001e04:	4313      	orrs	r3, r2
 8001e06:	d100      	bne.n	8001e0a <__aeabi_dsub+0x62>
 8001e08:	e123      	b.n	8002052 <__aeabi_dsub+0x2aa>
 8001e0a:	1e73      	subs	r3, r6, #1
 8001e0c:	2b00      	cmp	r3, #0
 8001e0e:	d000      	beq.n	8001e12 <__aeabi_dsub+0x6a>
 8001e10:	e1ba      	b.n	8002188 <__aeabi_dsub+0x3e0>
 8001e12:	1a86      	subs	r6, r0, r2
 8001e14:	4663      	mov	r3, ip
 8001e16:	42b0      	cmp	r0, r6
 8001e18:	4180      	sbcs	r0, r0
 8001e1a:	2501      	movs	r5, #1
 8001e1c:	1ac9      	subs	r1, r1, r3
 8001e1e:	4240      	negs	r0, r0
 8001e20:	1a09      	subs	r1, r1, r0
 8001e22:	020b      	lsls	r3, r1, #8
 8001e24:	d400      	bmi.n	8001e28 <__aeabi_dsub+0x80>
 8001e26:	e147      	b.n	80020b8 <__aeabi_dsub+0x310>
 8001e28:	0249      	lsls	r1, r1, #9
 8001e2a:	0a4b      	lsrs	r3, r1, #9
 8001e2c:	4698      	mov	r8, r3
 8001e2e:	4643      	mov	r3, r8
 8001e30:	2b00      	cmp	r3, #0
 8001e32:	d100      	bne.n	8001e36 <__aeabi_dsub+0x8e>
 8001e34:	e189      	b.n	800214a <__aeabi_dsub+0x3a2>
 8001e36:	4640      	mov	r0, r8
 8001e38:	f000 fbf2 	bl	8002620 <__clzsi2>
 8001e3c:	0003      	movs	r3, r0
 8001e3e:	3b08      	subs	r3, #8
 8001e40:	2b1f      	cmp	r3, #31
 8001e42:	dd00      	ble.n	8001e46 <__aeabi_dsub+0x9e>
 8001e44:	e17c      	b.n	8002140 <__aeabi_dsub+0x398>
 8001e46:	2220      	movs	r2, #32
 8001e48:	0030      	movs	r0, r6
 8001e4a:	1ad2      	subs	r2, r2, r3
 8001e4c:	4641      	mov	r1, r8
 8001e4e:	40d0      	lsrs	r0, r2
 8001e50:	4099      	lsls	r1, r3
 8001e52:	0002      	movs	r2, r0
 8001e54:	409e      	lsls	r6, r3
 8001e56:	430a      	orrs	r2, r1
 8001e58:	429d      	cmp	r5, r3
 8001e5a:	dd00      	ble.n	8001e5e <__aeabi_dsub+0xb6>
 8001e5c:	e16a      	b.n	8002134 <__aeabi_dsub+0x38c>
 8001e5e:	1b5d      	subs	r5, r3, r5
 8001e60:	1c6b      	adds	r3, r5, #1
 8001e62:	2b1f      	cmp	r3, #31
 8001e64:	dd00      	ble.n	8001e68 <__aeabi_dsub+0xc0>
 8001e66:	e194      	b.n	8002192 <__aeabi_dsub+0x3ea>
 8001e68:	2120      	movs	r1, #32
 8001e6a:	0010      	movs	r0, r2
 8001e6c:	0035      	movs	r5, r6
 8001e6e:	1ac9      	subs	r1, r1, r3
 8001e70:	408e      	lsls	r6, r1
 8001e72:	40da      	lsrs	r2, r3
 8001e74:	4088      	lsls	r0, r1
 8001e76:	40dd      	lsrs	r5, r3
 8001e78:	1e71      	subs	r1, r6, #1
 8001e7a:	418e      	sbcs	r6, r1
 8001e7c:	0011      	movs	r1, r2
 8001e7e:	2207      	movs	r2, #7
 8001e80:	4328      	orrs	r0, r5
 8001e82:	2500      	movs	r5, #0
 8001e84:	4306      	orrs	r6, r0
 8001e86:	4032      	ands	r2, r6
 8001e88:	2a00      	cmp	r2, #0
 8001e8a:	d009      	beq.n	8001ea0 <__aeabi_dsub+0xf8>
 8001e8c:	230f      	movs	r3, #15
 8001e8e:	4033      	ands	r3, r6
 8001e90:	2b04      	cmp	r3, #4
 8001e92:	d005      	beq.n	8001ea0 <__aeabi_dsub+0xf8>
 8001e94:	1d33      	adds	r3, r6, #4
 8001e96:	42b3      	cmp	r3, r6
 8001e98:	41b6      	sbcs	r6, r6
 8001e9a:	4276      	negs	r6, r6
 8001e9c:	1989      	adds	r1, r1, r6
 8001e9e:	001e      	movs	r6, r3
 8001ea0:	020b      	lsls	r3, r1, #8
 8001ea2:	d400      	bmi.n	8001ea6 <__aeabi_dsub+0xfe>
 8001ea4:	e23d      	b.n	8002322 <__aeabi_dsub+0x57a>
 8001ea6:	1c6a      	adds	r2, r5, #1
 8001ea8:	4b91      	ldr	r3, [pc, #580]	; (80020f0 <__aeabi_dsub+0x348>)
 8001eaa:	0555      	lsls	r5, r2, #21
 8001eac:	0d6d      	lsrs	r5, r5, #21
 8001eae:	429a      	cmp	r2, r3
 8001eb0:	d100      	bne.n	8001eb4 <__aeabi_dsub+0x10c>
 8001eb2:	e119      	b.n	80020e8 <__aeabi_dsub+0x340>
 8001eb4:	4a8f      	ldr	r2, [pc, #572]	; (80020f4 <__aeabi_dsub+0x34c>)
 8001eb6:	08f6      	lsrs	r6, r6, #3
 8001eb8:	400a      	ands	r2, r1
 8001eba:	0757      	lsls	r7, r2, #29
 8001ebc:	0252      	lsls	r2, r2, #9
 8001ebe:	4337      	orrs	r7, r6
 8001ec0:	0b12      	lsrs	r2, r2, #12
 8001ec2:	e09b      	b.n	8001ffc <__aeabi_dsub+0x254>
 8001ec4:	2e00      	cmp	r6, #0
 8001ec6:	d000      	beq.n	8001eca <__aeabi_dsub+0x122>
 8001ec8:	e0c5      	b.n	8002056 <__aeabi_dsub+0x2ae>
 8001eca:	1c6e      	adds	r6, r5, #1
 8001ecc:	0576      	lsls	r6, r6, #21
 8001ece:	0d76      	lsrs	r6, r6, #21
 8001ed0:	2e01      	cmp	r6, #1
 8001ed2:	dc00      	bgt.n	8001ed6 <__aeabi_dsub+0x12e>
 8001ed4:	e148      	b.n	8002168 <__aeabi_dsub+0x3c0>
 8001ed6:	4667      	mov	r7, ip
 8001ed8:	1a86      	subs	r6, r0, r2
 8001eda:	1bcb      	subs	r3, r1, r7
 8001edc:	42b0      	cmp	r0, r6
 8001ede:	41bf      	sbcs	r7, r7
 8001ee0:	427f      	negs	r7, r7
 8001ee2:	46b8      	mov	r8, r7
 8001ee4:	001f      	movs	r7, r3
 8001ee6:	4643      	mov	r3, r8
 8001ee8:	1aff      	subs	r7, r7, r3
 8001eea:	003b      	movs	r3, r7
 8001eec:	46b8      	mov	r8, r7
 8001eee:	021b      	lsls	r3, r3, #8
 8001ef0:	d500      	bpl.n	8001ef4 <__aeabi_dsub+0x14c>
 8001ef2:	e15f      	b.n	80021b4 <__aeabi_dsub+0x40c>
 8001ef4:	4337      	orrs	r7, r6
 8001ef6:	d19a      	bne.n	8001e2e <__aeabi_dsub+0x86>
 8001ef8:	2200      	movs	r2, #0
 8001efa:	2400      	movs	r4, #0
 8001efc:	2500      	movs	r5, #0
 8001efe:	e079      	b.n	8001ff4 <__aeabi_dsub+0x24c>
 8001f00:	2e00      	cmp	r6, #0
 8001f02:	dc00      	bgt.n	8001f06 <__aeabi_dsub+0x15e>
 8001f04:	e0fa      	b.n	80020fc <__aeabi_dsub+0x354>
 8001f06:	2f00      	cmp	r7, #0
 8001f08:	d100      	bne.n	8001f0c <__aeabi_dsub+0x164>
 8001f0a:	e08d      	b.n	8002028 <__aeabi_dsub+0x280>
 8001f0c:	4b78      	ldr	r3, [pc, #480]	; (80020f0 <__aeabi_dsub+0x348>)
 8001f0e:	429d      	cmp	r5, r3
 8001f10:	d067      	beq.n	8001fe2 <__aeabi_dsub+0x23a>
 8001f12:	2380      	movs	r3, #128	; 0x80
 8001f14:	4667      	mov	r7, ip
 8001f16:	041b      	lsls	r3, r3, #16
 8001f18:	431f      	orrs	r7, r3
 8001f1a:	46bc      	mov	ip, r7
 8001f1c:	2e38      	cmp	r6, #56	; 0x38
 8001f1e:	dc00      	bgt.n	8001f22 <__aeabi_dsub+0x17a>
 8001f20:	e152      	b.n	80021c8 <__aeabi_dsub+0x420>
 8001f22:	4663      	mov	r3, ip
 8001f24:	4313      	orrs	r3, r2
 8001f26:	1e5a      	subs	r2, r3, #1
 8001f28:	4193      	sbcs	r3, r2
 8001f2a:	181e      	adds	r6, r3, r0
 8001f2c:	4286      	cmp	r6, r0
 8001f2e:	4180      	sbcs	r0, r0
 8001f30:	4240      	negs	r0, r0
 8001f32:	1809      	adds	r1, r1, r0
 8001f34:	020b      	lsls	r3, r1, #8
 8001f36:	d400      	bmi.n	8001f3a <__aeabi_dsub+0x192>
 8001f38:	e0be      	b.n	80020b8 <__aeabi_dsub+0x310>
 8001f3a:	4b6d      	ldr	r3, [pc, #436]	; (80020f0 <__aeabi_dsub+0x348>)
 8001f3c:	3501      	adds	r5, #1
 8001f3e:	429d      	cmp	r5, r3
 8001f40:	d100      	bne.n	8001f44 <__aeabi_dsub+0x19c>
 8001f42:	e0d2      	b.n	80020ea <__aeabi_dsub+0x342>
 8001f44:	4a6b      	ldr	r2, [pc, #428]	; (80020f4 <__aeabi_dsub+0x34c>)
 8001f46:	0873      	lsrs	r3, r6, #1
 8001f48:	400a      	ands	r2, r1
 8001f4a:	2101      	movs	r1, #1
 8001f4c:	400e      	ands	r6, r1
 8001f4e:	431e      	orrs	r6, r3
 8001f50:	0851      	lsrs	r1, r2, #1
 8001f52:	07d3      	lsls	r3, r2, #31
 8001f54:	2207      	movs	r2, #7
 8001f56:	431e      	orrs	r6, r3
 8001f58:	4032      	ands	r2, r6
 8001f5a:	e795      	b.n	8001e88 <__aeabi_dsub+0xe0>
 8001f5c:	001e      	movs	r6, r3
 8001f5e:	4316      	orrs	r6, r2
 8001f60:	d000      	beq.n	8001f64 <__aeabi_dsub+0x1bc>
 8001f62:	e745      	b.n	8001df0 <__aeabi_dsub+0x48>
 8001f64:	e740      	b.n	8001de8 <__aeabi_dsub+0x40>
 8001f66:	4b62      	ldr	r3, [pc, #392]	; (80020f0 <__aeabi_dsub+0x348>)
 8001f68:	429d      	cmp	r5, r3
 8001f6a:	d03a      	beq.n	8001fe2 <__aeabi_dsub+0x23a>
 8001f6c:	2380      	movs	r3, #128	; 0x80
 8001f6e:	4667      	mov	r7, ip
 8001f70:	041b      	lsls	r3, r3, #16
 8001f72:	431f      	orrs	r7, r3
 8001f74:	46bc      	mov	ip, r7
 8001f76:	2e38      	cmp	r6, #56	; 0x38
 8001f78:	dd00      	ble.n	8001f7c <__aeabi_dsub+0x1d4>
 8001f7a:	e0eb      	b.n	8002154 <__aeabi_dsub+0x3ac>
 8001f7c:	2e1f      	cmp	r6, #31
 8001f7e:	dc00      	bgt.n	8001f82 <__aeabi_dsub+0x1da>
 8001f80:	e13a      	b.n	80021f8 <__aeabi_dsub+0x450>
 8001f82:	0033      	movs	r3, r6
 8001f84:	4667      	mov	r7, ip
 8001f86:	3b20      	subs	r3, #32
 8001f88:	40df      	lsrs	r7, r3
 8001f8a:	003b      	movs	r3, r7
 8001f8c:	2e20      	cmp	r6, #32
 8001f8e:	d005      	beq.n	8001f9c <__aeabi_dsub+0x1f4>
 8001f90:	2740      	movs	r7, #64	; 0x40
 8001f92:	1bbf      	subs	r7, r7, r6
 8001f94:	4666      	mov	r6, ip
 8001f96:	40be      	lsls	r6, r7
 8001f98:	4332      	orrs	r2, r6
 8001f9a:	4690      	mov	r8, r2
 8001f9c:	4646      	mov	r6, r8
 8001f9e:	1e72      	subs	r2, r6, #1
 8001fa0:	4196      	sbcs	r6, r2
 8001fa2:	4333      	orrs	r3, r6
 8001fa4:	e0da      	b.n	800215c <__aeabi_dsub+0x3b4>
 8001fa6:	2b00      	cmp	r3, #0
 8001fa8:	d100      	bne.n	8001fac <__aeabi_dsub+0x204>
 8001faa:	e214      	b.n	80023d6 <__aeabi_dsub+0x62e>
 8001fac:	4663      	mov	r3, ip
 8001fae:	4313      	orrs	r3, r2
 8001fb0:	d100      	bne.n	8001fb4 <__aeabi_dsub+0x20c>
 8001fb2:	e168      	b.n	8002286 <__aeabi_dsub+0x4de>
 8001fb4:	2380      	movs	r3, #128	; 0x80
 8001fb6:	074e      	lsls	r6, r1, #29
 8001fb8:	08c0      	lsrs	r0, r0, #3
 8001fba:	08c9      	lsrs	r1, r1, #3
 8001fbc:	031b      	lsls	r3, r3, #12
 8001fbe:	4306      	orrs	r6, r0
 8001fc0:	4219      	tst	r1, r3
 8001fc2:	d008      	beq.n	8001fd6 <__aeabi_dsub+0x22e>
 8001fc4:	4660      	mov	r0, ip
 8001fc6:	08c0      	lsrs	r0, r0, #3
 8001fc8:	4218      	tst	r0, r3
 8001fca:	d104      	bne.n	8001fd6 <__aeabi_dsub+0x22e>
 8001fcc:	4663      	mov	r3, ip
 8001fce:	0001      	movs	r1, r0
 8001fd0:	08d2      	lsrs	r2, r2, #3
 8001fd2:	075e      	lsls	r6, r3, #29
 8001fd4:	4316      	orrs	r6, r2
 8001fd6:	00f3      	lsls	r3, r6, #3
 8001fd8:	4699      	mov	r9, r3
 8001fda:	00c9      	lsls	r1, r1, #3
 8001fdc:	0f72      	lsrs	r2, r6, #29
 8001fde:	4d44      	ldr	r5, [pc, #272]	; (80020f0 <__aeabi_dsub+0x348>)
 8001fe0:	4311      	orrs	r1, r2
 8001fe2:	464b      	mov	r3, r9
 8001fe4:	08de      	lsrs	r6, r3, #3
 8001fe6:	4b42      	ldr	r3, [pc, #264]	; (80020f0 <__aeabi_dsub+0x348>)
 8001fe8:	074f      	lsls	r7, r1, #29
 8001fea:	4337      	orrs	r7, r6
 8001fec:	08ca      	lsrs	r2, r1, #3
 8001fee:	429d      	cmp	r5, r3
 8001ff0:	d100      	bne.n	8001ff4 <__aeabi_dsub+0x24c>
 8001ff2:	e06e      	b.n	80020d2 <__aeabi_dsub+0x32a>
 8001ff4:	0312      	lsls	r2, r2, #12
 8001ff6:	056d      	lsls	r5, r5, #21
 8001ff8:	0b12      	lsrs	r2, r2, #12
 8001ffa:	0d6d      	lsrs	r5, r5, #21
 8001ffc:	2100      	movs	r1, #0
 8001ffe:	0312      	lsls	r2, r2, #12
 8002000:	0b13      	lsrs	r3, r2, #12
 8002002:	0d0a      	lsrs	r2, r1, #20
 8002004:	0512      	lsls	r2, r2, #20
 8002006:	431a      	orrs	r2, r3
 8002008:	4b3b      	ldr	r3, [pc, #236]	; (80020f8 <__aeabi_dsub+0x350>)
 800200a:	052d      	lsls	r5, r5, #20
 800200c:	4013      	ands	r3, r2
 800200e:	432b      	orrs	r3, r5
 8002010:	005b      	lsls	r3, r3, #1
 8002012:	07e4      	lsls	r4, r4, #31
 8002014:	085b      	lsrs	r3, r3, #1
 8002016:	4323      	orrs	r3, r4
 8002018:	0038      	movs	r0, r7
 800201a:	0019      	movs	r1, r3
 800201c:	bc3c      	pop	{r2, r3, r4, r5}
 800201e:	4690      	mov	r8, r2
 8002020:	4699      	mov	r9, r3
 8002022:	46a2      	mov	sl, r4
 8002024:	46ab      	mov	fp, r5
 8002026:	bdf8      	pop	{r3, r4, r5, r6, r7, pc}
 8002028:	4663      	mov	r3, ip
 800202a:	4313      	orrs	r3, r2
 800202c:	d011      	beq.n	8002052 <__aeabi_dsub+0x2aa>
 800202e:	1e73      	subs	r3, r6, #1
 8002030:	2b00      	cmp	r3, #0
 8002032:	d000      	beq.n	8002036 <__aeabi_dsub+0x28e>
 8002034:	e107      	b.n	8002246 <__aeabi_dsub+0x49e>
 8002036:	1886      	adds	r6, r0, r2
 8002038:	4286      	cmp	r6, r0
 800203a:	4180      	sbcs	r0, r0
 800203c:	4461      	add	r1, ip
 800203e:	4240      	negs	r0, r0
 8002040:	1809      	adds	r1, r1, r0
 8002042:	2501      	movs	r5, #1
 8002044:	020b      	lsls	r3, r1, #8
 8002046:	d537      	bpl.n	80020b8 <__aeabi_dsub+0x310>
 8002048:	2502      	movs	r5, #2
 800204a:	e77b      	b.n	8001f44 <__aeabi_dsub+0x19c>
 800204c:	003e      	movs	r6, r7
 800204e:	4661      	mov	r1, ip
 8002050:	4691      	mov	r9, r2
 8002052:	0035      	movs	r5, r6
 8002054:	e7c5      	b.n	8001fe2 <__aeabi_dsub+0x23a>
 8002056:	465c      	mov	r4, fp
 8002058:	2d00      	cmp	r5, #0
 800205a:	d000      	beq.n	800205e <__aeabi_dsub+0x2b6>
 800205c:	e0e1      	b.n	8002222 <__aeabi_dsub+0x47a>
 800205e:	000b      	movs	r3, r1
 8002060:	4303      	orrs	r3, r0
 8002062:	d0f3      	beq.n	800204c <__aeabi_dsub+0x2a4>
 8002064:	1c73      	adds	r3, r6, #1
 8002066:	d100      	bne.n	800206a <__aeabi_dsub+0x2c2>
 8002068:	e1ac      	b.n	80023c4 <__aeabi_dsub+0x61c>
 800206a:	4b21      	ldr	r3, [pc, #132]	; (80020f0 <__aeabi_dsub+0x348>)
 800206c:	429f      	cmp	r7, r3
 800206e:	d100      	bne.n	8002072 <__aeabi_dsub+0x2ca>
 8002070:	e13a      	b.n	80022e8 <__aeabi_dsub+0x540>
 8002072:	43f3      	mvns	r3, r6
 8002074:	2b38      	cmp	r3, #56	; 0x38
 8002076:	dd00      	ble.n	800207a <__aeabi_dsub+0x2d2>
 8002078:	e16f      	b.n	800235a <__aeabi_dsub+0x5b2>
 800207a:	2b1f      	cmp	r3, #31
 800207c:	dd00      	ble.n	8002080 <__aeabi_dsub+0x2d8>
 800207e:	e18c      	b.n	800239a <__aeabi_dsub+0x5f2>
 8002080:	2520      	movs	r5, #32
 8002082:	000e      	movs	r6, r1
 8002084:	1aed      	subs	r5, r5, r3
 8002086:	40ae      	lsls	r6, r5
 8002088:	46b0      	mov	r8, r6
 800208a:	0006      	movs	r6, r0
 800208c:	46aa      	mov	sl, r5
 800208e:	40de      	lsrs	r6, r3
 8002090:	4645      	mov	r5, r8
 8002092:	4335      	orrs	r5, r6
 8002094:	002e      	movs	r6, r5
 8002096:	4655      	mov	r5, sl
 8002098:	40d9      	lsrs	r1, r3
 800209a:	40a8      	lsls	r0, r5
 800209c:	4663      	mov	r3, ip
 800209e:	1e45      	subs	r5, r0, #1
 80020a0:	41a8      	sbcs	r0, r5
 80020a2:	1a5b      	subs	r3, r3, r1
 80020a4:	469c      	mov	ip, r3
 80020a6:	4330      	orrs	r0, r6
 80020a8:	1a16      	subs	r6, r2, r0
 80020aa:	42b2      	cmp	r2, r6
 80020ac:	4192      	sbcs	r2, r2
 80020ae:	4663      	mov	r3, ip
 80020b0:	4252      	negs	r2, r2
 80020b2:	1a99      	subs	r1, r3, r2
 80020b4:	003d      	movs	r5, r7
 80020b6:	e6b4      	b.n	8001e22 <__aeabi_dsub+0x7a>
 80020b8:	2207      	movs	r2, #7
 80020ba:	4032      	ands	r2, r6
 80020bc:	2a00      	cmp	r2, #0
 80020be:	d000      	beq.n	80020c2 <__aeabi_dsub+0x31a>
 80020c0:	e6e4      	b.n	8001e8c <__aeabi_dsub+0xe4>
 80020c2:	4b0b      	ldr	r3, [pc, #44]	; (80020f0 <__aeabi_dsub+0x348>)
 80020c4:	08f6      	lsrs	r6, r6, #3
 80020c6:	074f      	lsls	r7, r1, #29
 80020c8:	4337      	orrs	r7, r6
 80020ca:	08ca      	lsrs	r2, r1, #3
 80020cc:	429d      	cmp	r5, r3
 80020ce:	d000      	beq.n	80020d2 <__aeabi_dsub+0x32a>
 80020d0:	e790      	b.n	8001ff4 <__aeabi_dsub+0x24c>
 80020d2:	003b      	movs	r3, r7
 80020d4:	4313      	orrs	r3, r2
 80020d6:	d100      	bne.n	80020da <__aeabi_dsub+0x332>
 80020d8:	e1a6      	b.n	8002428 <__aeabi_dsub+0x680>
 80020da:	2380      	movs	r3, #128	; 0x80
 80020dc:	031b      	lsls	r3, r3, #12
 80020de:	431a      	orrs	r2, r3
 80020e0:	0312      	lsls	r2, r2, #12
 80020e2:	0b12      	lsrs	r2, r2, #12
 80020e4:	4d02      	ldr	r5, [pc, #8]	; (80020f0 <__aeabi_dsub+0x348>)
 80020e6:	e789      	b.n	8001ffc <__aeabi_dsub+0x254>
 80020e8:	0015      	movs	r5, r2
 80020ea:	2200      	movs	r2, #0
 80020ec:	2700      	movs	r7, #0
 80020ee:	e785      	b.n	8001ffc <__aeabi_dsub+0x254>
 80020f0:	000007ff 	.word	0x000007ff
 80020f4:	ff7fffff 	.word	0xff7fffff
 80020f8:	800fffff 	.word	0x800fffff
 80020fc:	2e00      	cmp	r6, #0
 80020fe:	d000      	beq.n	8002102 <__aeabi_dsub+0x35a>
 8002100:	e0c7      	b.n	8002292 <__aeabi_dsub+0x4ea>
 8002102:	1c6b      	adds	r3, r5, #1
 8002104:	055e      	lsls	r6, r3, #21
 8002106:	0d76      	lsrs	r6, r6, #21
 8002108:	2e01      	cmp	r6, #1
 800210a:	dc00      	bgt.n	800210e <__aeabi_dsub+0x366>
 800210c:	e0f0      	b.n	80022f0 <__aeabi_dsub+0x548>
 800210e:	4dc8      	ldr	r5, [pc, #800]	; (8002430 <__aeabi_dsub+0x688>)
 8002110:	42ab      	cmp	r3, r5
 8002112:	d100      	bne.n	8002116 <__aeabi_dsub+0x36e>
 8002114:	e0b9      	b.n	800228a <__aeabi_dsub+0x4e2>
 8002116:	1885      	adds	r5, r0, r2
 8002118:	000a      	movs	r2, r1
 800211a:	4285      	cmp	r5, r0
 800211c:	4189      	sbcs	r1, r1
 800211e:	4462      	add	r2, ip
 8002120:	4249      	negs	r1, r1
 8002122:	1851      	adds	r1, r2, r1
 8002124:	2207      	movs	r2, #7
 8002126:	07ce      	lsls	r6, r1, #31
 8002128:	086d      	lsrs	r5, r5, #1
 800212a:	432e      	orrs	r6, r5
 800212c:	0849      	lsrs	r1, r1, #1
 800212e:	4032      	ands	r2, r6
 8002130:	001d      	movs	r5, r3
 8002132:	e6a9      	b.n	8001e88 <__aeabi_dsub+0xe0>
 8002134:	49bf      	ldr	r1, [pc, #764]	; (8002434 <__aeabi_dsub+0x68c>)
 8002136:	1aed      	subs	r5, r5, r3
 8002138:	4011      	ands	r1, r2
 800213a:	2207      	movs	r2, #7
 800213c:	4032      	ands	r2, r6
 800213e:	e6a3      	b.n	8001e88 <__aeabi_dsub+0xe0>
 8002140:	0032      	movs	r2, r6
 8002142:	3828      	subs	r0, #40	; 0x28
 8002144:	4082      	lsls	r2, r0
 8002146:	2600      	movs	r6, #0
 8002148:	e686      	b.n	8001e58 <__aeabi_dsub+0xb0>
 800214a:	0030      	movs	r0, r6
 800214c:	f000 fa68 	bl	8002620 <__clzsi2>
 8002150:	3020      	adds	r0, #32
 8002152:	e673      	b.n	8001e3c <__aeabi_dsub+0x94>
 8002154:	4663      	mov	r3, ip
 8002156:	4313      	orrs	r3, r2
 8002158:	1e5a      	subs	r2, r3, #1
 800215a:	4193      	sbcs	r3, r2
 800215c:	1ac6      	subs	r6, r0, r3
 800215e:	42b0      	cmp	r0, r6
 8002160:	4180      	sbcs	r0, r0
 8002162:	4240      	negs	r0, r0
 8002164:	1a09      	subs	r1, r1, r0
 8002166:	e65c      	b.n	8001e22 <__aeabi_dsub+0x7a>
 8002168:	000e      	movs	r6, r1
 800216a:	4667      	mov	r7, ip
 800216c:	4306      	orrs	r6, r0
 800216e:	4317      	orrs	r7, r2
 8002170:	2d00      	cmp	r5, #0
 8002172:	d15e      	bne.n	8002232 <__aeabi_dsub+0x48a>
 8002174:	2e00      	cmp	r6, #0
 8002176:	d000      	beq.n	800217a <__aeabi_dsub+0x3d2>
 8002178:	e0f3      	b.n	8002362 <__aeabi_dsub+0x5ba>
 800217a:	2f00      	cmp	r7, #0
 800217c:	d100      	bne.n	8002180 <__aeabi_dsub+0x3d8>
 800217e:	e11e      	b.n	80023be <__aeabi_dsub+0x616>
 8002180:	465c      	mov	r4, fp
 8002182:	4661      	mov	r1, ip
 8002184:	4691      	mov	r9, r2
 8002186:	e72c      	b.n	8001fe2 <__aeabi_dsub+0x23a>
 8002188:	4fa9      	ldr	r7, [pc, #676]	; (8002430 <__aeabi_dsub+0x688>)
 800218a:	42be      	cmp	r6, r7
 800218c:	d07b      	beq.n	8002286 <__aeabi_dsub+0x4de>
 800218e:	001e      	movs	r6, r3
 8002190:	e6f1      	b.n	8001f76 <__aeabi_dsub+0x1ce>
 8002192:	0010      	movs	r0, r2
 8002194:	3d1f      	subs	r5, #31
 8002196:	40e8      	lsrs	r0, r5
 8002198:	2b20      	cmp	r3, #32
 800219a:	d003      	beq.n	80021a4 <__aeabi_dsub+0x3fc>
 800219c:	2140      	movs	r1, #64	; 0x40
 800219e:	1acb      	subs	r3, r1, r3
 80021a0:	409a      	lsls	r2, r3
 80021a2:	4316      	orrs	r6, r2
 80021a4:	1e73      	subs	r3, r6, #1
 80021a6:	419e      	sbcs	r6, r3
 80021a8:	2207      	movs	r2, #7
 80021aa:	4306      	orrs	r6, r0
 80021ac:	4032      	ands	r2, r6
 80021ae:	2100      	movs	r1, #0
 80021b0:	2500      	movs	r5, #0
 80021b2:	e783      	b.n	80020bc <__aeabi_dsub+0x314>
 80021b4:	1a16      	subs	r6, r2, r0
 80021b6:	4663      	mov	r3, ip
 80021b8:	42b2      	cmp	r2, r6
 80021ba:	4180      	sbcs	r0, r0
 80021bc:	1a59      	subs	r1, r3, r1
 80021be:	4240      	negs	r0, r0
 80021c0:	1a0b      	subs	r3, r1, r0
 80021c2:	4698      	mov	r8, r3
 80021c4:	465c      	mov	r4, fp
 80021c6:	e632      	b.n	8001e2e <__aeabi_dsub+0x86>
 80021c8:	2e1f      	cmp	r6, #31
 80021ca:	dd00      	ble.n	80021ce <__aeabi_dsub+0x426>
 80021cc:	e0ab      	b.n	8002326 <__aeabi_dsub+0x57e>
 80021ce:	2720      	movs	r7, #32
 80021d0:	1bbb      	subs	r3, r7, r6
 80021d2:	469a      	mov	sl, r3
 80021d4:	4663      	mov	r3, ip
 80021d6:	4657      	mov	r7, sl
 80021d8:	40bb      	lsls	r3, r7
 80021da:	4699      	mov	r9, r3
 80021dc:	0013      	movs	r3, r2
 80021de:	464f      	mov	r7, r9
 80021e0:	40f3      	lsrs	r3, r6
 80021e2:	431f      	orrs	r7, r3
 80021e4:	003b      	movs	r3, r7
 80021e6:	4657      	mov	r7, sl
 80021e8:	40ba      	lsls	r2, r7
 80021ea:	1e57      	subs	r7, r2, #1
 80021ec:	41ba      	sbcs	r2, r7
 80021ee:	4313      	orrs	r3, r2
 80021f0:	4662      	mov	r2, ip
 80021f2:	40f2      	lsrs	r2, r6
 80021f4:	1889      	adds	r1, r1, r2
 80021f6:	e698      	b.n	8001f2a <__aeabi_dsub+0x182>
 80021f8:	2720      	movs	r7, #32
 80021fa:	1bbb      	subs	r3, r7, r6
 80021fc:	469a      	mov	sl, r3
 80021fe:	4663      	mov	r3, ip
 8002200:	4657      	mov	r7, sl
 8002202:	40bb      	lsls	r3, r7
 8002204:	4699      	mov	r9, r3
 8002206:	0013      	movs	r3, r2
 8002208:	464f      	mov	r7, r9
 800220a:	40f3      	lsrs	r3, r6
 800220c:	431f      	orrs	r7, r3
 800220e:	003b      	movs	r3, r7
 8002210:	4657      	mov	r7, sl
 8002212:	40ba      	lsls	r2, r7
 8002214:	1e57      	subs	r7, r2, #1
 8002216:	41ba      	sbcs	r2, r7
 8002218:	4313      	orrs	r3, r2
 800221a:	4662      	mov	r2, ip
 800221c:	40f2      	lsrs	r2, r6
 800221e:	1a89      	subs	r1, r1, r2
 8002220:	e79c      	b.n	800215c <__aeabi_dsub+0x3b4>
 8002222:	4b83      	ldr	r3, [pc, #524]	; (8002430 <__aeabi_dsub+0x688>)
 8002224:	429f      	cmp	r7, r3
 8002226:	d05f      	beq.n	80022e8 <__aeabi_dsub+0x540>
 8002228:	2580      	movs	r5, #128	; 0x80
 800222a:	042d      	lsls	r5, r5, #16
 800222c:	4273      	negs	r3, r6
 800222e:	4329      	orrs	r1, r5
 8002230:	e720      	b.n	8002074 <__aeabi_dsub+0x2cc>
 8002232:	2e00      	cmp	r6, #0
 8002234:	d10c      	bne.n	8002250 <__aeabi_dsub+0x4a8>
 8002236:	2f00      	cmp	r7, #0
 8002238:	d100      	bne.n	800223c <__aeabi_dsub+0x494>
 800223a:	e0d0      	b.n	80023de <__aeabi_dsub+0x636>
 800223c:	465c      	mov	r4, fp
 800223e:	4661      	mov	r1, ip
 8002240:	4691      	mov	r9, r2
 8002242:	4d7b      	ldr	r5, [pc, #492]	; (8002430 <__aeabi_dsub+0x688>)
 8002244:	e6cd      	b.n	8001fe2 <__aeabi_dsub+0x23a>
 8002246:	4f7a      	ldr	r7, [pc, #488]	; (8002430 <__aeabi_dsub+0x688>)
 8002248:	42be      	cmp	r6, r7
 800224a:	d01c      	beq.n	8002286 <__aeabi_dsub+0x4de>
 800224c:	001e      	movs	r6, r3
 800224e:	e665      	b.n	8001f1c <__aeabi_dsub+0x174>
 8002250:	2f00      	cmp	r7, #0
 8002252:	d018      	beq.n	8002286 <__aeabi_dsub+0x4de>
 8002254:	08c0      	lsrs	r0, r0, #3
 8002256:	074e      	lsls	r6, r1, #29
 8002258:	4306      	orrs	r6, r0
 800225a:	2080      	movs	r0, #128	; 0x80
 800225c:	08c9      	lsrs	r1, r1, #3
 800225e:	0300      	lsls	r0, r0, #12
 8002260:	4201      	tst	r1, r0
 8002262:	d008      	beq.n	8002276 <__aeabi_dsub+0x4ce>
 8002264:	4663      	mov	r3, ip
 8002266:	08dc      	lsrs	r4, r3, #3
 8002268:	4204      	tst	r4, r0
 800226a:	d104      	bne.n	8002276 <__aeabi_dsub+0x4ce>
 800226c:	0021      	movs	r1, r4
 800226e:	46da      	mov	sl, fp
 8002270:	08d2      	lsrs	r2, r2, #3
 8002272:	075e      	lsls	r6, r3, #29
 8002274:	4316      	orrs	r6, r2
 8002276:	00f3      	lsls	r3, r6, #3
 8002278:	4699      	mov	r9, r3
 800227a:	2401      	movs	r4, #1
 800227c:	4653      	mov	r3, sl
 800227e:	00c9      	lsls	r1, r1, #3
 8002280:	0f72      	lsrs	r2, r6, #29
 8002282:	4311      	orrs	r1, r2
 8002284:	401c      	ands	r4, r3
 8002286:	4d6a      	ldr	r5, [pc, #424]	; (8002430 <__aeabi_dsub+0x688>)
 8002288:	e6ab      	b.n	8001fe2 <__aeabi_dsub+0x23a>
 800228a:	001d      	movs	r5, r3
 800228c:	2200      	movs	r2, #0
 800228e:	2700      	movs	r7, #0
 8002290:	e6b4      	b.n	8001ffc <__aeabi_dsub+0x254>
 8002292:	2d00      	cmp	r5, #0
 8002294:	d159      	bne.n	800234a <__aeabi_dsub+0x5a2>
 8002296:	000b      	movs	r3, r1
 8002298:	4303      	orrs	r3, r0
 800229a:	d100      	bne.n	800229e <__aeabi_dsub+0x4f6>
 800229c:	e6d6      	b.n	800204c <__aeabi_dsub+0x2a4>
 800229e:	1c73      	adds	r3, r6, #1
 80022a0:	d100      	bne.n	80022a4 <__aeabi_dsub+0x4fc>
 80022a2:	e0b2      	b.n	800240a <__aeabi_dsub+0x662>
 80022a4:	4b62      	ldr	r3, [pc, #392]	; (8002430 <__aeabi_dsub+0x688>)
 80022a6:	429f      	cmp	r7, r3
 80022a8:	d01e      	beq.n	80022e8 <__aeabi_dsub+0x540>
 80022aa:	43f3      	mvns	r3, r6
 80022ac:	2b38      	cmp	r3, #56	; 0x38
 80022ae:	dc6f      	bgt.n	8002390 <__aeabi_dsub+0x5e8>
 80022b0:	2b1f      	cmp	r3, #31
 80022b2:	dd00      	ble.n	80022b6 <__aeabi_dsub+0x50e>
 80022b4:	e097      	b.n	80023e6 <__aeabi_dsub+0x63e>
 80022b6:	2520      	movs	r5, #32
 80022b8:	000e      	movs	r6, r1
 80022ba:	1aed      	subs	r5, r5, r3
 80022bc:	40ae      	lsls	r6, r5
 80022be:	46b0      	mov	r8, r6
 80022c0:	0006      	movs	r6, r0
 80022c2:	46aa      	mov	sl, r5
 80022c4:	40de      	lsrs	r6, r3
 80022c6:	4645      	mov	r5, r8
 80022c8:	4335      	orrs	r5, r6
 80022ca:	002e      	movs	r6, r5
 80022cc:	4655      	mov	r5, sl
 80022ce:	40a8      	lsls	r0, r5
 80022d0:	40d9      	lsrs	r1, r3
 80022d2:	1e45      	subs	r5, r0, #1
 80022d4:	41a8      	sbcs	r0, r5
 80022d6:	448c      	add	ip, r1
 80022d8:	4306      	orrs	r6, r0
 80022da:	18b6      	adds	r6, r6, r2
 80022dc:	4296      	cmp	r6, r2
 80022de:	4192      	sbcs	r2, r2
 80022e0:	4251      	negs	r1, r2
 80022e2:	4461      	add	r1, ip
 80022e4:	003d      	movs	r5, r7
 80022e6:	e625      	b.n	8001f34 <__aeabi_dsub+0x18c>
 80022e8:	003d      	movs	r5, r7
 80022ea:	4661      	mov	r1, ip
 80022ec:	4691      	mov	r9, r2
 80022ee:	e678      	b.n	8001fe2 <__aeabi_dsub+0x23a>
 80022f0:	000b      	movs	r3, r1
 80022f2:	4303      	orrs	r3, r0
 80022f4:	2d00      	cmp	r5, #0
 80022f6:	d000      	beq.n	80022fa <__aeabi_dsub+0x552>
 80022f8:	e655      	b.n	8001fa6 <__aeabi_dsub+0x1fe>
 80022fa:	2b00      	cmp	r3, #0
 80022fc:	d0f5      	beq.n	80022ea <__aeabi_dsub+0x542>
 80022fe:	4663      	mov	r3, ip
 8002300:	4313      	orrs	r3, r2
 8002302:	d100      	bne.n	8002306 <__aeabi_dsub+0x55e>
 8002304:	e66d      	b.n	8001fe2 <__aeabi_dsub+0x23a>
 8002306:	1886      	adds	r6, r0, r2
 8002308:	4286      	cmp	r6, r0
 800230a:	4180      	sbcs	r0, r0
 800230c:	4461      	add	r1, ip
 800230e:	4240      	negs	r0, r0
 8002310:	1809      	adds	r1, r1, r0
 8002312:	2200      	movs	r2, #0
 8002314:	020b      	lsls	r3, r1, #8
 8002316:	d400      	bmi.n	800231a <__aeabi_dsub+0x572>
 8002318:	e6d0      	b.n	80020bc <__aeabi_dsub+0x314>
 800231a:	4b46      	ldr	r3, [pc, #280]	; (8002434 <__aeabi_dsub+0x68c>)
 800231c:	3501      	adds	r5, #1
 800231e:	4019      	ands	r1, r3
 8002320:	e5b2      	b.n	8001e88 <__aeabi_dsub+0xe0>
 8002322:	46b1      	mov	r9, r6
 8002324:	e65d      	b.n	8001fe2 <__aeabi_dsub+0x23a>
 8002326:	0033      	movs	r3, r6
 8002328:	4667      	mov	r7, ip
 800232a:	3b20      	subs	r3, #32
 800232c:	40df      	lsrs	r7, r3
 800232e:	003b      	movs	r3, r7
 8002330:	2e20      	cmp	r6, #32
 8002332:	d005      	beq.n	8002340 <__aeabi_dsub+0x598>
 8002334:	2740      	movs	r7, #64	; 0x40
 8002336:	1bbf      	subs	r7, r7, r6
 8002338:	4666      	mov	r6, ip
 800233a:	40be      	lsls	r6, r7
 800233c:	4332      	orrs	r2, r6
 800233e:	4690      	mov	r8, r2
 8002340:	4646      	mov	r6, r8
 8002342:	1e72      	subs	r2, r6, #1
 8002344:	4196      	sbcs	r6, r2
 8002346:	4333      	orrs	r3, r6
 8002348:	e5ef      	b.n	8001f2a <__aeabi_dsub+0x182>
 800234a:	4b39      	ldr	r3, [pc, #228]	; (8002430 <__aeabi_dsub+0x688>)
 800234c:	429f      	cmp	r7, r3
 800234e:	d0cb      	beq.n	80022e8 <__aeabi_dsub+0x540>
 8002350:	2580      	movs	r5, #128	; 0x80
 8002352:	042d      	lsls	r5, r5, #16
 8002354:	4273      	negs	r3, r6
 8002356:	4329      	orrs	r1, r5
 8002358:	e7a8      	b.n	80022ac <__aeabi_dsub+0x504>
 800235a:	4308      	orrs	r0, r1
 800235c:	1e41      	subs	r1, r0, #1
 800235e:	4188      	sbcs	r0, r1
 8002360:	e6a2      	b.n	80020a8 <__aeabi_dsub+0x300>
 8002362:	2f00      	cmp	r7, #0
 8002364:	d100      	bne.n	8002368 <__aeabi_dsub+0x5c0>
 8002366:	e63c      	b.n	8001fe2 <__aeabi_dsub+0x23a>
 8002368:	4663      	mov	r3, ip
 800236a:	1a86      	subs	r6, r0, r2
 800236c:	1acf      	subs	r7, r1, r3
 800236e:	42b0      	cmp	r0, r6
 8002370:	419b      	sbcs	r3, r3
 8002372:	425b      	negs	r3, r3
 8002374:	1afb      	subs	r3, r7, r3
 8002376:	4698      	mov	r8, r3
 8002378:	021b      	lsls	r3, r3, #8
 800237a:	d54e      	bpl.n	800241a <__aeabi_dsub+0x672>
 800237c:	1a16      	subs	r6, r2, r0
 800237e:	4663      	mov	r3, ip
 8002380:	42b2      	cmp	r2, r6
 8002382:	4192      	sbcs	r2, r2
 8002384:	1a59      	subs	r1, r3, r1
 8002386:	4252      	negs	r2, r2
 8002388:	1a89      	subs	r1, r1, r2
 800238a:	465c      	mov	r4, fp
 800238c:	2200      	movs	r2, #0
 800238e:	e57b      	b.n	8001e88 <__aeabi_dsub+0xe0>
 8002390:	4301      	orrs	r1, r0
 8002392:	000e      	movs	r6, r1
 8002394:	1e71      	subs	r1, r6, #1
 8002396:	418e      	sbcs	r6, r1
 8002398:	e79f      	b.n	80022da <__aeabi_dsub+0x532>
 800239a:	001d      	movs	r5, r3
 800239c:	000e      	movs	r6, r1
 800239e:	3d20      	subs	r5, #32
 80023a0:	40ee      	lsrs	r6, r5
 80023a2:	46b0      	mov	r8, r6
 80023a4:	2b20      	cmp	r3, #32
 80023a6:	d004      	beq.n	80023b2 <__aeabi_dsub+0x60a>
 80023a8:	2540      	movs	r5, #64	; 0x40
 80023aa:	1aeb      	subs	r3, r5, r3
 80023ac:	4099      	lsls	r1, r3
 80023ae:	4308      	orrs	r0, r1
 80023b0:	4681      	mov	r9, r0
 80023b2:	4648      	mov	r0, r9
 80023b4:	4643      	mov	r3, r8
 80023b6:	1e41      	subs	r1, r0, #1
 80023b8:	4188      	sbcs	r0, r1
 80023ba:	4318      	orrs	r0, r3
 80023bc:	e674      	b.n	80020a8 <__aeabi_dsub+0x300>
 80023be:	2200      	movs	r2, #0
 80023c0:	2400      	movs	r4, #0
 80023c2:	e617      	b.n	8001ff4 <__aeabi_dsub+0x24c>
 80023c4:	1a16      	subs	r6, r2, r0
 80023c6:	4663      	mov	r3, ip
 80023c8:	42b2      	cmp	r2, r6
 80023ca:	4192      	sbcs	r2, r2
 80023cc:	1a59      	subs	r1, r3, r1
 80023ce:	4252      	negs	r2, r2
 80023d0:	1a89      	subs	r1, r1, r2
 80023d2:	003d      	movs	r5, r7
 80023d4:	e525      	b.n	8001e22 <__aeabi_dsub+0x7a>
 80023d6:	4661      	mov	r1, ip
 80023d8:	4691      	mov	r9, r2
 80023da:	4d15      	ldr	r5, [pc, #84]	; (8002430 <__aeabi_dsub+0x688>)
 80023dc:	e601      	b.n	8001fe2 <__aeabi_dsub+0x23a>
 80023de:	2280      	movs	r2, #128	; 0x80
 80023e0:	2400      	movs	r4, #0
 80023e2:	0312      	lsls	r2, r2, #12
 80023e4:	e679      	b.n	80020da <__aeabi_dsub+0x332>
 80023e6:	001d      	movs	r5, r3
 80023e8:	000e      	movs	r6, r1
 80023ea:	3d20      	subs	r5, #32
 80023ec:	40ee      	lsrs	r6, r5
 80023ee:	46b0      	mov	r8, r6
 80023f0:	2b20      	cmp	r3, #32
 80023f2:	d004      	beq.n	80023fe <__aeabi_dsub+0x656>
 80023f4:	2540      	movs	r5, #64	; 0x40
 80023f6:	1aeb      	subs	r3, r5, r3
 80023f8:	4099      	lsls	r1, r3
 80023fa:	4308      	orrs	r0, r1
 80023fc:	4681      	mov	r9, r0
 80023fe:	464e      	mov	r6, r9
 8002400:	4643      	mov	r3, r8
 8002402:	1e71      	subs	r1, r6, #1
 8002404:	418e      	sbcs	r6, r1
 8002406:	431e      	orrs	r6, r3
 8002408:	e767      	b.n	80022da <__aeabi_dsub+0x532>
 800240a:	1886      	adds	r6, r0, r2
 800240c:	4296      	cmp	r6, r2
 800240e:	419b      	sbcs	r3, r3
 8002410:	4461      	add	r1, ip
 8002412:	425b      	negs	r3, r3
 8002414:	18c9      	adds	r1, r1, r3
 8002416:	003d      	movs	r5, r7
 8002418:	e58c      	b.n	8001f34 <__aeabi_dsub+0x18c>
 800241a:	4647      	mov	r7, r8
 800241c:	4337      	orrs	r7, r6
 800241e:	d0ce      	beq.n	80023be <__aeabi_dsub+0x616>
 8002420:	2207      	movs	r2, #7
 8002422:	4641      	mov	r1, r8
 8002424:	4032      	ands	r2, r6
 8002426:	e649      	b.n	80020bc <__aeabi_dsub+0x314>
 8002428:	2700      	movs	r7, #0
 800242a:	003a      	movs	r2, r7
 800242c:	e5e6      	b.n	8001ffc <__aeabi_dsub+0x254>
 800242e:	46c0      	nop			; (mov r8, r8)
 8002430:	000007ff 	.word	0x000007ff
 8002434:	ff7fffff 	.word	0xff7fffff

08002438 <__aeabi_d2iz>:
 8002438:	b530      	push	{r4, r5, lr}
 800243a:	4d14      	ldr	r5, [pc, #80]	; (800248c <__aeabi_d2iz+0x54>)
 800243c:	030a      	lsls	r2, r1, #12
 800243e:	004b      	lsls	r3, r1, #1
 8002440:	0b12      	lsrs	r2, r2, #12
 8002442:	0d5b      	lsrs	r3, r3, #21
 8002444:	0fc9      	lsrs	r1, r1, #31
 8002446:	2400      	movs	r4, #0
 8002448:	42ab      	cmp	r3, r5
 800244a:	dd11      	ble.n	8002470 <__aeabi_d2iz+0x38>
 800244c:	4c10      	ldr	r4, [pc, #64]	; (8002490 <__aeabi_d2iz+0x58>)
 800244e:	42a3      	cmp	r3, r4
 8002450:	dc10      	bgt.n	8002474 <__aeabi_d2iz+0x3c>
 8002452:	2480      	movs	r4, #128	; 0x80
 8002454:	0364      	lsls	r4, r4, #13
 8002456:	4322      	orrs	r2, r4
 8002458:	4c0e      	ldr	r4, [pc, #56]	; (8002494 <__aeabi_d2iz+0x5c>)
 800245a:	1ae4      	subs	r4, r4, r3
 800245c:	2c1f      	cmp	r4, #31
 800245e:	dd0c      	ble.n	800247a <__aeabi_d2iz+0x42>
 8002460:	480d      	ldr	r0, [pc, #52]	; (8002498 <__aeabi_d2iz+0x60>)
 8002462:	1ac3      	subs	r3, r0, r3
 8002464:	40da      	lsrs	r2, r3
 8002466:	0013      	movs	r3, r2
 8002468:	425c      	negs	r4, r3
 800246a:	2900      	cmp	r1, #0
 800246c:	d100      	bne.n	8002470 <__aeabi_d2iz+0x38>
 800246e:	001c      	movs	r4, r3
 8002470:	0020      	movs	r0, r4
 8002472:	bd30      	pop	{r4, r5, pc}
 8002474:	4b09      	ldr	r3, [pc, #36]	; (800249c <__aeabi_d2iz+0x64>)
 8002476:	18cc      	adds	r4, r1, r3
 8002478:	e7fa      	b.n	8002470 <__aeabi_d2iz+0x38>
 800247a:	4d09      	ldr	r5, [pc, #36]	; (80024a0 <__aeabi_d2iz+0x68>)
 800247c:	40e0      	lsrs	r0, r4
 800247e:	46ac      	mov	ip, r5
 8002480:	4463      	add	r3, ip
 8002482:	409a      	lsls	r2, r3
 8002484:	0013      	movs	r3, r2
 8002486:	4303      	orrs	r3, r0
 8002488:	e7ee      	b.n	8002468 <__aeabi_d2iz+0x30>
 800248a:	46c0      	nop			; (mov r8, r8)
 800248c:	000003fe 	.word	0x000003fe
 8002490:	0000041d 	.word	0x0000041d
 8002494:	00000433 	.word	0x00000433
 8002498:	00000413 	.word	0x00000413
 800249c:	7fffffff 	.word	0x7fffffff
 80024a0:	fffffbed 	.word	0xfffffbed

080024a4 <__aeabi_i2d>:
 80024a4:	b570      	push	{r4, r5, r6, lr}
 80024a6:	2800      	cmp	r0, #0
 80024a8:	d02d      	beq.n	8002506 <__aeabi_i2d+0x62>
 80024aa:	17c3      	asrs	r3, r0, #31
 80024ac:	18c5      	adds	r5, r0, r3
 80024ae:	405d      	eors	r5, r3
 80024b0:	0fc4      	lsrs	r4, r0, #31
 80024b2:	0028      	movs	r0, r5
 80024b4:	f000 f8b4 	bl	8002620 <__clzsi2>
 80024b8:	4b15      	ldr	r3, [pc, #84]	; (8002510 <__aeabi_i2d+0x6c>)
 80024ba:	1a1b      	subs	r3, r3, r0
 80024bc:	055b      	lsls	r3, r3, #21
 80024be:	0d5b      	lsrs	r3, r3, #21
 80024c0:	280a      	cmp	r0, #10
 80024c2:	dd15      	ble.n	80024f0 <__aeabi_i2d+0x4c>
 80024c4:	380b      	subs	r0, #11
 80024c6:	4085      	lsls	r5, r0
 80024c8:	2200      	movs	r2, #0
 80024ca:	032d      	lsls	r5, r5, #12
 80024cc:	0b2d      	lsrs	r5, r5, #12
 80024ce:	2100      	movs	r1, #0
 80024d0:	0010      	movs	r0, r2
 80024d2:	032d      	lsls	r5, r5, #12
 80024d4:	0d0a      	lsrs	r2, r1, #20
 80024d6:	0b2d      	lsrs	r5, r5, #12
 80024d8:	0512      	lsls	r2, r2, #20
 80024da:	432a      	orrs	r2, r5
 80024dc:	4d0d      	ldr	r5, [pc, #52]	; (8002514 <__aeabi_i2d+0x70>)
 80024de:	051b      	lsls	r3, r3, #20
 80024e0:	402a      	ands	r2, r5
 80024e2:	4313      	orrs	r3, r2
 80024e4:	005b      	lsls	r3, r3, #1
 80024e6:	07e4      	lsls	r4, r4, #31
 80024e8:	085b      	lsrs	r3, r3, #1
 80024ea:	4323      	orrs	r3, r4
 80024ec:	0019      	movs	r1, r3
 80024ee:	bd70      	pop	{r4, r5, r6, pc}
 80024f0:	0002      	movs	r2, r0
 80024f2:	0029      	movs	r1, r5
 80024f4:	3215      	adds	r2, #21
 80024f6:	4091      	lsls	r1, r2
 80024f8:	000a      	movs	r2, r1
 80024fa:	210b      	movs	r1, #11
 80024fc:	1a08      	subs	r0, r1, r0
 80024fe:	40c5      	lsrs	r5, r0
 8002500:	032d      	lsls	r5, r5, #12
 8002502:	0b2d      	lsrs	r5, r5, #12
 8002504:	e7e3      	b.n	80024ce <__aeabi_i2d+0x2a>
 8002506:	2400      	movs	r4, #0
 8002508:	2300      	movs	r3, #0
 800250a:	2500      	movs	r5, #0
 800250c:	2200      	movs	r2, #0
 800250e:	e7de      	b.n	80024ce <__aeabi_i2d+0x2a>
 8002510:	0000041e 	.word	0x0000041e
 8002514:	800fffff 	.word	0x800fffff

08002518 <__aeabi_ui2d>:
 8002518:	b510      	push	{r4, lr}
 800251a:	1e04      	subs	r4, r0, #0
 800251c:	d025      	beq.n	800256a <__aeabi_ui2d+0x52>
 800251e:	f000 f87f 	bl	8002620 <__clzsi2>
 8002522:	4b14      	ldr	r3, [pc, #80]	; (8002574 <__aeabi_ui2d+0x5c>)
 8002524:	1a1b      	subs	r3, r3, r0
 8002526:	055b      	lsls	r3, r3, #21
 8002528:	0d5b      	lsrs	r3, r3, #21
 800252a:	280a      	cmp	r0, #10
 800252c:	dd12      	ble.n	8002554 <__aeabi_ui2d+0x3c>
 800252e:	380b      	subs	r0, #11
 8002530:	4084      	lsls	r4, r0
 8002532:	2200      	movs	r2, #0
 8002534:	0324      	lsls	r4, r4, #12
 8002536:	0b24      	lsrs	r4, r4, #12
 8002538:	2100      	movs	r1, #0
 800253a:	0010      	movs	r0, r2
 800253c:	0324      	lsls	r4, r4, #12
 800253e:	0d0a      	lsrs	r2, r1, #20
 8002540:	0b24      	lsrs	r4, r4, #12
 8002542:	0512      	lsls	r2, r2, #20
 8002544:	4322      	orrs	r2, r4
 8002546:	4c0c      	ldr	r4, [pc, #48]	; (8002578 <__aeabi_ui2d+0x60>)
 8002548:	051b      	lsls	r3, r3, #20
 800254a:	4022      	ands	r2, r4
 800254c:	4313      	orrs	r3, r2
 800254e:	005b      	lsls	r3, r3, #1
 8002550:	0859      	lsrs	r1, r3, #1
 8002552:	bd10      	pop	{r4, pc}
 8002554:	0002      	movs	r2, r0
 8002556:	0021      	movs	r1, r4
 8002558:	3215      	adds	r2, #21
 800255a:	4091      	lsls	r1, r2
 800255c:	000a      	movs	r2, r1
 800255e:	210b      	movs	r1, #11
 8002560:	1a08      	subs	r0, r1, r0
 8002562:	40c4      	lsrs	r4, r0
 8002564:	0324      	lsls	r4, r4, #12
 8002566:	0b24      	lsrs	r4, r4, #12
 8002568:	e7e6      	b.n	8002538 <__aeabi_ui2d+0x20>
 800256a:	2300      	movs	r3, #0
 800256c:	2400      	movs	r4, #0
 800256e:	2200      	movs	r2, #0
 8002570:	e7e2      	b.n	8002538 <__aeabi_ui2d+0x20>
 8002572:	46c0      	nop			; (mov r8, r8)
 8002574:	0000041e 	.word	0x0000041e
 8002578:	800fffff 	.word	0x800fffff

0800257c <__aeabi_f2d>:
 800257c:	0041      	lsls	r1, r0, #1
 800257e:	0e09      	lsrs	r1, r1, #24
 8002580:	1c4b      	adds	r3, r1, #1
 8002582:	b570      	push	{r4, r5, r6, lr}
 8002584:	b2db      	uxtb	r3, r3
 8002586:	0246      	lsls	r6, r0, #9
 8002588:	0a75      	lsrs	r5, r6, #9
 800258a:	0fc4      	lsrs	r4, r0, #31
 800258c:	2b01      	cmp	r3, #1
 800258e:	dd14      	ble.n	80025ba <__aeabi_f2d+0x3e>
 8002590:	23e0      	movs	r3, #224	; 0xe0
 8002592:	009b      	lsls	r3, r3, #2
 8002594:	076d      	lsls	r5, r5, #29
 8002596:	0b36      	lsrs	r6, r6, #12
 8002598:	18cb      	adds	r3, r1, r3
 800259a:	2100      	movs	r1, #0
 800259c:	0d0a      	lsrs	r2, r1, #20
 800259e:	0028      	movs	r0, r5
 80025a0:	0512      	lsls	r2, r2, #20
 80025a2:	4d1c      	ldr	r5, [pc, #112]	; (8002614 <__aeabi_f2d+0x98>)
 80025a4:	4332      	orrs	r2, r6
 80025a6:	055b      	lsls	r3, r3, #21
 80025a8:	402a      	ands	r2, r5
 80025aa:	085b      	lsrs	r3, r3, #1
 80025ac:	4313      	orrs	r3, r2
 80025ae:	005b      	lsls	r3, r3, #1
 80025b0:	07e4      	lsls	r4, r4, #31
 80025b2:	085b      	lsrs	r3, r3, #1
 80025b4:	4323      	orrs	r3, r4
 80025b6:	0019      	movs	r1, r3
 80025b8:	bd70      	pop	{r4, r5, r6, pc}
 80025ba:	2900      	cmp	r1, #0
 80025bc:	d114      	bne.n	80025e8 <__aeabi_f2d+0x6c>
 80025be:	2d00      	cmp	r5, #0
 80025c0:	d01e      	beq.n	8002600 <__aeabi_f2d+0x84>
 80025c2:	0028      	movs	r0, r5
 80025c4:	f000 f82c 	bl	8002620 <__clzsi2>
 80025c8:	280a      	cmp	r0, #10
 80025ca:	dc1c      	bgt.n	8002606 <__aeabi_f2d+0x8a>
 80025cc:	230b      	movs	r3, #11
 80025ce:	002a      	movs	r2, r5
 80025d0:	1a1b      	subs	r3, r3, r0
 80025d2:	40da      	lsrs	r2, r3
 80025d4:	0003      	movs	r3, r0
 80025d6:	3315      	adds	r3, #21
 80025d8:	409d      	lsls	r5, r3
 80025da:	4b0f      	ldr	r3, [pc, #60]	; (8002618 <__aeabi_f2d+0x9c>)
 80025dc:	0312      	lsls	r2, r2, #12
 80025de:	1a1b      	subs	r3, r3, r0
 80025e0:	055b      	lsls	r3, r3, #21
 80025e2:	0b16      	lsrs	r6, r2, #12
 80025e4:	0d5b      	lsrs	r3, r3, #21
 80025e6:	e7d8      	b.n	800259a <__aeabi_f2d+0x1e>
 80025e8:	2d00      	cmp	r5, #0
 80025ea:	d006      	beq.n	80025fa <__aeabi_f2d+0x7e>
 80025ec:	0b32      	lsrs	r2, r6, #12
 80025ee:	2680      	movs	r6, #128	; 0x80
 80025f0:	0336      	lsls	r6, r6, #12
 80025f2:	076d      	lsls	r5, r5, #29
 80025f4:	4316      	orrs	r6, r2
 80025f6:	4b09      	ldr	r3, [pc, #36]	; (800261c <__aeabi_f2d+0xa0>)
 80025f8:	e7cf      	b.n	800259a <__aeabi_f2d+0x1e>
 80025fa:	4b08      	ldr	r3, [pc, #32]	; (800261c <__aeabi_f2d+0xa0>)
 80025fc:	2600      	movs	r6, #0
 80025fe:	e7cc      	b.n	800259a <__aeabi_f2d+0x1e>
 8002600:	2300      	movs	r3, #0
 8002602:	2600      	movs	r6, #0
 8002604:	e7c9      	b.n	800259a <__aeabi_f2d+0x1e>
 8002606:	0003      	movs	r3, r0
 8002608:	002a      	movs	r2, r5
 800260a:	3b0b      	subs	r3, #11
 800260c:	409a      	lsls	r2, r3
 800260e:	2500      	movs	r5, #0
 8002610:	e7e3      	b.n	80025da <__aeabi_f2d+0x5e>
 8002612:	46c0      	nop			; (mov r8, r8)
 8002614:	800fffff 	.word	0x800fffff
 8002618:	00000389 	.word	0x00000389
 800261c:	000007ff 	.word	0x000007ff

08002620 <__clzsi2>:
 8002620:	211c      	movs	r1, #28
 8002622:	2301      	movs	r3, #1
 8002624:	041b      	lsls	r3, r3, #16
 8002626:	4298      	cmp	r0, r3
 8002628:	d301      	bcc.n	800262e <__clzsi2+0xe>
 800262a:	0c00      	lsrs	r0, r0, #16
 800262c:	3910      	subs	r1, #16
 800262e:	0a1b      	lsrs	r3, r3, #8
 8002630:	4298      	cmp	r0, r3
 8002632:	d301      	bcc.n	8002638 <__clzsi2+0x18>
 8002634:	0a00      	lsrs	r0, r0, #8
 8002636:	3908      	subs	r1, #8
 8002638:	091b      	lsrs	r3, r3, #4
 800263a:	4298      	cmp	r0, r3
 800263c:	d301      	bcc.n	8002642 <__clzsi2+0x22>
 800263e:	0900      	lsrs	r0, r0, #4
 8002640:	3904      	subs	r1, #4
 8002642:	a202      	add	r2, pc, #8	; (adr r2, 800264c <__clzsi2+0x2c>)
 8002644:	5c10      	ldrb	r0, [r2, r0]
 8002646:	1840      	adds	r0, r0, r1
 8002648:	4770      	bx	lr
 800264a:	46c0      	nop			; (mov r8, r8)
 800264c:	02020304 	.word	0x02020304
 8002650:	01010101 	.word	0x01010101
	...

0800265c <__clzdi2>:
 800265c:	b510      	push	{r4, lr}
 800265e:	2900      	cmp	r1, #0
 8002660:	d103      	bne.n	800266a <__clzdi2+0xe>
 8002662:	f7ff ffdd 	bl	8002620 <__clzsi2>
 8002666:	3020      	adds	r0, #32
 8002668:	e002      	b.n	8002670 <__clzdi2+0x14>
 800266a:	1c08      	adds	r0, r1, #0
 800266c:	f7ff ffd8 	bl	8002620 <__clzsi2>
 8002670:	bd10      	pop	{r4, pc}
 8002672:	46c0      	nop			; (mov r8, r8)

08002674 <MY_FLASH_EraseSector>:
static uint8_t MY_SectorNum;

//functions definitions
//1. Erase Sector
static void MY_FLASH_EraseSector(void)
{
 8002674:	b580      	push	{r7, lr}
 8002676:	af00      	add	r7, sp, #0
	HAL_FLASH_Unlock();
 8002678:	f005 ff3a 	bl	80084f0 <HAL_FLASH_Unlock>
	//Erase the required Flash sector
	FLASH_PageErase(MY_PageAddrs);
 800267c:	4b04      	ldr	r3, [pc, #16]	; (8002690 <MY_FLASH_EraseSector+0x1c>)
 800267e:	681b      	ldr	r3, [r3, #0]
 8002680:	0018      	movs	r0, r3
 8002682:	f006 f8a7 	bl	80087d4 <FLASH_PageErase>
	HAL_FLASH_Lock();
 8002686:	f005 ff83 	bl	8008590 <HAL_FLASH_Lock>
}
 800268a:	46c0      	nop			; (mov r8, r8)
 800268c:	46bd      	mov	sp, r7
 800268e:	bd80      	pop	{r7, pc}
 8002690:	20000198 	.word	0x20000198

08002694 <MY_FLASH_SetSectorAddrs>:

//2. Set Sector Adress
void MY_FLASH_SetSectorAddrs(uint8_t sector, uint32_t addrs)
{
 8002694:	b580      	push	{r7, lr}
 8002696:	b082      	sub	sp, #8
 8002698:	af00      	add	r7, sp, #0
 800269a:	0002      	movs	r2, r0
 800269c:	6039      	str	r1, [r7, #0]
 800269e:	1dfb      	adds	r3, r7, #7
 80026a0:	701a      	strb	r2, [r3, #0]
	MY_SectorNum = sector;
 80026a2:	4b05      	ldr	r3, [pc, #20]	; (80026b8 <MY_FLASH_SetSectorAddrs+0x24>)
 80026a4:	1dfa      	adds	r2, r7, #7
 80026a6:	7812      	ldrb	r2, [r2, #0]
 80026a8:	701a      	strb	r2, [r3, #0]
	MY_PageAddrs = addrs;
 80026aa:	4b04      	ldr	r3, [pc, #16]	; (80026bc <MY_FLASH_SetSectorAddrs+0x28>)
 80026ac:	683a      	ldr	r2, [r7, #0]
 80026ae:	601a      	str	r2, [r3, #0]

}
 80026b0:	46c0      	nop			; (mov r8, r8)
 80026b2:	46bd      	mov	sp, r7
 80026b4:	b002      	add	sp, #8
 80026b6:	bd80      	pop	{r7, pc}
 80026b8:	2000019c 	.word	0x2000019c
 80026bc:	20000198 	.word	0x20000198

080026c0 <MY_FLASH_WriteN>:

//3. Write Flash
void MY_FLASH_WriteN(uint32_t idx, void *wrBuf, uint32_t Nsize, DataTypeDef dataType)
{
 80026c0:	b580      	push	{r7, lr}
 80026c2:	b088      	sub	sp, #32
 80026c4:	af00      	add	r7, sp, #0
 80026c6:	60f8      	str	r0, [r7, #12]
 80026c8:	60b9      	str	r1, [r7, #8]
 80026ca:	607a      	str	r2, [r7, #4]
 80026cc:	001a      	movs	r2, r3
 80026ce:	1cfb      	adds	r3, r7, #3
 80026d0:	701a      	strb	r2, [r3, #0]
	 uint32_t flashAddress = MY_PageAddrs + idx;
 80026d2:	4b30      	ldr	r3, [pc, #192]	; (8002794 <MY_FLASH_WriteN+0xd4>)
 80026d4:	681b      	ldr	r3, [r3, #0]
 80026d6:	68fa      	ldr	r2, [r7, #12]
 80026d8:	18d3      	adds	r3, r2, r3
 80026da:	61fb      	str	r3, [r7, #28]

	//Erase sector before write
	MY_FLASH_EraseSector();
 80026dc:	f7ff ffca 	bl	8002674 <MY_FLASH_EraseSector>

	//Unlock Flash
	HAL_FLASH_Unlock();
 80026e0:	f005 ff06 	bl	80084f0 <HAL_FLASH_Unlock>
	//Write to Flash
	switch(dataType)
 80026e4:	1cfb      	adds	r3, r7, #3
 80026e6:	781b      	ldrb	r3, [r3, #0]
 80026e8:	2b01      	cmp	r3, #1
 80026ea:	d01b      	beq.n	8002724 <MY_FLASH_WriteN+0x64>
 80026ec:	2b02      	cmp	r3, #2
 80026ee:	d032      	beq.n	8002756 <MY_FLASH_WriteN+0x96>
 80026f0:	2b00      	cmp	r3, #0
 80026f2:	d148      	bne.n	8002786 <MY_FLASH_WriteN+0xc6>
	{
		case DATA_TYPE_8:
				for(uint32_t i=0; i<Nsize; i++)
 80026f4:	2300      	movs	r3, #0
 80026f6:	61bb      	str	r3, [r7, #24]
 80026f8:	e00f      	b.n	800271a <MY_FLASH_WriteN+0x5a>
				{
					HAL_FLASH_Program(FLASH_TYPEPROGRAM_WORD, flashAddress , ((uint8_t *)wrBuf)[i]);
 80026fa:	68ba      	ldr	r2, [r7, #8]
 80026fc:	69bb      	ldr	r3, [r7, #24]
 80026fe:	18d3      	adds	r3, r2, r3
 8002700:	781b      	ldrb	r3, [r3, #0]
 8002702:	001a      	movs	r2, r3
 8002704:	69fb      	ldr	r3, [r7, #28]
 8002706:	0019      	movs	r1, r3
 8002708:	2002      	movs	r0, #2
 800270a:	f005 feb5 	bl	8008478 <HAL_FLASH_Program>
					flashAddress++;
 800270e:	69fb      	ldr	r3, [r7, #28]
 8002710:	3301      	adds	r3, #1
 8002712:	61fb      	str	r3, [r7, #28]
				for(uint32_t i=0; i<Nsize; i++)
 8002714:	69bb      	ldr	r3, [r7, #24]
 8002716:	3301      	adds	r3, #1
 8002718:	61bb      	str	r3, [r7, #24]
 800271a:	69ba      	ldr	r2, [r7, #24]
 800271c:	687b      	ldr	r3, [r7, #4]
 800271e:	429a      	cmp	r2, r3
 8002720:	d3eb      	bcc.n	80026fa <MY_FLASH_WriteN+0x3a>
				}
			break;
 8002722:	e030      	b.n	8002786 <MY_FLASH_WriteN+0xc6>

		case DATA_TYPE_16:
				for(uint32_t i=0; i<Nsize; i++)
 8002724:	2300      	movs	r3, #0
 8002726:	617b      	str	r3, [r7, #20]
 8002728:	e010      	b.n	800274c <MY_FLASH_WriteN+0x8c>
				{
					HAL_FLASH_Program(FLASH_TYPEPROGRAM_WORD, flashAddress , ((uint16_t *)wrBuf)[i]);
 800272a:	697b      	ldr	r3, [r7, #20]
 800272c:	005b      	lsls	r3, r3, #1
 800272e:	68ba      	ldr	r2, [r7, #8]
 8002730:	18d3      	adds	r3, r2, r3
 8002732:	881b      	ldrh	r3, [r3, #0]
 8002734:	001a      	movs	r2, r3
 8002736:	69fb      	ldr	r3, [r7, #28]
 8002738:	0019      	movs	r1, r3
 800273a:	2002      	movs	r0, #2
 800273c:	f005 fe9c 	bl	8008478 <HAL_FLASH_Program>
					flashAddress+=2;
 8002740:	69fb      	ldr	r3, [r7, #28]
 8002742:	3302      	adds	r3, #2
 8002744:	61fb      	str	r3, [r7, #28]
				for(uint32_t i=0; i<Nsize; i++)
 8002746:	697b      	ldr	r3, [r7, #20]
 8002748:	3301      	adds	r3, #1
 800274a:	617b      	str	r3, [r7, #20]
 800274c:	697a      	ldr	r2, [r7, #20]
 800274e:	687b      	ldr	r3, [r7, #4]
 8002750:	429a      	cmp	r2, r3
 8002752:	d3ea      	bcc.n	800272a <MY_FLASH_WriteN+0x6a>
				}
			break;
 8002754:	e017      	b.n	8002786 <MY_FLASH_WriteN+0xc6>

		case DATA_TYPE_32:
				for(uint32_t i=0; i<Nsize; i++)
 8002756:	2300      	movs	r3, #0
 8002758:	613b      	str	r3, [r7, #16]
 800275a:	e00f      	b.n	800277c <MY_FLASH_WriteN+0xbc>
				{
					HAL_FLASH_Program(FLASH_TYPEPROGRAM_WORD, flashAddress , ((uint32_t *)wrBuf)[i]);
 800275c:	693b      	ldr	r3, [r7, #16]
 800275e:	009b      	lsls	r3, r3, #2
 8002760:	68ba      	ldr	r2, [r7, #8]
 8002762:	18d3      	adds	r3, r2, r3
 8002764:	681a      	ldr	r2, [r3, #0]
 8002766:	69fb      	ldr	r3, [r7, #28]
 8002768:	0019      	movs	r1, r3
 800276a:	2002      	movs	r0, #2
 800276c:	f005 fe84 	bl	8008478 <HAL_FLASH_Program>
					flashAddress++;
 8002770:	69fb      	ldr	r3, [r7, #28]
 8002772:	3301      	adds	r3, #1
 8002774:	61fb      	str	r3, [r7, #28]
				for(uint32_t i=0; i<Nsize; i++)
 8002776:	693b      	ldr	r3, [r7, #16]
 8002778:	3301      	adds	r3, #1
 800277a:	613b      	str	r3, [r7, #16]
 800277c:	693a      	ldr	r2, [r7, #16]
 800277e:	687b      	ldr	r3, [r7, #4]
 8002780:	429a      	cmp	r2, r3
 8002782:	d3eb      	bcc.n	800275c <MY_FLASH_WriteN+0x9c>
				}
			break;
 8002784:	46c0      	nop			; (mov r8, r8)
	}
	//Lock the Flash space
	HAL_FLASH_Lock();
 8002786:	f005 ff03 	bl	8008590 <HAL_FLASH_Lock>
}
 800278a:	46c0      	nop			; (mov r8, r8)
 800278c:	46bd      	mov	sp, r7
 800278e:	b008      	add	sp, #32
 8002790:	bd80      	pop	{r7, pc}
 8002792:	46c0      	nop			; (mov r8, r8)
 8002794:	20000198 	.word	0x20000198

08002798 <BSP_sensor_Read>:
void *TEMPERATURE_handle = NULL;
void *PRESSURE_handle = NULL;
#endif

void BSP_sensor_Read(sensor_t *sensor_data)
{
 8002798:	b580      	push	{r7, lr}
 800279a:	b086      	sub	sp, #24
 800279c:	af00      	add	r7, sp, #0
 800279e:	6078      	str	r0, [r7, #4]
  /* USER CODE BEGIN 5 */
  float HUMIDITY_Value = 0;
 80027a0:	2300      	movs	r3, #0
 80027a2:	617b      	str	r3, [r7, #20]
  float TEMPERATURE_Value = 0;
 80027a4:	2300      	movs	r3, #0
 80027a6:	613b      	str	r3, [r7, #16]
  float PRESSURE_Value = 0;
 80027a8:	2300      	movs	r3, #0
 80027aa:	60fb      	str	r3, [r7, #12]
#if defined(SENSOR_ENABLED) || defined (LRWAN_NS1)
  BSP_HUMIDITY_Get_Hum(HUMIDITY_handle, &HUMIDITY_Value);
  BSP_TEMPERATURE_Get_Temp(TEMPERATURE_handle, &TEMPERATURE_Value);
  BSP_PRESSURE_Get_Press(PRESSURE_handle, &PRESSURE_Value);
#endif
  sensor_data->humidity    = HUMIDITY_Value;
 80027ac:	687b      	ldr	r3, [r7, #4]
 80027ae:	697a      	ldr	r2, [r7, #20]
 80027b0:	609a      	str	r2, [r3, #8]
  sensor_data->temperature = TEMPERATURE_Value;
 80027b2:	687b      	ldr	r3, [r7, #4]
 80027b4:	693a      	ldr	r2, [r7, #16]
 80027b6:	605a      	str	r2, [r3, #4]
  sensor_data->pressure    = PRESSURE_Value;
 80027b8:	687b      	ldr	r3, [r7, #4]
 80027ba:	68fa      	ldr	r2, [r7, #12]
 80027bc:	601a      	str	r2, [r3, #0]

  sensor_data->latitude  = (int32_t)((STSOP_LATTITUDE  * MAX_GPS_POS) / 90);
 80027be:	687b      	ldr	r3, [r7, #4]
 80027c0:	4a06      	ldr	r2, [pc, #24]	; (80027dc <BSP_sensor_Read+0x44>)
 80027c2:	60da      	str	r2, [r3, #12]
  sensor_data->longitude = (int32_t)((STSOP_LONGITUDE  * MAX_GPS_POS) / 180);
 80027c4:	687b      	ldr	r3, [r7, #4]
 80027c6:	4a06      	ldr	r2, [pc, #24]	; (80027e0 <BSP_sensor_Read+0x48>)
 80027c8:	611a      	str	r2, [r3, #16]
  sensor_data->Total1 = Total;
 80027ca:	4b06      	ldr	r3, [pc, #24]	; (80027e4 <BSP_sensor_Read+0x4c>)
 80027cc:	681a      	ldr	r2, [r3, #0]
 80027ce:	687b      	ldr	r3, [r7, #4]
 80027d0:	61da      	str	r2, [r3, #28]
  /* USER CODE END 5 */
}
 80027d2:	46c0      	nop			; (mov r8, r8)
 80027d4:	46bd      	mov	sp, r7
 80027d6:	b006      	add	sp, #24
 80027d8:	bd80      	pop	{r7, pc}
 80027da:	46c0      	nop			; (mov r8, r8)
 80027dc:	003e090d 	.word	0x003e090d
 80027e0:	000503ab 	.word	0x000503ab
 80027e4:	20001450 	.word	0x20001450

080027e8 <BSP_sensor_Init>:

void  BSP_sensor_Init(void)
{
 80027e8:	b580      	push	{r7, lr}
 80027ea:	af00      	add	r7, sp, #0
  BSP_HUMIDITY_Sensor_Enable(HUMIDITY_handle);
  BSP_TEMPERATURE_Sensor_Enable(TEMPERATURE_handle);
  BSP_PRESSURE_Sensor_Enable(PRESSURE_handle);
#endif
  /* USER CODE END 6 */
}
 80027ec:	46c0      	nop			; (mov r8, r8)
 80027ee:	46bd      	mov	sp, r7
 80027f0:	bd80      	pop	{r7, pc}
	...

080027f4 <init_gpio_interrupt>:
void init_gpio_interrupt()
{
 80027f4:	b580      	push	{r7, lr}
 80027f6:	b086      	sub	sp, #24
 80027f8:	af00      	add	r7, sp, #0
    GPIO_InitTypeDef initStruct = {0};
 80027fa:	1d3b      	adds	r3, r7, #4
 80027fc:	0018      	movs	r0, r3
 80027fe:	2314      	movs	r3, #20
 8002800:	001a      	movs	r2, r3
 8002802:	2100      	movs	r1, #0
 8002804:	f016 ff80 	bl	8019708 <memset>
    initStruct.Mode = GPIO_MODE_IT_FALLING;
 8002808:	1d3b      	adds	r3, r7, #4
 800280a:	4a15      	ldr	r2, [pc, #84]	; (8002860 <init_gpio_interrupt+0x6c>)
 800280c:	605a      	str	r2, [r3, #4]
    initStruct.Pull = GPIO_PULLDOWN;
 800280e:	1d3b      	adds	r3, r7, #4
 8002810:	2202      	movs	r2, #2
 8002812:	609a      	str	r2, [r3, #8]
    initStruct.Speed = GPIO_SPEED_HIGH;
 8002814:	1d3b      	adds	r3, r7, #4
 8002816:	2203      	movs	r2, #3
 8002818:	60da      	str	r2, [r3, #12]

//    HW_GPIO_Init(USER_BUTTON_GPIO_PORT, USER_BUTTON_PIN, &initStruct);
//    HW_GPIO_SetIrq(USER_BUTTON_GPIO_PORT, USER_BUTTON_PIN, 0, do_when_gpio_interrupted);
    HW_GPIO_Init(GPIOB, GPIO_PIN_12, &initStruct);
 800281a:	1d3a      	adds	r2, r7, #4
 800281c:	2380      	movs	r3, #128	; 0x80
 800281e:	015b      	lsls	r3, r3, #5
 8002820:	4810      	ldr	r0, [pc, #64]	; (8002864 <init_gpio_interrupt+0x70>)
 8002822:	0019      	movs	r1, r3
 8002824:	f000 f9c6 	bl	8002bb4 <HW_GPIO_Init>
    HW_GPIO_SetIrq(GPIOB, GPIO_PIN_12, 0, switch2_interruptFunction);
 8002828:	4a0f      	ldr	r2, [pc, #60]	; (8002868 <init_gpio_interrupt+0x74>)
 800282a:	2380      	movs	r3, #128	; 0x80
